:020000040000FA
:1000000066EFFEF08FEF00F0E9CF0BF1EACF0CF1D5
:10001000D9CF0DF175EFFDF0D8CF2EF0E8CF2FF04E
:10002000E0CF30F0E9CF31F0EACF32F0E1CF33F07A
:10003000E2CF34F0D9CF35F0DACF36F0F3CF37F066
:10004000F4CF38F0F6CF39F0F7CF3AF0F8CF3BF0F5
:10005000F5CF3CF09DA001D001D00AD09EA001D0E8
:1000600001D006D09FB001D001D002D0DAECA3F0CD
:10007000A0A201D001D00AD0A1A201D001D006D007
:10008000A2B201D001D002D053ECEFF09DA401D078
:1000900001D00AD09EA401D001D006D09FB401D0D7
:1000A00001D002D0C0EC23F09DAA01D001D00AD02B
:1000B0009EAA01D001D006D09FBA01D001D002D0B3
:1000C000CDECDEF0A3AA01D001D00AD0A4AA01D0C1
:1000D00001D006D0A5BA01D001D002D022EC26F082
:1000E0003CC0F5FF3BC0F8FF3AC0F7FF39C0F6FF50
:1000F00038C0F4FF37C0F3FF36C0DAFF35C0D9FF90
:1001000034C0E2FF33C0E1FF32C0EAFF31C0E9FF93
:1001100030C0E0FF2FC0E8FF2EC0D8FF100044EF32
:1001200007F0FFFFFFFFFFFFFFFFFFFFFFFFFFFFE6
:10013000FFFFFFFFFFFFFFFFFFFFFFFFFFFFFFFFCF
:10014000FFFFFFFFFFFFFFFFFFFFFFFFFFFFFFFFBF
:10015000FFFFFFFFFFFFFFFFFFFFFFFFFFFFFFFFAF
:10016000FFFFFFFFFFFFFFFFFFFFFFFFFFFFFFFF9F
:100400001F1F1F1B1B1B1B1B13131313131319116C
:10041000130919191919191919191B1D1919190075
:100420000001310391033203920333039303340336
:1004300094033501950139039903360137013801D9
:1004400098010000960144030A0314000101020010
:100450000000DFFF00904A54FE1234000003030046
:100460002228123403010104000A020601000000E0
:100470000F02033C02020800000000000000000020
:100480000909090909117801850140014101880123
:100490008903900370007101696E7465726E6574F2
:1004A0002E6C6D742E6C76000000000000000000C1
:1004B00000000031313131313131310000000000B4
:1004C00000000000000000003932330000323133F8
:1004D0002E32312E3139362E363800000047736DFA
:1004E00054736300000000000000000000000000E2
:1004F00000000000000000000000000000000000FC
:1005000000000000000000000000000000000000EB
:1005100000000000000000000000000000000000DB
:1005200000000000000000000000000000000000CB
:1005300000000000000000000000000000000000BB
:1005400000000000000000000000000000000000AB
:10055000000000000000000000000000000000009B
:10056000000000000000000000000000000000008B
:10057000000000000000000000000000000000007B
:10058000000000000000000000000000000000006B
:10059000000000000000000000000000000000005B
:1005A000000000000000000000000000000000004B
:1005B000000000000000000000000000000000003B
:1005C000000000000000000000000000000000002B
:1005D000000000000000000000000000000000001B
:1005E000000000000000000000000000000000000B
:1005F00000000000000000000000000000000000FB
:1006000000000000000000000000000000000000EA
:1006100000000000000000000000000000000000DA
:1006200000000000000000000000000000000000CA
:1006300000000000000000000000000000000000BA
:1006400000000000000000000000000000000000AA
:10065000000000000000000000000000000000009A
:10066000000000000000000000000000000000008A
:10067000000000000000000000000000000000007A
:10068000000000000000000000000000000000006A
:10069000000000000000000000000000000000005A
:1006A000000000000000000000000000000000004A
:1006B00000000000460145014201430101A0A1A242
:1006C000A3A4A5A6A7A8A9AAABACADAEAF01B0B133
:1006D000B2B3B4B5B6B7B8B9BABBBCBDBEBF01C042
:1006E000C1C2C3C4C5C6C7C8C9CACBCCCDCECFD082
:1006F000D1D2D3D4D5D6D7D8D9DADBDCDDDEDFE072
:10070000E1E2E3E4E5E6E7E8E9EAEBECEDEEEF0051
:1007100000000000000000000000000000000000D9
:10072000696E7465726E6574000000000000000060
:1007300000000000000000000000000000000000B9
:1007400000000000000000000000000000000000A9
:100750000000000000000000000000000000000099
:100760000000000000000000000000000000000089
:100770000000000000000000000000000000000079
:100780000000000000000000000000000000000069
:100790000000000000000000000000000000000059
:1007A0000000000000000000000000000000000049
:1007B0000000000000000000000000000000000039
:1007C0000000000000000000000000000000000029
:1007D0000000000000000000000000000000000019
:1007E0000000000000000000000000000000000009
:1007F00000000000000000000000000000000000F9
:10080000E8CF24F1276B24072451330D8D0EF324F8
:10081000286F130EF420296F28C118F129C119F18E
:10082000E7EC19F0256F266B284B292B2651800AFF
:10083000800F020ED8B4255D07E32651800A800F91
:10084000180ED8B4255D20E31F69206912002829FD
:10085000186F000E2921196FE7EC19F0216F28C1DC
:1008600018F129C119F1E7EC19F0236F2151226F1A
:1008700022513F0A2311D8B4272B2507D8A02607D9
:10088000020E2827000E29232651800A800F010E10
:10089000D8B4255DDCE2020E276505D0F00E206F8E
:1008A000000E1F6F000C2751020A04E12069000EA0
:1008B0001F6F000C2705C8E12069F00E1F6FF00CB8
:1008C0001F6B206B216B02D01B4B1C2B1BC1D9FF54
:1008D0001CC1DAFFDF5033EC2DF0F6E22D0E1BC108
:1008E000D9FF1CC1DAFFDF6202D01F2B07D02B0E0D
:1008F0001BC1D9FF1CC1DAFFDF621FD01B4B1C2BB1
:100900001CD0225113EC2EF004E32251C0EC2EF047
:10091000226F225146EC2EF0D00ED8A0A90E22272D
:10092000203B213BF00E211720510F0B2113F00E1D
:10093000201722512027000E21231BC1D9FF1CC1E3
:10094000DAFF1B4B1C2BDF50226F01012251C7EC39
:1009500028F0D7E21F510DE020C11DF121C11EF189
:100960001D1F1E1F1D4B1E2B1DC11BF11EC11CF187
:10097000120020C11BF121C11CF112001B6B000EE3
:1009800053EC29F01C6F19C115F11AC116F11CC1E5
:1009900017F1FEEC14F002E301011B81040E53EC8D
:1009A00029F01C6F19C115F11AC116F11CC117F1FC
:1009B0003FEC15F002E301011B83080E53EC29F014
:1009C0001C6F19C115F11AC116F11CC117F17CEC8D
:1009D00014F002E301011B850C0E53EC29F01C6F8F
:1009E00019C115F11AC116F11CC117F1BDEC14F0B3
:1009F00002E301011B87100E53EC29F01C6F19C193
:100A000015F11AC116F11CC117F180EC15F002E3C3
:100A100001011B891C0E53EC29F01C6F19C115F143
:100A20001AC116F11CC117F1C1EC15F002E3010166
:100A30001B8B01011B511200F90E0101176F330EC0
:100A4000166F010E28EC1DF02C0EA7EC2DF0060100
:100A5000A4510FE0220EA7EC2DF0060E0101176F36
:100A6000A40E166F000E28EC1DF0220EA7EC2DF040
:100A700006D0220EA7EC2DF0220EA7EC2DF02C0EA6
:100A8000A7EC2DF0220EA7EC2DF00501D75108E0C0
:100A9000050E0101176FD70E166F000E28EC1DF022
:100AA000220EA7EC2DF02C0EA7EC2DF0220EA7ECB9
:100AB0002DF00501E05108E0050E0101176FE00E71
:100AC000166F000E28EC1DF0220EA7EC2DF0F20E92
:100AD0000101176F880E166F000E28EC1DF00D0E29
:100AE000A7EC2DF0130E01012A6F880E296FBAEFC3
:100AF00021F000010FB608D020EE03F01E50D926D9
:100B00001F50DA22030EDF1649D803E13FD8D8B4CC
:100B10001200020E3EEC2AF000010FA60AD020EED1
:100B200008F01E50D9261F50DA22DF503EEC2AF082
:100B300024D020EE05F01E50D9261F50DA22DF3ACD
:100B400020EE05F01E50D9261F50DA2210EE05F0D7
:100B50001E50E1261F50E222E750206ED89020322E
:100B6000D8902030030BDF6E20EE05F01E50D92602
:100B70001F50DA22DF503EEC2AF010D83EEC2AF06B
:100B800005D83EEC2AF000010D88120020EE02F09C
:100B90001E50D9261F50DA22DF50120020EE03F03B
:100BA0001E50D9261F50DA22DF501200E8CF27F15D
:100BB000000112BA02D0D890120005C315F101014C
:100BC00027515BEC2BF0F7E30301E751070AF3E150
:100BD000330EE725D96EDA6A030EDA22DF6A360EA3
:100BE0000101256F030E266F25C11BF126C11CF1E3
:100BF00060EC04F01BC128F11CC129F128C11FF1D0
:100C000029C120F11CEC29F0D6E30A980A960B9032
:100C1000089C02014C6B08BA8A9C069C468417A863
:100C20000FD0020E0101166FDD0E156F32EC06F0CB
:100C3000186B540E176F2F0E196F84EC1FF00ED027
:100C4000020E0101166FDD0E156F32EC06F0186B07
:100C5000540E176F0F0E196F84EC1FF000014694AD
:100C6000D880120013B6118012AA1AD001011551B2
:100C7000220A161110E01551260A16110CE0155122
:100C80002A0A161108E015512E0A161104E0155112
:100C9000360A161105E1088C08BA8A8C5CC24CF23F
:100CA000130E0101B6652BD0B6071C6B17D0D89078
:100CB0001C35176F020E01011725D96EDA6A050E71
:100CC000DA221C51020D000EF324E16EE26A050ED9
:100CD000E222DECFE6FFDDCFE5FF1C2BB6C117F128
:100CE000186B1CC119F11A6B19BF1A071A51800A27
:100CF0001B6F1751195D1851800A1B59D8E3B65163
:100D0000020D000EF324D96EDA6A050EDA22010113
:100D100015C1DEFF16C1DDFFB62B1200F30E010177
:100D2000176F500E166F010E28EC1DF0060E010114
:100D3000176FA40E166F000E28EC1DF0220EA7EC04
:100D40002DF00D0EA7EC2DF0130E01012A6F880E69
:100D5000296FBAEC21F0F10E0101176FD30E166F57
:100D6000010E28EC1DF0130E01012A6F880E296F69
:100D7000BAEC21F0F10E0101176FEB0E166F010EA8
:100D800028EC1DF0130E01012A6F880E296FBAECB2
:100D900021F0F20E0101176FA00E166F010E28EC64
:100DA0001DF0130E01012A6F880E296FBAEC21F095
:100DB000F20E0101176F8B0E166F010E28EC1DF05D
:100DC000130E01012A6F880E296FBAEC21F01CEF77
:100DD00005F002014E51BAEC2DF01F6F750E0101A6
:100DE0004CD81E6F1EAF1200750E1F25D96EDA6A21
:100DF000050EDA22DF2A750E40D81E6F3F0E1E1731
:100E0000030E1E5D02E38F801280750E010135D83E
:100E10003F0B050A09E1530E0201A06F300EA16FCE
:100E200001011F5197EC23F0750E01011F25D96EAA
:100E3000DA6A0501050EDA22DF503F0B3F0AD8A41B
:100E40001200530E0201A06F200EA16F01011F516D
:100E500097EC23F0750E01011F25D96EDA6A050E95
:100E6000DA22DF6A960E1F25176F186B020E182301
:100E7000750E03D8196F84EF1FF01F25D96EDA6A3B
:100E8000050EDA22DF50120004EE00F0D60EEE6AF4
:100E9000E806FDE10AEE00F0F00EEE6AE806FDE17C
:100EA00009EE00F0F00EEE6AE806FDE108EE00F053
:100EB000F00EEE6AE806FDE107EE00F0F00EEE6AD5
:100EC000E806FDE106EE00F010EEFFF0EE6AE550F8
:100ED000E150FCE1E250FAE105EE00F0F10EEE6ABD
:100EE000E806FDE103EE00F0FE0EEE6AE806FDE125
:100EF00002EE00F0B80EEE6AE806FDE101EEA1F0A8
:100F00001F0EEE6AE806FDE100EEE9F0170EEE6A4C
:100F1000E806FDE100EE01F01C0EEE6AE806FDE1D8
:100F200000EE3DF0090EEE6AE806FDE104EED6F0B3
:100F3000280EEE6AE806FDE100010DEF8DF013B614
:100F4000118012AA19D01D50220A1E1010E01D5047
:100F5000260A1E100CE01D502A0A1E1008E01D5023
:100F60002E0A1E1004E01D50360A1E1005E1088CE2
:100F700008BA8A8C5CC24CF2130E0101B6652BD004
:100F8000B607246A16D0D89024341F6E020E1F2490
:100F9000D96EDA6A050EDA222450020D000EF3240F
:100FA000E16EE26A050EE222DECFE6FFDDCFE5FF6D
:100FB000242A0101B6C11FF0206A24C021F0226A50
:100FC00021BE22062250800A236E1F50215C205031
:100FD000800A2358D8E3B651020D000EF324D96ECF
:100FE000DA6A050EDA221DC0DEFF1EC0DDFF010138
:100FF000B62B12003D6B50D83D512225186F000EC4
:101000002321196FE7EC19F0DF6E46D8DF5004E0BA
:101010003D2B100E3D65EFD72A5107E02351020A00
:10102000410ED8B4221901E0198001013B6B2A510D
:101030002B0A03E1010E3B6F3D07B85109E0B8519F
:101040003D5D3C6F3C51800A7F0F02E33C513B27E2
:101050002A0E266F010E276F3B512627000E2723ED
:1010600026C11BF127C11CF1220E286F030E296F28
:1010700024512827000E292328C11DF129C11EF162
:1010800025C11FF1206BD5EC11F01C511B1102E1A1
:10109000D8801200D89012002A0E3D25D96EDA6A47
:1010A000010EDA22120020EE01F01E51D9261F5146
:1010B000DA22DF50156F166BC8EC0FF015C124F162
:1010C00016C125F120EE04F02451D9262551DA224B
:1010D000DF50206F20EE03F02451D9262551DA226B
:1010E000DF50216F2139F00B2011226F20EE02F02A
:1010F0001E51D9261F51DA22DF50CFEC26F0236F84
:1011000020EE02F01E51D9261F51DA2223C120F110
:10111000203B0F0E20171EC1E1FF1FC1E2FFE75069
:10112000F00B2011DF6E20EE01F01E51D9261F5169
:10113000DA2210EE02F02451E1262551E222E75096
:10114000206F2339F00B2011DF6E1EC1D9FF1FC1A4
:10115000DAFF22C1DFFF1200E8CF2BF1FE0E176F7E
:10116000820E166F010E28EC1DF03D0EA7EC2DF03F
:1011700001012BC115F1166BC8EC0FF015C12DF153
:1011800016C12EF120EE03F02D51D9262E51DA2270
:10119000DF5057EC2EF0A7EC2DF0010120EE04F00B
:1011A0002D51D9262E51DA22DF5057EC2EF0A7EC24
:1011B0002DF00D0EA7EC2DF0EAEC2FF001012C6BB9
:1011C00019D0BDEC2FF016E3EEEC2FF001012F6FDC
:1011D0000DD02F519EEC2BF00DE301012C2B0AD0EA
:1011E0002F5172EC2BF0D8B0120004D02C51F1E04A
:1011F000010AF6E0D2EC2FF0D10E0101295D070EB5
:101200002A59D8B01200DDD717C1D9FF18C1DAFFAB
:10121000DF500001F25FF251D8B41200010120EE5C
:1012200001F01751D9261851DA22000EDF6E32D0A4
:1012300017C1D9FF18C1DAFFDF5034D81AC1D9FF5E
:101240001BC1DAFF10EE02F01751E1261851E2221D
:10125000DFCFE7FF20EE02F01751D9261851DA222E
:1012600010EE01F01751E1261851E222E7501AD88A
:101270001AC1E1FF1BC1E2FFDFCFE7FF20EE01F063
:101280001751D9261851DA22DF2A17C1D9FF18C100
:10129000DAFFDF2A17C1D9FF18C1DAFF3F0EDF647A
:1012A000C7D73F0C196F195115251A6FE86A19BF76
:1012B000E86816211B6F1200236A000E56EC2AF014
:1012C000246E21C01DF022C01EF024C01FF083EC4C
:1012D00016F0D8B02380040E56EC2AF0246E21C0FC
:1012E0001DF022C01EF024C01FF001EC17F0D8B092
:1012F0002382080E56EC2AF0246E21C01DF022C075
:101300001EF024C01FF0FDEC17F0D8B023840C0EA3
:1013100056EC2AF0246E21C01DF022C01EF024C01D
:101320001FF0BEEC17F0D8B02386100E56EC2AF052
:10133000246E21C01DF022C01EF024C01FF07FECDF
:1013400017F0D8B023881C0E56EC2AF0246E21C06A
:101350001DF022C01EF024C01FF040EC17F0D8B0E2
:10136000238A2350120020EE01F01E51D9261F516E
:10137000DA22DF50156F166BC8EC0FF015C124F19F
:1013800016C125F120EE04F02451D9262551DA2288
:10139000DF50206F20EE03F02451D9262551DA22A8
:1013A000DF50216F2139F00B2011226F20EE02F067
:1013B0001E51D9261F51DA22DF50236F20EE02F092
:1013C0001E51D9261F51DA2223C120F1203B0F0ED6
:1013D00020171EC1E1FF1FC1E2FFE750F00B2011F3
:1013E000DF6E20EE01F01E51D9261F51DA2210EED9
:1013F00002F02451E1262551E222E750206F2339E3
:10140000F00B2011DF6E1EC1D9FF1FC1DAFF22C110
:10141000DFFF1200E8CF4DF102C315F14D515BEC37
:101420002BF002E2D89012000301E751070AFAE11B
:10143000330EE725D96EDA6A030EDA22DF6A360E3A
:101440000101486F030E496F48C11BF149C11CF1EE
:1014500060EC04F01BC14AF11CC14BF14AC11FF101
:101460004BC120F11CEC29F0DDE300011CB002D0DF
:1014700000010E808DECF3F001014D39F00B4C6F43
:10148000800E2F6F4C5112ECE5F02FC14AF130C1A4
:101490004BF1030102516BEC2FF002E2D8801200F5
:1014A0004D51B6EC2AF04C6F4AC139F14BC13AF1BB
:1014B0004DC13BF14CC13CF1030E3D6FC5EC1DF03D
:1014C000EDD73251C0EC22F047D8320502E1280EA8
:1014D0000AD03251020AFBE03251030AF8E03251DD
:1014E000040AF5E0020E356F3551365D1AE3F30E4E
:1014F000176FA60E166F000E28EC1DF008ECD7F043
:1015000068EC9EF032C118F1000E1EEC12F0325160
:10151000C0EC22F021D8500E206FE00E1F6FE6ECD9
:1015200021F037C1D9FF38C1DAFFDF2A010132517A
:101530006AEC22F015C133F116C134F13651020DB7
:10154000F3503325D96E000E3421DA6E30C1DEFF40
:1015500031C1DDFFD880120015C137F116C138F155
:1015600037C1D9FF38C1DAFFDF50366F12002FC103
:1015700074F130C175F139D0C00E7425316FFF0E92
:101580007521326F3251800A800F010ED8B4315D5F
:1015900014E3766B2FD87651800A400FFBE333D8E3
:1015A000400E2A6F8BEC26F0400E2D27000E2E23C6
:1015B000C00E7427FF0E752318D0766B01D01AD891
:1015C00076C131F1326B31BF32073251800A336F4D
:1015D0007451315D7551800A3359F1E314D874C1E7
:1015E0002AF18BEC26F0746B756B75517411D8B4BD
:1015F0001200C2D7340E7625D96EDA6A010EDA22CD
:10160000DF68762B12002DC126F12EC127F1010EC5
:10161000296F340E286F12000101BC511F0B02E02C
:10162000149201D0148202014B2B4B513E0A06E169
:101630004B6B0001468471ECE0F046940101B50566
:1016400007E10001F96702D002EF2EF0F90712005E
:10165000B551020A0FE10001F967F8D70201922B98
:101660009251080AF1E1926B179C8B9C960E000137
:10167000F96F960C00010BB0120006AC0CD0000103
:10168000F967E4D70201922B9251060ADDE1926BD1
:10169000179C8B8CEBD714A204D000010C908B8C80
:1016A00012000CA00AD002017A5107E00001F9678C
:1016B000CDD702017A0702EF2EF000010C908B9C2F
:1016C0001200E8CF4DF103C315F14D515BEC2BF047
:1016D00002E2D89012000301E751070AFAE1330E43
:1016E000E725D96EDA6A030EDA22DF6A360E0101C7
:1016F000486F030E496F48C11BF149C11CF160ECF2
:1017000004F01BC14AF11CC14BF14AC11FF14BC18E
:1017100020F11CEC29F0DDE300010D8E8DECF3F0DF
:1017200001014D39F00B4C6F840E2F6F4C5112ECB0
:10173000E5F02FC14AF130C14BF1030103516BECCD
:101740002FF002E2D88012004D51B6EC2AF04C6F17
:101750004AC139F14BC13AF14DC13BF14CC13CF1A9
:10176000030E3D6FC5EC1DF0EDD70101186B196B31
:101770000BD047D8240EDF6203D00101192B04D00F
:1017800040D8DF50181BF9D73CD8DF50F2E1330EB8
:101790001925D96EDA6A030EDA222A0EDF6E19C114
:1017A00016F1176B16BF1707340E1625D96E030EE8
:1017B0001721DA6E18390F0B18BFF00957EC2EF00D
:1017C000DF6E19C116F1176B16BF1707350E010131
:1017D0001625D96E030E1721DA6E18510F0B57EC30
:1017E0002EF0DF6E19C116F1176B16BF1707360EF4
:1017F00001011625D96E030E1721DA6E000EDF6E79
:10180000000C330E01011925D96EDA6A030EDA22B3
:101810001200E8CF4DF136C515F14D515BEC2BF0C0
:1018200002E2D89012000301E751070AFAE1330EF1
:10183000E725D96EDA6A030EDA22DF6A360E010175
:10184000486F030E496F48C11BF149C11CF160ECA0
:1018500004F01BC14AF11CC14BF14AC11FF14BC13D
:1018600020F11CEC29F0DDE38DEC21F08DECF3F0A0
:1018700001014D39F00B4C6F150E2F6F4C5112ECCE
:10188000E5F02FC14AF130C14BF1050136516BEC47
:101890002FF002E2D88012004D51B6EC2AF04C6FC6
:1018A0004AC139F14BC13AF14DC13BF14CC13CF158
:1018B000030E3D6FC5EC1DF0EDD70A0E236FA00E91
:1018C000226F256B48D02307B36B64EC2CF0010129
:1018D000225199EC27F00101B3672FD0185199ECF0
:1018E00027F00101175199EC27F00101246B1DD05D
:1018F00024511925D96E000E1A21DA6EDF5099ECA9
:1019000027F00101252BC00E1715206F1851216FEC
:10191000174B182BC00E17151C6F18511D6F21196E
:1019200002E120511C1904E1242B1B51245DE0E34A
:10193000D7EC29F0010125511200070E1F6FD00EC0
:101940001E6F01D000F001011E07D8A01F071E293D
:10195000D8B41F29F7E12351800A7F0FEBE3B3D7F7
:10196000080E0401CB6F0401C5610CD0C5C4CBF4D3
:101970000401BF0502E1020EBF6F0401BF6702D080
:10198000010EBF6F040104930491CBC405F404015C
:10199000CB510401C55DC56F040E0401CA6F280E4A
:1019A000C96F0401C4A11DD022D0C2C4F6FFC3C4B4
:1019B000F7FF000EF86EC9C4D9FFCAC4DAFF0F0ED4
:1019C000F76403D00800F55005D0F6CFE9FFF7CF54
:1019D000EAFFEF50DF6E0401C24BC32B0401C94B79
:1019E000CA2B0401CB07CB29D8B41200DED7C2C45E
:1019F000C7F4C3C4C8F413EC27F0C7C4C2F4C8C406
:101A0000C3F41200080E0401CB6F0401C5610CD0B1
:101A1000C5C4CBF40401BF0502E1020EBF6F04018F
:101A2000BF6702D0010EBF6F040104930491CBC4C1
:101A300005F40401CB510401C55DC56F040E04011A
:101A4000CA6F280EC96F0401C4A11DD022D0C2C420
:101A5000F6FFC3C4F7FF000EF86EC9C4D9FFCAC4AD
:101A6000DAFF0F0EF76403D00800F55005D0F6CF6B
:101A7000E9FFF7CFEAFFEF50DF6E0401C24BC32B43
:101A80000401C94BCA2B0401CB07CB29D8B41200DF
:101A9000DED7C2C4C7F4C3C4C8F435EC27F0C7C44A
:101AA000C2F4C8C4C3F41200E8CF4FF1000105BC72
:101AB00002D0D890120039C515F101014F515BECED
:101AC0002BF0F7E3040E0301E76101D0F2D723EE18
:101AD000E7F0050EDF6401D0ECD78DECF3F00101E7
:101AE0004F39F00B466F180E2F6F465112ECE5F090
:101AF000080E0101476F0301E751040A09E134515F
:101B0000BAEC2DF0486F35C349F136C34AF111D014
:101B10003551BAEC2DF0446F03013451BAEC2DF07D
:101B2000456F4539F00B4411486F36C349F137C34F
:101B30004AF14B6B4C6B4D6B4E6B010E176F470EA2
:101B4000166F88EC2BF0D8801200050E356F02015D
:101B50002F512E1105E1FEEC25F03FE3D880120055
:101B60002EC233F12FC234F10101315133273251EA
:101B700034233451800A7D0FE90ED8B4335D2DE350
:101B800002012E6B2F6BB9EC18F023E3E7D7E7ECDB
:101B9000FBF014E2FEEC25F0E1E22FC116F130C1BA
:101BA00017F1000E28EC1DF00101315102012E2722
:101BB0000101325102012F23D8901200EAEC2FF0DC
:101BC000D2EC2FF0890E0101295D130E2A59F8E39A
:101BD000350701013567DBD7C1D72FC116F130C1F9
:101BE00017F1000E28EC1DF0DFD7FD0E0101176F75
:101BF000830E166F010E28EC1DF008ECD7F068EC90
:101C00009EF00101306F05018551800A500F04E3F9
:101C10008551800A460F12E3010130510C0A0EE093
:101C20003051090A0BE0880E296F130E2A6F2B6BB7
:101C30002C6B010E2D6F68EC9EF0E3D70101305143
:101C40000C0A03E13051090A1DE0306B850E0101D9
:101C50003025D96EDA6A050EDA22D60E3025E16E0D
:101C6000E26A040EE222DFCFE7FF302B3051800A18
:101C7000710FECE3130E2A6F880E296FBAEC21F076
:101C8000D8901200D88012000101706BB0390F0B90
:101C9000506F516B50510F0B57EC2EF06B6F3BD8C0
:101CA000B0510F0B57EC2EF0DF6E35D8AF390F0B5C
:101CB00057EC2EF0DF6E2FD8AF510F0B57EC2EF0F4
:101CC000DF6E29D8DF6A010E226F520E216FFC0EE3
:101CD000246F9A0E236F060E0101266FDF0E256F0B
:101CE000010E286F6B0E276FEBECD8F02151706F4F
:101CF000520E7025D96EDA6A010EDA22DF6A2C6F75
:101D0000520E2B6F000E2E6B2D6BD1ECEBF001E21F
:101D1000000C07EFF2F0702B6B0E7025D96EDA6AAB
:101D2000010EDA221200000108BE1200010E1EC0D0
:101D3000D9FF1FC0DAFFDF6204D0060E3EEC2AF0A6
:101D400003D0070E3EEC2AF020EE02F033D820EE4E
:101D500001F01E5024D83EEC2AF020EE05F02AD8DF
:101D6000203A0F0E2016201620EE03F01E5017D832
:101D70003EEC2AF020EE05F01DD82038F00B226E44
:101D800022503EEC2AF020EE04F01E50D9261F50BF
:101D9000DA22DF503EEC2AF000010D881200D9262D
:101DA0001F50DA22DF50216E2138F00B2010226EF6
:101DB000225012001E50D9261F50DA22DF50206E0A
:101DC00012006598080E0401016F0401C4BF1BD006
:101DD0000401C1510EE0020E0401C06F0401056B45
:101DE000C80E046F040E036F280E026FC80E006F3A
:101DF000C80C040E0401036F200E026F8C0E006FDE
:101E0000840E046F840C0401C151D8A41200040193
:101E100020AFE1D70401C5510401265D000E27590A
:101E2000D8A026C4C5F402EC0DF0010E0401C06F69
:101E3000040E0401036F200E026F800E006F080E67
:101E4000016F040E036F200E026F800E006F040EF0
:101E5000076F280E066FC80E046FC80C6598080E31
:101E60000401016F0401C4BF1BD00401C1510EE085
:101E7000020E0401C06F0401056BC80E046F040E4E
:101E8000036F280E026FC80E006FC80C040E040109
:101E9000036F200E026F8C0E006F840E046F840C93
:101EA0000401C151D8A41200040120AFE1D70401FC
:101EB000C5510401265D000E2759D8A026C4C5F4DB
:101EC000B0EC0CF0010E0401C06F040E0401036FAE
:101ED000200E026F800E006F080E016F040E036F5C
:101EE000200E026F800E006F040E076F280E066F23
:101EF000C80E046FC80CE8CF25F01A9225B21A82DA
:101F000000010BA008D025A21200000117AA1200A0
:101F1000000107841200000106AC120000010AB89B
:101F2000120000010AA613D000F025A208D01E6AF4
:101F3000260E1D6E9FEC07F000011A8012001E6A2B
:101F4000280E1D6E9FEC07F000011A90120025A2CA
:101F500012000A8817A804D0020169C228F203D02F
:101F6000020168C228F2296B283B293BF00E291791
:101F700028510F0B2913F00E281729512811D8A426
:101F800012000A980A861E6A260E1D6E9FEF07F041
:101F90000101010E186F190E176F196B1A6B1B6B6D
:101FA0001C6B1D6B100E155D270E16590AE3192BBD
:101FB000100E155F270E165B100E155D270E1659B5
:101FC000F6E2E80E155D030E16590AE31A2BE80E29
:101FD000155F030E165BE80E155D030E1659F6E24B
:101FE000640E155D000E16590AE31B2B640E155F77
:101FF000000E165B640E155D000E1659F6E20A0E11
:10200000155D000E16590AE31C2B0A0E155F000E13
:10201000165B0A0E155D000E1659F6E215C11DF18C
:1020200017C115F118C116F11200E8CF4BF119B024
:1020300009D001014B5103E04B51050A03E1010EA8
:102040004B6F118229C515F101014B515BEC2BF04F
:1020500002E2D8901200000111A20CD011920101ED
:102060002B6B010E2C6F050EBDECBFF0F2E3050EDD
:1020700001014B6F8DECF3F001014B39F00B4A6F0E
:102080008D0E2F6F4A5112ECE5F02FC148F130C18F
:1020900049F1050129516BEC2FF002E2D8801200C2
:1020A0004B51B6EC2AF04A6F48C139F149C13AF1B7
:1020B0004BC13BF14AC13CF1030E3D6FC5EC1DF035
:1020C000EDD7040120511F0B0101156F1505D8A490
:1020D000120004012039E832030B0101156F1505C8
:1020E000D8A41200040124512AE02405D8A4120027
:1020F00026D0040E0401C36FB50EC26F080EC56F63
:10210000C4810401C48F1200040E0401C36FB50E14
:10211000C26FF7D7010E0401C16F010C040E040158
:10212000C36FCE0EC26F070EC56F810EC46F810CD8
:1021300022C4CCF40401CC8F0401C48F120004012A
:102140002151D7E0010AE0E0210AE4E0010AE6E0DB
:10215000030AD8A41200ECD7040120511F0B01017F
:10216000006F0005D8A4120004012039E832030BE7
:102170000101006F0005D8A41200040124512AE0D7
:102180002405D8A4120026D0040E0401C36FB50E96
:10219000C26F080EC56FC4810401C48F1200040E03
:1021A0000401C36FB50EC26FF7D7010E0401C16FF2
:1021B000010C040E0401C36FCE0EC26F070EC56F73
:1021C000810EC46F810C22C4CCF40401CC8F0401B5
:1021D000C48F120004012151D7E0010AE0E0210A76
:1021E000E4E0010AE6E0030AD8A41200ECD70401F7
:1021F0002039E832030BD8A412002ED00401C48F7A
:10220000080E0401CD6F080CAEEF24F0E7EF1BF0D1
:10221000040E0401C36FBD0EC26F0401C481010E20
:10222000C56FC48F010C02EF16F00AEFF4F0BE0E7A
:102230000101036F040E046F0401245101010327FF
:10224000000E042303C1C2F404C1C3F4E6D70401A1
:10225000C48F22C4BEF4120004012151E4E0010A3B
:10226000E4E0020AE2E0060AC9E0030ACDE00E0A51
:10227000CFE0010ACBE0030ADAE0010AD8A4120099
:10228000E6D73DD022C11BF123C11CF124C11DF1B1
:1022900025C11EF124C115F125C116F103EC21F071
:1022A00015C11FF116C120F1D5EC11F01C511B1105
:1022B00005E122C122F123C123F112002229156F69
:1022C000000E2321166F24C1F6FF25C1F7FF000E73
:1022D000F86E0F0EF76403D00800F55005D0F6CF66
:1022E000E9FFF7CFEAFFEF500101176F186B17BF37
:1022F000180744EC2BF015C122F116C123F123512C
:10230000221106E022C1D9FF23C1DAFFDF50BAE172
:10231000226B236B120004012039E832030BD8A48E
:1023200012002ED00401C48F080E0401CD6F080CDA
:10233000D4EF24F01DEF1CF0040E0401C36FBD0E9A
:10234000C26F0401C481010EC56FC48F010CEFEF91
:1023500012F0ABEFF7F0BE0E0101186F040E196F0B
:102360000401245101011827000E192318C1C2F4D9
:1023700019C1C3F4E6D70401C48F22C4BEF412000D
:1023800004012151E4E0010AE4E0020AE2E0060A65
:10239000C9E0030ACDE00E0ACFE0010ACBE0030A50
:1023A000DAE0010AD8A41200E6D735D01BC1D9FF64
:1023B0001CC1DAFFDF5013E039D8F76403D00800FE
:1023C000F55005D0F6CFE9FFF7CFEAFFEF50010156
:1023D000216F1BC1D9FF1CC1DAFFDF1818E01BC138
:1023E000D9FF1CC1DAFFDF50216F20D8F76403D07A
:1023F0000800F55005D0F6CFE9FFF7CFEAFFEF5020
:102400000101215D1B6F1C6BD8A01C0712001B4B28
:102410001C2B1D4B1E2B1F07D8A0200701011F29B5
:10242000D8B42029C3E11B6B1C6B12001DC1F6FF41
:102430001EC1F7FF000EF86E0F0E1200E8CF1CF160
:1024400001011851C0EC22F015C11DF116C11EF199
:102450001DC1D9FF1EC1DAFFDF50216F216701D0F6
:10246000120018516AEC22F015C11FF116C120F1BB
:102470001DC1D9FF1EC1DAFFDF50DF06216F1CC16D
:1024800022F11ED0D8902235196F19511F251A6FCD
:10249000E86A19BFE86820211B6F020E1A25D96E61
:1024A000000E1B21DA6E2251020DF3501F25E16E42
:1024B000000E2021E26EDECFE6FFDDCFE5FF222B0E
:1024C0002151225DD8B01200DDD733D01DC0D9FF15
:1024D0001EC0DAFFDF5012E036D8F76403D00800E0
:1024E000F55005D0F6CFE9FFF7CFEAFFEF50236EA6
:1024F0001DC0D9FF1EC0DAFFDF1817E01DC0D9FFCD
:102500001EC0DAFFDF50236E1ED8F76403D0080028
:10251000F55005D0F6CFE9FFF7CFEAFFEF50235C87
:102520001D6E1E6AD8A01E0612001D4A1E2A1F4AD2
:10253000202A2106D8A022062128D8B42228C6E1C4
:102540001D6A1E6A12001FC0F6FF20C0F7FF000EB2
:10255000F86E0F0E1200190E1D6E280EC26EC2808C
:102560001D061D28FDE1C282320E1D6E1D061D28AE
:1025700002E0C2B2FBD7C4CF1EF0C26A280E1E60B2
:1025800007D00201572B020E5765020CFF00020C08
:1025900002015B511E5C0FE3586B576B5A2B770E91
:1025A0005A65770C5A6B07980796000107AE120020
:1025B000078C079E12001E50595DD8A012005A6B5E
:1025C000576B582B3B0E020158653B0C586B078824
:1025D000078E000107B61200078A07861200040161
:1025E000286B296B24D00401C48F040128810401C5
:1025F000C65125E00401288322D00401C48F1FD0D6
:102600000401C48F0BEC2DF025D8F76403D008002B
:10261000F55005D0F6CFE9FFF7CFEAFFEF50010103
:10262000156F15A50CD0010E0401286F08D0040108
:1026300020511F0BD8E0010AE0E0030AE1E00401A9
:10264000C4AF1200040EC36F280EC26FC481020E05
:10265000C56F020CC7C4F6FFC8C4F7FF000EF86EC2
:102660000F0E1200E8CF25F00001FA670AD025A06E
:1026700003D01E6A220E02D01E6A240E1D6E9FEF2A
:1026800007F0FA0522E10AA803D0199C25B0198C9D
:1026900000010AB8120017A803D0000119BE1200E9
:1026A000000106AC120025A008D01E6A220E1D6E85
:1026B0009FEC07F00001198A12001E6A240E1D6E9D
:1026C0009FEC07F00001199A1200FA51020AD8A4EF
:1026D000120017A803D0000119BE1200000106ACB9
:1026E000120025B0E2D7E9D70201346B356BFC0E3E
:1026F0000101176FBD0E166F010E28EC1DF008ECDE
:10270000D7F068EC9EF00101306F880E296F130E30
:102710002A6F2B6B2C6B010E2D6F68EC9EF0010164
:102720003051180AD8B412003051160AD8B4120029
:1027300030511A0AD8B4120030511B0AD8B4120012
:102740003051170AD8B41200EAEC2FF0D2EC2FF077
:10275000D10E0101295D070E2A59F8E3780E020116
:10276000345D000E3559D8B01200C1D7E8CF25F03E
:102770000001FB670AD025A403D01E6A2A0E02D0EE
:102780001E6A2C0E1D6E9FEF07F0FB0522E10AA8C2
:1027900003D01A9625B41A8600010AB8120017A8A9
:1027A00003D000011AB81200000106AC120025A4E3
:1027B00008D01E6A2A0E1D6E9FEC07F000011A84D5
:1027C00012001E6A2C0E1D6E9FEC07F000011A9479
:1027D0001200FB51020AD8A4120017A803D000016E
:1027E0001AB81200000106AC120025B4E2D7E9D7EE
:1027F000E8CF25F00001FD670AD025A803D01E6AA6
:10280000360E02D01E6A380E1D6E9FEF07F0FD05D2
:1028100022E10AA803D01B9225B81B8200010AB846
:10282000120017A803D000011BB41200000106AC6F
:10283000120025A808D01E6A360E1D6E9FEC07F008
:1028400000011B8012001E6A380E1D6E9FEC07F0FF
:1028500000011B901200FD51020AD8A4120017A813
:1028600003D000011BB41200000106AC120025B811
:10287000E2D7E9D7E8CF25F00001FC670AD025A60A
:1028800003D01E6A2E0E02D01E6A300E1D6E9FEF00
:1028900007F0FC0522E10AA803D01A9C25B61A8C81
:1028A00000010AB8120017A803D000011ABE1200D6
:1028B000000106AC120025A608D01E6A2E0E1D6E61
:1028C0009FEC07F000011A8A12001E6A300E1D6E7E
:1028D0009FEC07F000011A9A1200FC51020AD8A4DA
:1028E000120017A803D000011ABE1200000106ACA6
:1028F000120025B6E2D7E9D712BA0AAA24D0180ED8
:102900000101176503D03C0E176502D0018801D084
:10291000019829D824E00201144B152B010115510F
:102920000201145D01011651020115590AE300016B
:10293000019A01B8018A01BA02D0D8901200D88059
:1029400012000001F8D73E0E0101176102D0019874
:1029500004D04C0E176501D0018805D8DCE10201D6
:10296000146B156BEED7010E01A8000E0101186F54
:10297000010E01AA000E181B120012BA0AAA24D0D6
:10298000180E0101176503D03C0E176502D0018CAB
:1029900001D0019C29D824E00201164B172B01011C
:1029A00015510201165D01011651020117590AE382
:1029B0000001019E01BC018E01BE02D0D890120020
:1029C000D88012000001F8D73E0E0101176102D035
:1029D000019C04D04C0E176501D0018C05D8DCE1B8
:1029E0000201166B176BEED7010E01AC000E010150
:1029F000186F010E01AE000E181B120012BA0AAABF
:102A000024D0180E0101176503D03C0E176502D0C3
:102A1000018001D0019029D824E00201104B112B34
:102A2000010115510201105D0101165102011159F8
:102A30000AE30001019201B0018201B202D0D890F4
:102A40001200D88012000001F8D73E0E0101176174
:102A500002D0019004D04C0E176501D0018005D83A
:102A6000DCE10201106B116BEED7010E01A0000E2C
:102A70000101186F010E01A2000E181B120012BAFC
:102A80000AAA24D0180E0101176503D03C0E176561
:102A900002D0018401D0019429D824E00201124B14
:102AA000132B010115510201125D010116510201A2
:102AB00013590AE30001019601B4018601B602D060
:102AC000D8901200D88012000001F8D73E0E010104
:102AD000176102D0019404D04C0E176501D0018417
:102AE00005D8DCE10201126B136BEED7010E01A4D5
:102AF000000E0101186F010E01A6000E181B120036
:102B000012BA0AAA24D0180E0101176503D03C0E90
:102B1000176502D0028001D0029029D824E002017A
:102B2000184B192B010115510201185D01011651B5
:102B3000020119590AE30001029202B0028202B2B4
:102B400002D0D8901200D88012000001F8D73E0EB3
:102B50000101176102D0029004D04C0E176501D01C
:102B6000028005D8DCE10201186B196BEED7010E6B
:102B700002A0000E0101186F010E02A2000E181B28
:102B8000120012BA0AAA24D0180E0101176503D048
:102B90003C0E176502D0028401D0029429D824E0AB
:102BA00002011A4B1B2B0101155102011A5D010193
:102BB000165102011B590AE30001029602B4028673
:102BC00002B602D0D8901200D88012000001F8D7C7
:102BD0003E0E0101176102D0029404D04C0E17651D
:102BE00001D0028405D8DCE102011A6B1B6BEED721
:102BF000010E02A4000E0101186F010E02A6000EC4
:102C0000181B12000401286B296B2AD00401C48F01
:102C1000040128810401C6512BE00401288328D037
:102C20000401C48F25D00401C48FCFEC2CF0C7C49D
:102C3000F6FFC8C4F7FF000EF86E0F0EF76403D05E
:102C40000800F55005D0F6CFE9FFF7CFEAFFEF50C7
:102C50000101006F00A50CD0010E0401286F08D0FF
:102C6000040120511F0BD2E0010ADAE0030ADBE085
:102C70000401C4AF1200040EC36F280EC26FC481DA
:102C8000020EC56F020C33D024C11BF125C11CF10B
:102C900026C11DF127C11EF126C115F127C116F16C
:102CA00003EC21F015C11FF116C120F189EC1CF0D5
:102CB0001C511B1105E124C124F125C125F112008D
:102CC0002429166F000E2521176F26C1F6FF27C194
:102CD000F7FF000EF86E0800F550186F196B18BF5B
:102CE000190757EC27F016C124F117C125F125511A
:102CF000241106E024C1D9FF25C1DAFFDF50C4E169
:102D0000246B256B120012BA0AAA26D0180E1F6473
:102D100003D03C0E1F6402D0018001D00190010E4F
:102D200001A0000E206E010E01A2000E201A26E066
:102D30000201104B112B1D50105D1E5011590AE35A
:102D40000001019201B0018201B202D0D8901200BC
:102D5000D88012000001F8D73E0E1F6002D001900B
:102D600004D04C0E1F6401D00180010E01A0000EA2
:102D7000206E010E01A2000E201ADAE10201106B92
:102D8000116BE8D7FC0E176FAC0E166F010E28EC16
:102D90001DF0300E0101296F750E2A6F000E2B6B8E
:102DA0002C6B2D6B68EC9EF00101306F30510C0ADA
:102DB00003E03051090A01E1000C30C131F1300E5D
:102DC000296F750E2A6F2B6B2C6B010E2D6F68EC23
:102DD0009EF0080AF1E1010131510B0A0AE1EAEC27
:102DE0002FF0D2EC2FF0890E0101295D130E2A5924
:102DF000F8E331510A0A03E031510B0ADDE13151A8
:102E0000120012BA0AAA26D0180E1F6403D03C0E74
:102E10001F6402D0018401D00194010E01A4000EB0
:102E2000206E010E01A6000E201A26E00201124BB0
:102E3000132B1D50125D1E5013590AE30001019619
:102E400001B4018601B602D0D8901200D8801200D9
:102E50000001F8D73E0E1F6002D0019404D04C0E42
:102E60001F6401D00184010E01A4000E206E010E2A
:102E700001A6000E201ADAE10201126B136BE8D7EB
:102E800012BA0AAA26D0180E1F6403D03C0E1F6483
:102E900002D0028401D00294010E02A4000E206E22
:102EA000010E02A6000E201A26E002011A4B1B2B6F
:102EB0001D501A5D1E501B590AE30001029602B410
:102EC000028602B602D0D8901200D880120000010B
:102ED000F8D73E0E1F6002D0029404D04C0E1F643F
:102EE00001D00284010E02A4000E206E010E02A683
:102EF000000E201ADAE102011A6B1B6BE8D712BA36
:102F00000AAA26D0180E1F6403D03C0E1F6402D0FC
:102F1000028001D00290010E02A0000E206E010E70
:102F200002A2000E201A26E00201184B192B1D5098
:102F3000185D1E5019590AE30001029202B0028284
:102F400002B202D0D8901200D88012000001F8D747
:102F50003E0E1F6002D0029004D04C0E1F6401D0C0
:102F60000280010E02A0000E206E010E02A2000ED1
:102F7000201ADAE10201186B196BE8D712BA0AAA13
:102F800026D0180E1F6403D03C0E1F6402D0018CA3
:102F900001D0019C010E01AC000E206E010E01AEAD
:102FA000000E201A26E00201164B172B1D50165D4D
:102FB0001E5017590AE30001019E01BC018E01BE9B
:102FC00002D0D8901200D88012000001F8D73E0E2F
:102FD0001F6002D0019C04D04C0E1F6401D0018CF4
:102FE000010E01AC000E206E010E01AE000E201A83
:102FF000DAE10201166B176BE8D712BA0AAA26D0DB
:10300000180E1F6403D03C0E1F6402D0018801D04B
:103010000198010E01A8000E206E010E01AA000EFB
:10302000201A26E00201144B152B1D50145D1E5072
:1030300015590AE30001019A01B8018A01BA02D0C8
:10304000D8901200D88012000001F8D73E0E1F6001
:1030500002D0019804D04C0E1F6401D00188010EEB
:1030600001A8000E206E010E01AA000E201ADAE15E
:103070000201146B156BE8D7E8CF17F10101175166
:10308000FE0F166F0001EF6B0101186B0DD09D0E46
:1030900001011825D96EDA6A0201020EDA22DF5028
:1030A000AFEC2FF00101182B1651185DF0E3000171
:1030B000EF390F0B57EC2EF0186F9B0E01011725FF
:1030C000D96EDA6A020EDA22DF50181902E0D890BF
:1030D00012000001EF510F0B57EC2EF0186F9C0EF1
:1030E00001011725D96EDA6A020EDA22DF501819AB
:1030F000EEE1D8801200010EC0EC22F015C118F1EB
:1031000016C119F118C1D9FF19C1DAFFDF6A020E21
:10311000C0EC22F015C118F116C119F118C1D9FF80
:1031200019C1DAFFDF6A030EC0EC22F015C118F1F5
:1031300016C119F118C1D9FF19C1DAFFDF6A040EEF
:10314000C0EC22F015C118F116C119F118C1D9FF50
:1031500019C1DAFFDF6A050EC0EC22F015C118F1C3
:1031600016C119F118C1D9FF19C1DAFF000EDF6EBF
:10317000000C1A0EA7EC2DF00201306B316B029897
:103180002FD0A6ECDAF002A82BD002980001F0674D
:1031900001D026D0060E01011C6F320E1B6FFD0EF2
:1031A0001E6F6D0E1D6F206B070E1F6FD5EC11F09B
:1031B0001C511B1102E1D8901200060E01011C6F78
:1031C000320E1B6FFB0E1E6F4C0E1D6F206B090E17
:1031D0001F6FD5EC11F01C511B1102E1D8801200B9
:1031E000310E0201305D750E3159F8E2CAD7E8CFD1
:1031F00021F1196B580E186FE7EC19F0226F1F05BB
:1032000007E1186B580E176F2251FE0B21110CD0DD
:103210001F51020A0CE1186B580E176FD890213518
:10322000206F2251FD0B15D0196F84EF1FF01F5135
:10323000030A05E1186B0FD82251FB0B0AD01F516E
:10324000040AD8A41200186B06D8D890203722514F
:10325000F70B2011E9D7580E176F21C120F1D89034
:103260002037D8902037580C1A6B18AF06D0176D3E
:10327000181FD8B0182B010E1A6F16AF06D0156D97
:10328000161FD8B0162B010E1A1B1B6B1C6B185186
:1032900017111BE0010E196F04D0D890173718379B
:1032A000192B18AFFAD7D8901B371C371751155D5B
:1032B0001851165905E31751155F1851165B1B81FC
:1032C000D89018331733192FEED71A5104E01B6D1D
:1032D0001C1FD8B01C2B1BC115F11CC116F112000C
:1032E00015C1D9FF16C1DAFF10EE06F028D810EE8E
:1032F00005F01551E1261651E222DFCFE7FF20EE5F
:1033000004F01551D9261651DA2215C1E1FF16C174
:10331000E2FFDFCFE7FF20EE02F01551D92616516C
:10332000DA2210EE04F00BD8B051DF6E20EE02F07E
:103330001551D9261651DA22AFC1DFFF12001551FF
:10334000E1261651E222DFCFE7FF20EE01F0155112
:10335000D9261651DA221200E8CF20F01F6A20C0C9
:103360001EF0010E1E161D50010B1E18D8A41F8042
:1033700020C01EF0020E1E161D50020B1E18D8A4EF
:103380001F8220C01EF0040E1E161D50040B1E18B6
:10339000D8A41F8420C01EF0080E1E161D50080B56
:1033A0001E18D8A41F8620C01EF0100E1E161D5019
:1033B000100B1E18D8A41F8820C01EF0200E1E1649
:1033C0001D50200B1E18D8A41F8A1F5012000A0E71
:1033D00001011D6FA00E1E6F30D01D07B36B64EC92
:1033E0002CF001011E5199EC27F00101B36717D0B1
:1033F000195199EC27F00101185199EC27F064EC70
:103400002CF001011E811E5199EC27F0000E33ECC7
:1034100028F01C6FD7EC29F001011C511200070E97
:103420001B6FD00E1A6F01D000F001011A07D8A04F
:103430001B071A29D8B41B29F7E11D51800A7F0FF9
:10344000CCE2000C080E236F33D00E0E256F1F2523
:10345000216F000E2021226F12D02507A10E01013D
:103460002525D96EDA6A010EDA222107D8A02207B3
:1034700021C118F122C119F1E7EC19F0DF6E2567BF
:10348000ECD7246B256BA10E2525D96EDA6A010EC7
:10349000DA22DF50241B252B2551800A730FF3E31A
:1034A000245121EEAEF0DF6202D0D8801200230753
:1034B0002367CBD7D8901200E8CF4BF12AC515F17E
:1034C0004B515BEC2BF002E2D890120000010CA2F1
:1034D000FBD78A8C0201206B216B000118888DECD0
:1034E000F3F001014B39F00B4A6F030E2F6F4A5175
:1034F00012ECE5F02FC148F130C149F105012A5124
:103500006BEC2FF002E2D88012004B51B6EC2AF09F
:103510004A6F48C139F149C13AF14BC13BF14AC147
:103520003CF1030E3D6FC5EC1DF0EDD7E8CF4BF13C
:1035300040C515F14B515BEC2BF002E2D890120024
:103540008DECF3F001014B39F00B4A6F010E2B6F3C
:103550002C6B040EBDECBFF0F1E3250E01012F6FC3
:103560004A5112ECE5F02FC148F130C149F1050193
:1035700040516BEC2FF002E2D88012004B51B6ECB8
:103580002AF04A6F48C139F149C13AF14BC13BF1C8
:103590004AC13CF1030E3D6FC5EC1DF0EDD7E8CFFD
:1035A0004BF13EC515F14B515BEC2BF002E2D8908C
:1035B00012008DECF3F001014B39F00B4A6F010E54
:1035C0002B6F2C6B020EBDECBFF0F1E3230E01015B
:1035D0002F6F4A5112ECE5F02FC148F130C149F18B
:1035E00005013E516BEC2FF002E2D88012004B51E6
:1035F000B6EC2AF04A6F48C139F149C13AF14BC1E2
:103600003BF14AC13CF1030E3D6FC5EC1DF0EDD717
:10361000E8CF4BF13FC515F14B515BEC2BF002E2CB
:10362000D89012008DECF3F001014B39F00B4A6F8A
:10363000010E2B6F2C6B030EBDECBFF0F1E3240EDB
:1036400001012F6F4A5112ECE5F02FC148F130C152
:1036500049F105013F516BEC2FF002E2D8801200D6
:103660004B51B6EC2AF04A6F48C139F149C13AF1E1
:103670004BC13BF14AC13CF1030E3D6FC5EC1DF05F
:10368000EDD720EE02F01551D9261651DA22DF507F
:10369000196F20EE02F024D8E750176F10EE02F0F9
:1036A0001551E1261651E222E750186F18390F0B19
:1036B0001711DF6E20EE01F013D8DFCFE7FF20EE09
:1036C00001F01551D9261651DA22DF6A20EE01F0F9
:1036D0001551D9261651DA221939F00BDF6E120076
:1036E0001551D9261651DA2215C1E1FF16C1E2FFA4
:1036F0001200E8CF4BF12BC515F14B515BEC2BF0D1
:1037000002E2D89012008A9C0201206B216B00011A
:1037100018988DECF3F001014B39F00B4A6F040E51
:103720002F6F4A5112ECE5F02FC148F130C149F139
:1037300005012B516BEC2FF002E2D88012004B51A7
:10374000B6EC2AF04A6F48C139F149C13AF14BC190
:103750003BF14AC13CF1030E3D6FC5EC1DF0EDD7C6
:10376000E8CF25F125074250BAEC2DF01F6F4150EC
:10377000BAEC2DF0206F2039F00B1F11236F25516B
:10378000220DF80EF324186F3F0EF420196FE7ECAA
:1037900019F0246F2451231902E0D890120025510A
:1037A000220DF90EF324216F3F0EF420226F21C168
:1037B00018F122C119F1E7EC19F0266F010E266508
:1037C000ECD7100E266501D0E8D7D880120004018E
:1037D000C48F0F014D6B4E6B0401BE6B22C4BDF450
:1037E0000401226704D0100E0401CD6F100C200ECE
:1037F0000401CD6F0401CE6B4B0ECF6FD06BD16B3C
:10380000D26BD36B080ED46F010ED56F0401CC6B55
:10381000CC8F0401B16B0401B06B1A0E0F014E6F17
:103820000401148D149F1E0E0F014F6F04011C8D97
:103830001C9F188D189FDAEF2EF00401C48F0F0122
:103840004D6B4E6B0401BE6B22C4BDF404012267B4
:1038500004D0100E0401CD6F100C200E0401CD6FAA
:103860000401CE6B4B0ECF6FD06BD16BD26BD36B91
:10387000080ED46F010ED56F0401CC6BCC8F040100
:10388000B16B0401B06B1A0E0F014E6F0401148D61
:10389000149F1E0E0F014F6F04011C8D1C9F188D6D
:1038A000189FE7EF2EF0E8CF9AF1000108B6050C5B
:1038B000000113BA050C99C19BF11DD09A6704D081
:1038C00012EC22F001019C6F9C5119E09B6701D022
:1038D00016D09C51040A03E09C51020AD8B41FEC94
:1038E0002DF0EAEC2FF0D2EC2FF0990E0101295DBA
:1038F0003A0E2A59F8E301019B079B29DFE19C510D
:10390000040A03E09C51020AD8B41FEC2DF09C512C
:10391000120029D01DC1F6FF1EC1F7FF000EF86E80
:103920000800F550CDEC2EF0216F1BC1D9FF1CC152
:10393000DAFFDF50CDEC2EF0226F2151225D236F94
:103940000101236706D01BC1D9FF1CC1DAFFDF507C
:1039500006E123511B6F1C6B1BBF1C0712001B4B86
:103960001C2B1D4B1E2B1F07D8A0200701011F2950
:10397000D8B42029CFE11B6B1C6B1200E8CF27F1D4
:1039800027C115F1166B270E186F100E176F7AEC02
:103990002CF01C51640DF3CF1FF1F4CF20F11D5119
:1039A0000A0DF3501F25216FF4502021226F15516D
:1039B0002125236F16512221246F1BC115F1166B8F
:1039C000030E186FE80E176F7AEC2CF015512325B3
:1039D000256F16512421266F1E5125251B6F000EC1
:1039E00026211C6F1200E8CF4BF12DC515F14B516C
:1039F0005BEC2BF002E2D890120000010CA4FBD784
:103A00008A8E8DECF3F001014B39F00B4A6F060EF4
:103A10002F6F4A5112ECE5F02FC148F130C149F146
:103A200005012D516BEC2FF002E2D88012004B51B2
:103A3000B6EC2AF04A6F48C139F149C13AF14BC19D
:103A40003BF14AC13CF1030E3D6FC5EC1DF0EDD7D3
:103A5000E8CF18F10101185118E0410EA7EC2DF044
:103A6000540EA7EC2DF011D001011FD8F76403D03C
:103A70000800F55005D0F6CFE9FFF7CFEAFFEF5089
:103A8000A7EC2DF00101164B172B01010ED8F7649E
:103A900003D00800F55005D0F6CFE9FFF7CFEAFFD5
:103AA000EF500009D8B41200DFD716C1F6FF17C1D6
:103AB000F7FF000EF86E0F0E1200E8CF27F145C594
:103AC00015F127515BEC2BF002E2D89012000301B4
:103AD000E751080AFAE1330EE725D96EDA6A030ED8
:103AE000DA22DF6A370E0101256F030E266F25C12A
:103AF0001BF126C11CF160EC04F01BC128F11CC1B4
:103B000029F128C11FF129C120F11CEC29F0DDE3C6
:103B1000500E206FD20E1F6FE6EC21F0FF00D88010
:103B200012001A6B16AF06D0156D161FD8B0162BE3
:103B3000010E1A6F18AF04D0176D181FD8B0182BCC
:103B40001851171117E0010E196F04D0D8901737CC
:103B50001837192B18AFFAD71751155D1851165988
:103B600004E31751155F1851165BD89018331733BB
:103B7000192FF2D71A5104E0156D161FD8B0162B65
:103B800015C115F116C116F1120039513E6F030E21
:103B90003A153F6F3DC140F1416B0D0ED890403753
:103BA0004137E82EFBD73BC142F1436B0A0ED89058
:103BB00042374337E82EFBD740514211446F415101
:103BC0004311456F3E514411466F3F514511476FB8
:103BD0003C51D8A4478F46C130F147C131F13BC1B8
:103BE00032F161EC0AF002E3D8801200D8901200A2
:103BF0000201346B356BF90E0101176F600E166F01
:103C0000010E28EC1DF008ECD7F068EC9EF00101E5
:103C1000306F30512D0A06E1130E2A6F880E296F7E
:103C2000BAEF21F0130E2A6F880E296FBAEC21F03B
:103C3000EAEC2FF0D2EC2FF0D10E0101295D070E36
:103C40002A59F8E3B40E0201345D000E3559D3E36E
:103C5000FF00D1D700010DA0000C01011C6B16D094
:103C6000500E01011C25D96EDA6A070EDA221C51AA
:103C70001525176FE86A1CBFE8681621186F17C171
:103C8000E1FF18C1E2FFDFCFE7FF1C2B80C217F175
:103C90000101186B1CC119F11A6B19BF1A071A51CF
:103CA000800A1B6F1751195D1851800A1B59D8E300
:103CB0000D90020180511200E8CF4BF12EC515F195
:103CC0004B515BEC2BF002E2D89012008A9E8DECF7
:103CD000F3F001014B39F00B4A6F070E2F6F4A5179
:103CE00012ECE5F02FC148F130C149F105012E5128
:103CF0006BEC2FF002E2D88012004B51B6EC2AF0A8
:103D00004A6F48C139F149C13AF14BC13BF14AC14F
:103D10003CF1030E3D6FC5EC1DF0EDD73F6A02018B
:103D20009D0502E0D89012000101016B9D0E01017A
:103D30000125D96EDA6A0201020EDA22DF50A56F80
:103D40000101006B0201A5513F18A66F0201A633C5
:103D500002E3180E3F1A00F000013F330201A533C1
:103D6000D8900101002B070E0065ECD7012B060E41
:103D70000165DCD70201A4513F18D4E1D8801200BC
:103D8000E8CF4BF13CC515F14B515BEC2BF002E257
:103D9000D89012008DECF3F001014B39F00B4A6F13
:103DA000210E2F6F4A5112ECE5F02FC148F130C1BE
:103DB00049F105013C516BEC2FF002E2D880120072
:103DC0004B51B6EC2AF04A6F48C139F149C13AF17A
:103DD0004BC13BF14AC13CF1030E3D6FC5EC1DF0F8
:103DE000EDD7E8CF4BF13BC515F14B515BEC2BF018
:103DF00002E2D89012008DECF3F001014B39F00B88
:103E00004A6F200E2F6F4A5112ECE5F02FC148F196
:103E100030C149F105013B516BEC2FF002E2D88033
:103E200012004B51B6EC2AF04A6F48C139F149C132
:103E30003AF14BC13BF14AC13CF1030E3D6FC5EC79
:103E40001DF0EDD7E8CF4BF13AC515F14B515BECC6
:103E50002BF002E2D89012008DECF3F001014B3907
:103E6000F00B4A6F190E2F6F4A5112ECE5F02FC17B
:103E700048F130C149F105013A516BEC2FF002E2F3
:103E8000D88012004B51B6EC2AF04A6F48C139F184
:103E900049C13AF14BC13BF14AC13CF1030E3D6FC0
:103EA000C5EC1DF0EDD7E8CF4BF13DC515F14B51F9
:103EB0005BEC2BF002E2D89012008DECF3F00101E4
:103EC0004B39F00B4A6F220E2F6F4A5112ECE5F07E
:103ED0002FC148F130C149F105013D516BEC2FF084
:103EE00002E2D88012004B51B6EC2AF04A6F48C16A
:103EF00039F149C13AF14BC13BF14AC13CF1030EE2
:103F00003D6FC5EC1DF0EDD70A0E1D6FA00E1C6FA6
:103F100026D01D07B36B64EC2CF001011C5199EC09
:103F200027F00101B3670DD0185199EC27F001017A
:103F3000175199EC27F00101195199EC27F0D7EFAF
:103F400029F0070E1B6FD00E1A6F01D000F001018F
:103F50001A07D8A01B071A29D8B41B29F7E11D514D
:103F6000800A7F0FD8A01200D4D70101326BC2ECB7
:103F700016F00101336F33510B0A03E1A6EC20F078
:103F800020D8335102E032511AE0EAEC2FF0D2ECA3
:103F90002FF0990E0101295D3A0E2A59F8E3326B90
:103FA000C2EC16F00101336F33510B0A03E1A6ECAA
:103FB00020F007D8335102E0325101E0010C45EF07
:103FC000E7F0010ED8A0000E326F12001FC19AF266
:103FD000199413D00101200507E11DC115F11EC17F
:103FE00016F1F1EC29F006D01DC115F11EC116F134
:103FF0002AEC1EF00201646F986B0201646702D024
:104000009A67E8D79A6703D000011984000C640707
:10401000985101011D25D96E000E1E21DA6EDF5068
:10402000216F0201982B010121511200E8CF50F1BC
:1040300028C515F150515BEC2BF002E2D89012002C
:104040005051B6EC2AF04F6F50C11FF14F51010A89
:10405000F7EC18F08DECF3F001015039F00B4F6FD5
:10406000010E2F6F4F5112ECE5F0050128516BEC5A
:104070002FF002E2D88012005051B6EC2AF04F6FB8
:104080004FC148F150511EECD7F0F4D72DC127F1A4
:104090002EC128F12FC129F130C12AF1B8EC27F047
:1040A0000201565121E0264B272BD89026350101DD
:1040B000316F280E3125D96EDA6A070EDA22020135
:1040C00042C2DEFF43C2DDFFD89026350101316FC9
:1040D000000E3125D96EDA6A0701070EDA22000ECA
:1040E000DE6EDD6ED880000CD8901200FC0E176FCB
:1040F000CD0E166F010E28EC1DF008ECD7F068EC21
:104100009EF00101306F30513A0AD8A41200070E18
:10411000306F850E01013025D96EDA6A050EDA227C
:10412000170E3025E16EE26A060EE222DFCFE7FFCE
:10413000302B3051800A660FECE30601316B130E11
:1041400001012A6F880E296FBAEF21F0FB0E176F5D
:10415000420E166F010E28EC1DF0E80E0101296FCA
:10416000FD0E2A6F000E2B6B2C6B2D6B68EC9EF0F6
:104170000101306F30510C0A11E03051090A0EE094
:104180003051080A0BE0E80E296FFD0E2A6F2B6BE9
:104190002C6B010E2D6F68EC9EF0EAD73051080AA7
:1041A00002E1D8901200D8801200C76A300EC66EA5
:1041B0000101166B176B186B196B550E1A6FE3EC38
:1041C0002CF0166B010E176F186B196BAA0E1A6F75
:1041D000E3EC2CF01490000E0101166B176B186BBA
:1041E000196B4EEC2CF0550A0BE1166B010E176F94
:1041F000000E186B196B4EEC2CF0AA0AD8B4120002
:1042000000011480120015C119F116C11AF1010143
:104210001951176F1A51186F194B1A2B17C1F6FF46
:1042200018C1F7FF000EF86E0F0EF76403D00800F8
:10423000F55005D0F6CFE9FFF7CFEAFFEF500009C0
:10424000E6E1010119C117F11AC118F11551175F03
:104250001651185BFF0E1725156FFF0E1821166FEC
:10426000120037C12BF138C12CF139C12DF13AC1FF
:104270002EF1D1ECEBF002E2D890120000010D908B
:10428000EAEC2FF013D000010DA010D0070E0101B1
:10429000256F500E246F37C126F138C127F106EC87
:1042A000EDF002E3D880120000010D90D2EC2FF067
:1042B000E90E0101295DFD0E2A59DEE2E4D7F294F0
:1042C0003D6602D045EF2FF03D0402E12FEF2FF0C5
:1042D0003D50020A02E14FEF2FF03D50030A02E188
:1042E000AAEF28F03D50040A02E141EF23F03D50CF
:1042F000050A02E1DEEF2DF03D50060A02E1F0EF83
:104300002DF03D50070A02E16EEF29F03D50080AFA
:1043100002E160EF24F03D6A120046840101186B4F
:10432000520E176FFFC019F184EC1FF00101196BD9
:10433000520E186FE7EC19F00001FE6F0101BB6B24
:104340003CC219F13DC21AF1BEEC04F00001FF6F4E
:1043500012BA0AAA04D0FE51E00BFF1903D00001E3
:10436000FF51FE190101BB6FBBC19BF21386000117
:10437000469412000201366B376B01012B6B1BD088
:10438000A6ECDAF0BDEC2FF016E3EEEC2FF0010115
:104390002C6F0DD02C519EEC2BF00DE301012B2B3B
:1043A0000AD02C5172EC2BF006E3D88012002B516E
:1043B000F1E0010AF6E0020136510101295D020136
:1043C000375101012A59DCE2D89012001F29186FD9
:1043D000000E2021196FE7EC19F0216F1FC118F1B1
:1043E00020C119F1E7EC19F0236F2151226F224B04
:1043F000232B2229D8B4232902E1226B236B1FC16E
:1044000017F120C118F12351196F84EC1FF0010E30
:1044100001011F25176F000E2021186F22C119F10D
:1044200084EF1FF0B5EC1FF0986F985102E098519F
:1044300012001CA008D00201616B12841786148A36
:1044400000010492000C0001158C44EC0EF00101F7
:10445000986F159C980503E09851030A0EE102013C
:10446000616B12841786148A049201019851030A21
:10447000E9E1010EDFECD0F0000C020C750E23D840
:10448000000EDB8E17A408D0750E5125D96EDA6A9E
:10449000050EDA22000EDB8C960E02015125010179
:1044A000176F186B020E1823750E0DD8DF5001011F
:1044B000196F84EC1FF0530E0201A06F100EA16F54
:1044C000515197EF23F002015125D96EDA6A050E9A
:1044D000DA221200E8CF17F1170506E1080E0101F4
:1044E000166F000E156F12001751020A06E1080E32
:1044F0000101166F500E156F12001751030A06E1E5
:10450000080E0101166FA00E156F12001751040A54
:1045100006E1090E0101166FA00E156F1200050EBF
:104520000101166FE90E156F1200E8CF31F1F5ECBD
:104530000DF0D8B0F5EC0DF0D8B012000101326BDF
:10454000316705D06A0E0DD884EC1FF004D0790EC7
:1045500008D884EC1FF00101322B0E0E3265F0D723
:104560000E0C3225176F186B130E1823D60E01018F
:104570003225D96EDA6A040EDA22DF50196F120082
:10458000E8CF17F10101170505E1020E166FB30E12
:10459000156F12001751020A06E1020E0101166F93
:1045A000B40E156F12001751030A06E1020E010145
:1045B000166FB50E156F12001751040A06E1020EB0
:1045C0000101166FB60E156F1200020E0101166F73
:1045D000B70E156F1200040E0101196F030E186F4C
:1045E000E7EC19F0216F040E196F020E186FE7EC5B
:1045F00019F0236F2151226FFF0E225D000E235907
:1046000004E2040E206F1F6F040C040E196F010EDC
:10461000186FE7EC19F0216F040E196F000E186B7C
:10462000E7EC19F0206F21511F6F1200F90E010104
:10463000176F1B0E166F010E28EC1DF0300E0101D6
:10464000296F750E2A6F000E2B6B2C6B2D6B68EC8F
:104650009EF00101306F3051240AD8B4120030515D
:104660000C0AD8B412003051090AD8B41200300E26
:10467000296F750E2A6F2B6B2C6B010E2D6F68EF57
:104680009EF03F6609D02F0E0101016F100E006FE2
:1046900045EC26F03D6A12003F06010E0101016F54
:1046A000690E006F45EC26F086A6120000F086A683
:1046B000120000F086A6120010A406D0010E02011E
:1046C0001D6FF40E1C6FE6D7330E02019D6F080EAE
:1046D0003E6E3D2ADEEF2DF086EC2AF0186F20EEBC
:1046E00003F01651D9261751DA2218C1DFFF86ECE4
:1046F0002AF0186F20EE02F01651D9261751DA224F
:1047000018C1DFFF86EC2AF016C1D9FF17C1DAFF06
:10471000DF6E86EC2AF0186F20EE01F01651D926D4
:104720001751DA2218C1DFFF0001089E1200E8CFFE
:104730001AF1060E02019D6F0101B05102019E6F38
:10474000AFC19FF2A26B750E01011A25D96EDA6A0C
:10475000050EDA22DF50196F19AD05D01A510F0B73
:104760000201A11304D01A39F00B0201A213A36BAA
:10477000A46B020E0101176F9D0E166F88EF2BF0D0
:104780009E9402018E6B000115B8120002018B91FC
:1047900082AC8B81080E8D2B8D6103D0D8908B3726
:1047A000080C8D6BA70E8C25D96EDA6A020EDA2200
:1047B0008BC2DFFF8C2B060E02018C65060C8C6B06
:1047C000829C949C829C158815868F8000011280A3
:1047D00012000251040A02E0D890120000C1D9FF71
:1047E00001C1DAFFDF504E0AF7E120EE01F000517F
:1047F000D9260151DA22DF50100AEEE120EE02F054
:104800000051D9260151DA22DF505E0AE5E120EE9F
:1048100003F00051D9260151DA22DF50AC0ADCE165
:10482000D8801200416A426AA12903E1390E416E23
:10483000426EA151030A0BE1A6390F0B57EC2EF083
:10484000416EA6510F0B57EC2EF0426E1200A15193
:10485000060A04E0A151070AD8A41200A5510F0BC3
:1048600057EC2EF0416EA6390F0B57EC2EF0426E2E
:104870001200E8CF21F121072151330D890EF324D5
:10488000226F130EF420236F246BED0E01012425FB
:10489000D96EDA6A0501050EDA2222C118F123C1A8
:1048A00019F1E7EC19F0DF6E224B232B242B030EBA
:1048B0002465EBD7050E0101206FED0E1F6F12006E
:1048C0003E2E12D08EEC1EF00CE31084010E02017D
:1048D0001D6FF40E1C6F1098189E3C0E526F010E47
:1048E000456E3D6A45EF2FF00201A4330201A33368
:1048F0000201A2330201A1330201A03302019F335E
:1049000002019E3302019D333D066EEF29F0E8CF90
:104910001DF01D502B0A03E10201486B1200000E2E
:1049200002014825D96EDA6A060EDA221DC0DFFFC1
:10493000482B4851160AD8A4120006010051430A18
:104940000AE10151470A07E10251530A04E1035108
:104950004E0AD8B41200000105961200040120513D
:10496000800AD8A41200800E0401C46F13D0F10E87
:104970000401C36F570EC26F120EC56F120CF10EF9
:104980000401C36F140EC26F430EC56F430C0401C4
:10499000C46B120004012351010AE9E0030AEFE0AD
:1049A000010AD8A41200F3D704012051800AD8A428
:1049B0001200800E0401C46F13D0F10E0401C36F06
:1049C000570EC26F120EC56F120CF10E0401C36FA9
:1049D000140EC26F430EC56F430C0401C46B12006A
:1049E00004012351010AE9E0030AEFE0010AD8A417
:1049F0001200F3D715C11BF116C11CF102D01B4BDD
:104A00001C2B1BC1D9FF1CC1DAFFDF50F8E1175185
:104A1000196F18511A6F174B182B19C1F6FF1AC1CD
:104A2000F7FF000EF86E1BC1D9FF1CC1DAFF1B4B4C
:104A30001C2B0800F5CFDFFFDF50D8B41200E7D7FA
:104A4000E8CF50F129C515F150515BEC2BF002E293
:104A5000D89012008DECF3F001015039F00B4F6F3C
:104A6000020E2F6F4F5112ECE5F0050129516BEC4E
:104A70002FF002E2D88012005051B6EC2AF04F6FAE
:104A80004FC148F150511EECD7F0F4D71A6B1B6B95
:104A9000185117111BE0010E196F04D0D890173769
:104AA0001837192B18AFFAD7D8901A371B37175168
:104AB000155D1851165905E31751155F1851165B0E
:104AC0001A81D89018331733192FEED71AC115F160
:104AD0001BC116F11200E8CF45F104C315F1455191
:104AE0005BEC2BF002E2D89012008DECF3F00101A8
:104AF0004539F00B446F790E2F6F445112ECE5F0FD
:104B00000001108CD9EC2FF01FEC2DF0189C148CA8
:104B10000001F45103E0F4050201836FD880120014
:104B20001DC115F11EC116F11FC117F120C118F1E9
:104B300034EC19F015C123F116C124F11DC115F192
:104B40001EC116F11FC117F120C118F191EC1DF023
:104B500015C121F116C122F121C11DF122C11EF1A1
:104B600023C11FF124C120F11200F294EB0E0101C8
:104B7000016F500E006F45EC26F0000110B20ED010
:104B800086B602D03F6A12003F2A3F50330AD8A4AB
:104B900012003F6A108200011084120086B6F2D71C
:104BA0003F2A3F50330AD8A412003F6A10920001F6
:104BB000108412000401FE51D8A41200000110BE9E
:104BC00012001D6A0101BCA102D006861D2A010146
:104BD000BCA302D006861D2A0101BCA502D0068610
:104BE0001D2A1D6601D0069607B802D013A403D073
:104BF000000108841200000108941200FA0E01015D
:104C0000176F310E166F010E28EC1DF0EAEC2FF035
:104C10000CD0BDEC2FF009E3EEEC2FF001012B6F6F
:104C20002B513E0A02E1D8901200D2EC2FF0890EEF
:104C30000101295D130E2A59ECE31B0EA7EC2DF0A0
:104C4000D880120005929CA29CB40582AACFEDF0F8
:104C500005A205D09C989C8800010594120005844B
:104C600000011CB0A5ECE8F0000112B402D0000174
:104C700015BC70ECF5F005A604D00001ED5187ECF1
:104C800024F00001ED51AAEFBBF0D59E0051026F58
:104C90000151036F046B056B02510008066F000E93
:104CA0000355076F010E0455086F000E0555096F77
:104CB00007C106F108C107F109C108F1096B08BF76
:104CC00009690651D76E00510008D66ED58E1200C4
:104CD000750E63EC22F0C00EDF16750E5125D96EED
:104CE000DA6A050EDA22DF5001011E6F1EAF3EEFB9
:104CF00022F0750E63EC22F0DF5001011E6F1EAD35
:104D000005D0000117B412003EEF22F0000117A4F5
:104D100012003EEF22F02AC12BF11CD026C117F160
:104D200027C118F128C119F129C11AF12BC11BF1B2
:104D30005DEC0CF02C6FB351D8A412002C51262737
:104D4000000E27232C51010DF3502827000E292394
:104D50002C512B5F2B67E2D7120074EC2FF000016F
:104D6000108EEBEC22F00201826B13920101010E16
:104D7000226F360E216FF90E246FFA0E236F0D0E7F
:104D8000266F710E256FEBECD8F02151476F010EA5
:104D9000166F360E156F47C117F196EF2EF0E8CF5C
:104DA00015F1150501E1010C1551020A01E1020C92
:104DB0001551040A01E1030C1551080A01E1040C24
:104DC0001551100A01E1050C1551200A01E1060CEC
:104DD0001551400A01E1070C1551800A01E1080C48
:104DE000000C456602D068EF2EF0450402E118EF92
:104DF0002FF04550020A02E162EF2FF04550030AFE
:104E0000F6E04550040AF8E04550050AF0E0455048
:104E1000060A02E13AEF2FF04550070A02E1F4EFEB
:104E20002EF0456A12001BD0C7C4F6FFC8C4F7FFB6
:104E3000000EF86EC9C4D9FFCAC4DAFF0F0EF764BA
:104E400003D00800F55005D0F6CFE9FFF7CFEAFF11
:104E5000EF50DF6E0401C74BC82BC94BCA2B0401AE
:104E6000CB07CB29D8B41200DFD71BD0C7C4F6FFBD
:104E7000C8C4F7FF000EF86EC9C4D9FFCAC4DAFF70
:104E80000F0EF76403D00800F55005D0F6CFE9FF08
:104E9000F7CFEAFFEF50DF6E0401C74BC82BC94BB9
:104EA000CA2B0401CB07CB29D8B41200DFD7185185
:104EB000CDEC2EF0186F196B18BF190710D016C162
:104EC000D9FF17C1DAFFDF50CDEC2EF0181905E13C
:104ED00016C116F117C117F11200164B172B16C188
:104EE000D9FF17C1DAFFDF50EAE1166B176B12002A
:104EF000040E0101186F176B196F84EC1FF0040E7C
:104F00000101186F010E176F040E196F84EC1FF06A
:104F1000040E0101186F020E176F000E196B84EC5E
:104F20001FF0040E0101186F030E176F196B84EF49
:104F30001FF0E8CF15F1166B15AF03D00001038CFD
:104F400002D00001039CE4EC28F00101D890153751
:104F5000162B1651800A780FEFE347EC2DF0000175
:104F600003AA12000101B3671200030EB36F030C12
:104F700027C122F128C123F129C124F12AC125F139
:104F8000E6EC2AF02B6F2B39F00B2C6F27C122F1A6
:104F900028C123F129C124F12AC125F1E6EC2AF028
:104FA0002C272C510201562701012C51120000011F
:104FB00008BE12001EC0D9FF1FC0DAFFDF503EEC52
:104FC0002AF020EE01F01E50D9261F50DA22DF50C1
:104FD0003EEC2AF020EE02F01E50D9261F50DA22B5
:104FE000DF503EEC2AF000010D8812001F511E1107
:104FF00017E0010E206F04D0D8901E371F37202BEA
:105000001FAFFAD71E511C5D1F511D5904E31E51DD
:105010001C5F1F511D5BD8901F331E33202FF2D70A
:105020001CC11CF11DC11DF11200636A626A9F0E52
:105030000F015D6F5E6B4D6B4E6BFB0E5C6F658C95
:105040000401C46B0401C16B0401BD6B0401CD6B91
:10505000659C160E0F014C6F02D06296040062B67A
:10506000FCD765981200E8CF15F10101176B166B9C
:1050700047EC2DF00101D8901737179103BA17812B
:10508000162B1651800A780FF3E3155107E0000143
:10509000039CE4EC28F00101175112000001038C7D
:1050A000F8D71F4B202B226B9E0E01012225D96EB3
:1050B000DA6A020EDA22DF50216F1F51186F205179
:1050C000196F1F4B202BE7EC19F0211902E0D89043
:1050D0001200222B050E2265E7D7D880050C4F0E53
:1050E00001011F6FDD0E1E6F206B1EC117F11FC166
:1050F00018F1000E196B84EC1FF0070E01011E273A
:10510000000E1F23202B0F0E2065EFD7069C186B77
:10511000540E176F196B84EF1FF0636A626A9F0E5B
:105120005D6F5E6B4D6B4E6BFB0E5C6F658C0401AF
:10513000C46B0401C16B0401BD6B0401CD6B659CA4
:10514000160E0F014C6F02D06296040062B6FCD7B7
:105150006598120086B611D000F086B60ED000F029
:1051600086B60BD0010E0101016F690E006F45EC90
:1051700026F03D2A050E3F6E050C2F0E0101016F32
:10518000100E006F45EC26F0010E3D6E010CE8CFCD
:105190001AF1010E196F1A51800A190F04E21A51FF
:1051A000800A1F0F0DE21A51800A390F04E21A51CA
:1051B000800A3F0F05E21A5146EC2EF0D8A0196B79
:1051C00019C118F11831120096929690000103ACA3
:1051D00009D0848284B209D00101B36706D0020EDF
:1051E000B36F03D0000103AC84928D8000F08DB0CA
:1051F00005D00101B36702D0010EB36F8D9012008C
:105200001B6B86EC2AF0186F1B511625196FE86A84
:105210001BBFE86817211A6F19C1D9FF1AC1DAFF3D
:1052200018C1DFFF1B2B1B51800A790FEAE386ECC4
:105230002AF00001089E12004F0E196FD40E186F4D
:10524000E7EC19F0216F4F0E196FD50E186FE7ECD0
:1052500019F0226F2151246F2251236F20512419FC
:1052600002E11F51231902E1D8801200D8901200E8
:1052700000C1D9FF01C1DAFFDF50060A02E0D89071
:10528000120020EE01F00051D9260151DA22180E49
:10529000DF6205D002510C0A02E1D88012000251EF
:1052A0000A0AFBE0ECD7E8CF15F115C1C2FFC280B6
:1052B000190E0101166F160701011629FCE1C282C1
:1052C000320E166FC2A204D0160701011629FAE1A8
:1052D000C450FC0B166FC26A16511200869698963F
:1052E000080E3F6E3F2EFED79886280E3F6E3F2E4B
:1052F000FED786A603D00201A48F02D00201A49F8C
:10530000010E0101016FA50E006F45EC26F03D2A4C
:1053100012001B6B86EC2AF0186F1B511625196FB3
:10532000E86A1BBFE86817211A6F19C1D9FF1AC1B3
:10533000DAFF18C1DFFF1B2B1B51800A7B0FEAE34A
:105340000001089E120017C118F1196B1551010BCD
:10535000181BD8901633153318A104D0010E151B55
:10536000A00E161BD8901833192B070E1965EED70F
:1053700015C115F116C116F1070C1B6B86EC2AF04E
:10538000186F1B511625196FE86A1BBFE8681721B3
:105390001A6F19C1D9FF1AC1DAFF18C1DFFF1B2B21
:1053A0001B51800A7D0FEAE30001089E12008492DF
:1053B00096928D80969000F000F08DB005D001019E
:1053C000B36702D0010EB36F848200F000F084B2A4
:1053D00005D00101B36702D0040EB36F8D9000F0C9
:1053E000120094EC2DF00101176F175111E0A098F5
:1053F000040E0401C86F300EC76F15C1C9F416C181
:10540000CAF417C1CBF413EC27F0A088E7EC2EF018
:105410000101175112001B6B86EC2AF0186F1B510B
:105420001625196FE86A1BBFE86817211A6F19C1A2
:10543000D9FF1AC1DAFF18C1DFFF1B2B1B51800AED
:105440007E0FEAE30001089E12000101206B1EC1DD
:1054500017F11FC118F19D0E01012025D96EDA6ADE
:10546000020EDA22DF50196F84EC1FF001011E4B8F
:105470001F2B202B060E2065EAD7060CE8CF1DF067
:10548000000E4024D96EDA6A0A0EDA221DC0DFFF50
:10549000402A4050F00AD8B4406A0001F12BF15183
:1054A000F00AD8A412000001088E1200E8CF1DF007
:1054B0001DC0C2FFC280190E1E6E1E061E28FDE111
:1054C000C282320E1E6EC2A203D01E061E28FBE14F
:1054D000C450FC0B1E6EC26A1E501200500E010119
:1054E0001F6F4D0E1E6F206B1EC117F11FC118F1EB
:1054F000000E196B84EC1FF0070E01011E27000E31
:105500001F23202B0F0E2065EFD70F0C000E02017A
:105510005D25D96EDA6A0A0EDA22DF500101156FB5
:1055200002015D2B5D51F00AD8B45D6B0001F107FB
:10553000F16701D00D98010115511200E8CF15F166
:10554000000E4024D96EDA6A0A0EDA2215C1DFFF96
:10555000402A4050F00AD8B4406A0001F12BF151C2
:10556000F00AD8A412000001088E1200E8CF21F141
:105570000101196B580E186FE7EC19F0226F21C169
:105580001FF1FF0E1F2722C120F11F2B02D0D89040
:1055900020331F2FFCD72051010B120002510E0A9D
:1055A00002E0D890120000C1D9FF01C1DAFF070E56
:1055B000DF6401D0F6D720EE01F00051D926015169
:1055C000DA22010EDF62EDD7D880010C22C11DF175
:1055D00023C11EF124C11FF125C120F1E6EC1FF00B
:1055E0000101266F266701D0000C400E266503D00E
:1055F0002651C90F12002651D00F1200010E0101D1
:105600001F6F750E01011F25D96EDA6A050EDA22A9
:10561000960E1F25186F196B020E1923E7EC19F06F
:10562000DF6E1F2B0F0E1F65ECD70F0C02510B0AFC
:1056300002E0D890120000C1D9FF01C1DAFFDF50AB
:105640004E0AF7E120EE01F00051D9260151DA228D
:10565000DF50610AEEE1D880120002510D0A02E02B
:10566000D890120000C1D9FF01C1DAFFDF504E0A05
:10567000F7E120EE01F00051D9260151DA22DF5086
:10568000620AEEE1D8801200175115C1D9FF16C188
:10569000DAFFDF6205D015C115F116C116F112004F
:1056A00015C1D9FF16C1DAFF154B162BDF50ECE1FF
:1056B000156B166B1200E8CF18F1185103E0185162
:1056C000050A02E1D890120018C116F1FF0E162744
:1056D00015C117F1162B02D0D8901733162FFCD70F
:1056E00017311200E8CF15F115510D0A04E115C16B
:1056F00046F2D890120015510A0A07E102014651FC
:105700000D0A03E1466BD88012000201466BF1D707
:10571000000108BE12000101186B18511625D96E40
:10572000000E1721DA6EDF509EEC2AF00101182BD3
:10573000070E1865F2D700010D88070CE8CF15F1A8
:1057400015514F0A04E115C147F2D89012001551C6
:105750004B0A07E1020147514F0A03E1476BD8802A
:1057600012000201476BF1D7E8CF1CF118516AEC27
:1057700022F015C11AF116C11BF11C51020DF35094
:105780001A25D96E000E1B21DA6EDECF18F1DDCF9F
:1057900019F11200000108BE12001EC0D9FF1FC07F
:1057A000DAFFDF503EEC2AF020EE01F01E50D92641
:1057B0001F50DA22DF503EEC2AF000010D88120063
:1057C000E8CF37F10101370508E1FA0E166FD40E64
:1057D000156F090E176F96EF2EF0FA0E2C6FD40E80
:1057E0002B6F2E6B090E2D6FD1EFEBF0216A226A21
:1057F0001DA004D01F50212620502222D8901F36F1
:105800002036D8901E321D321E501D10F1E121C0ED
:105810001DF022C01EF01200E8CF37F1010137055C
:1058200008E1F90E166FEF0E156F0A0E176F96EF5F
:105830002EF0F90E2C6FEF0E2B6F2E6B0A0E2D6FC4
:10584000D1EFEBF0E8CF37F10101370508E1F90EB0
:10585000166FE40E156F0A0E176F96EF2EF0F90E05
:105860002C6FE40E2B6F2E6B0A0E2D6FD1EFEBF029
:10587000E8CF37F10101370508E1FB0E166FEF0E97
:10588000156F080E176F96EF2EF0FB0E2C6FEF0EB4
:105890002B6F2E6B080E2D6FD1EFEBF08B92030E5A
:1058A0009FEC2FF0010118519FEC2FF001011751CF
:1058B0009FEC2FF016519FEC2FF0000E9FEC2FF075
:1058C0001A6F8B821A5112008D9096908482969254
:1058D00000F08D8000F000F08DB005D00101B367BD
:1058E00002D0010EB36F849200F000F000F08D90B2
:1058F00000F01200196B1A6B15A104D0175119276B
:1059000018511A23D89017371837D89016331533F3
:1059100016511511F1E119C115F11AC116F1120054
:105920000101B56706D0010EB56F0A840001F96B5D
:105930001200B50507E1020EB56F0001F96B020117
:10594000926B1200B56B00010B821200F2920FA253
:1059500003D00F92F19C8A820FA406D00F94F19C81
:1059600000010FBC8A8212008A92010E0201536F5D
:1059700000010E8C010C000108B6050C000113BAE1
:10598000050CFF0E01012C6FE00E2B6F000E2E6B2D
:105990002D6BD1ECEBF001E2000C07EFF2F004010B
:1059A00024510F0B080D000EF3240401C76FC86BC0
:1059B000040EC823040124AF1200040E0401C727FB
:1059C000000EC823000C8B92020E9FEC2FF00101F9
:1059D00018519FEC2FF0010117519FEC2FF0165139
:1059E0009FEC2FF01A519FEC2FF08B8212000001D8
:1059F0000BA00CD002017051D8A470077067120080
:105A000086EC2FF0320E706F6E2B320CF2EC2FF012
:105A100002016E6B1200040124510F0B080D000EE1
:105A2000F3240401C76FC86B040EC823040124AF1C
:105A30001200040E0401C727000EC823000CF90E43
:105A40000101176F1B0E166F010E28EC1DF0EAEC1A
:105A50002FF0D2EC2FF0E90E0101295D030E2A5937
:105A6000D8B01200F6D7E8CF17F1010E166F175114
:105A7000200A09E01751800A720F04E21751800AC8
:105A8000770FD8A0166B16C115F11531120096824A
:105A900096900001039A8D8000F08DB005D0010131
:105AA000B36702D0010EB36F00F084A202D00001F0
:105AB000038A8D901200E8CF15F10201246B256B4B
:105AC000000E236F0A0E226F00011B969EB803D0B2
:105AD00000011BA6FBD715C1AEFF1200E8CF1FF0D7
:105AE0001E6A090E1F6405D01E2A0A0E1F5E1F6063
:105AF000FBD71FC01DF00F0E1D161E38F00B1D101A
:105B000012001EC1AFF11FC1B0F1186B590E176F13
:105B10001F51196F84EC1FF00101186B5A0E176F9B
:105B20001EC119F184EF1FF0040118BF000C200EF4
:105B30000401CD6101D0000CA0A8000C040119677C
:105B400003D0E7EC2EF0000C040119511200E8CF4D
:105B500015F10201246B256B000E236F0A0E226FD4
:105B600000011B96A4B803D000011BA6FBD715C1EA
:105B7000A9FF1200E8CF15F1600E0101156503D0F1
:105B80001551A90F1200400E156503D01551C90F0C
:105B900012001551D00F1200040118BF1200200E80
:105BA0000401CD6101D0200CA0A8120004011967E6
:105BB00002D0DAEF2EF00401195112008696989661
:105BC000080E3F6E3F2EFED702019DB19886010E52
:105BD0000101016F870E006F45EC26F03D2A12008F
:105BE0009886080E3F6E3F2EFED73E2E05D0400E03
:105BF0003E6E3D2A6EEF29F00201D8909D333D069E
:105C0000DEEF2DF017AC0CD0179C8B9C0CA004D0B1
:105C1000320E0001F96F320C0F0E0001F96F0F0CFC
:105C2000178C8B8CF3D7E8CF17F1166B1751800ABE
:105C3000250F06E21751800A3F0F02E3010E166F8F
:105C400016C115F1153112004F0E186FD40E176FD3
:105C50001F51196F84EC1FF04F0E0101186FD50E04
:105C6000176F1EC119F184EF1FF0E8CF1FF01E6AF5
:105C70001F50800A460F06E21F50800A500F02E3B1
:105C8000010E1E6E1EC01DF01D301200E8CF17F170
:105C9000166B1751800A460F06E21751800A500F03
:105CA00002E3010E166F16C115F115311200E8CF8F
:105CB00015F10F0E010115170A0E156104D0300EF3
:105CC000152715511200370E152701011551120025
:105CD00002016E6702D0A7EF2FF06E0502E1F7EF29
:105CE0002CF06E51020A02E178EF2EF06E6B12007A
:105CF000702F1200F2EC2FF0230E2A5D000E2B59AC
:105D0000320ED8B0FA0E706F010E6E6F010CFB0EE2
:105D10000101176FB90E166F010E28EC1DF0130E5E
:105D200001012A6F880E296FBAEF21F0E0EC2FF005
:105D30000009FCE115C1B3F416C1B4F417C1B2F403
:105D4000010E0401B16F010CD9EC2FF01FEC2DF006
:105D500004ECAFF01CEC05F070ECCFF0148C0001FB
:105D6000188C1200E8CF4EF1000112A407D00101F7
:105D70004E0504E1A4EC2EF0D8801200D890120059
:105D8000E8CF15F11551800A250F05E21551800A5B
:105D90003F0FD8B0158B15511200E8CF15F11551F2
:105DA000800A050F05E21551800A1F0FD8B0159B18
:105DB00015511200400E0401181B040E1B6F300E0B
:105DC0001A6F400E196F1817880E1813880C400EA2
:105DD0000401181B040E1B6F300E1A6F400E196F52
:105DE0001817880E1813880C0001F851D8A4F8076A
:105DF000F867120086EC2FF04506640EF86F640C0D
:105E0000E8CF25F025AA03D01E6A900E02D01E6AA4
:105E1000920E1D6E9FEF07F04F0E186FD60E176F84
:105E2000000E196B84EC1FF06FEC28F06EEF2AF077
:105E30000001F851D8A4F807F867120086EC2FF09B
:105E4000452A120EF86F120C02016A6702D08FEF1A
:105E50002FF06A0502E197EF2FF06A6B1200869629
:105E600098960B0E0101016FC40E006F45EC26F0F1
:105E70003D2A12000001F82F68EF2EF0F2EC2FF00F
:105E8000456A02016A6B68EF2EF098862F0E0101B9
:105E9000016F100E006F45EC26F03D2A1200988627
:105EA000010E0101016F870E006F45EC26F03D2ABF
:105EB0001200F0925E0E776E786AA496A3860001B7
:105EC000148E12000001F82F1200F2EC2FF0452A78
:105ED000090EF86F090CE8CF15F1010115A902D0E0
:105EE000D8801200D89012000401D56B0401CC9F19
:105EF000A28815EC28F005EFE2F0A0B8A1A81200E6
:105F00003CECE1F0CCEC2DF0A1981200AA0ECB6E87
:105F1000550EBC6ECC6ACA843F0EBB6E3F0C0001AE
:105F20000AA8120086EC2FF002016A2B1200000171
:105F30000AB81200F2EC2FF002016A6B1200E8CFEF
:105F400015F115C1C9FFC7A0FED7C95012000BA09B
:105F500024EF2FF0320E0201706F6E2B320CE8CF5F
:105F600015F1010115510001EF1B1200400E040153
:105F70001C1B1C17880E1C13880C000105B402D0D2
:105F8000D8901200D8801200400E04011C1B1C1770
:105F9000880E1C13880C17C1F8FF16C1F7FF15C136
:105FA000F6FF1200A6ECDAF02CC229F12DC22AF17C
:105FB00012001294189C0201636B000118961200E3
:105FC000A0A8010C0401B1511200E8CF15F115C1D0
:105FD0000CF2120002012C6B2D6B120005940001D3
:105FE000ED511200CA94BB6A1200FFFFFFFFFFFFD2
:105FF000FFFFFFFFFFFFFFFFFFFFFFFFFFFFFFFFB1
:10600000FFFFFFFFFFFFFFFFFFFFFFFFFFFFFFFFA0
:10601000FFFFFFFFFFFFFFFFFFFFFFFFFFFFFFFF90
:10602000FFFFFFFFFFFFFFFFFFFFFFFFFFFFFFFF80
:10F04000FFFF30352F30312F30312C30303A303017
:10F050003A30300051495552433A2022636C6F7365
:10F0600065642200434D53204552524F523A20319D
:10F07000393300434D53204552524F523A203531D7
:10F080003500434D45204552524F523A203133000E
:10F09000434D45204552524F523A2031310051499B
:10F0A0005552433A2022726563762200434F4E4EFA
:10F0B000454354204641494C0051534D54505055FE
:10F0C000543A202D0001000A006400E80310274391
:10F0D00053513A20302C30004352494E473A2000D9
:10F0E000434D54493A2000435245473A2000434C8F
:10F0F0004F53454400735F6C6F636B002B4350426A
:10F1000052002B43504257002B434D47520022419F
:10F11000434B220009024300020100C064090400BD
:10F12000000102020000052400100104240202056F
:10F1300024060001052401000107058203080002DE
:10F1400009040100020A0000000705030240000153
:10F15000070583024000011201100102000008D8D7
:10F16000040A00010000000001466C617368696ECA
:10F17000672120446F6E277420706F776572206F4F
:10F180006666210D0A002B515552434346473D22E6
:10F19000757263706F7274222C22756172743122E1
:10F1A0000D002B51534D54504346473D22736D740F
:10F1B00070736572766572222C22002B514346478C
:10F1C0003D226E777363616E6D6F6465222C302C07
:10F1D000310D002B51494346473D227064702F7218
:10F1E00065747279222C302C310D002B5149434625
:10F1F000473D227064702F7265747279222C312C15
:10F20000310D002B51534D54504346473D22636FFF
:10F210006E746578746964222C3100464C41534801
:10F22000494E4720554E415641494C41424C450DAF
:10F230000A00556E706C75672074686520555342DE
:10F24000206361626C650D0A002B43504D533D22D3
:10F25000534D222C22534D222C22534D220D002B94
:10F2600051534D54504346473D226163636F756E61
:10F2700074222C22002B51534D54504346473D22BB
:10F2800073736C74797065222C30002B4347514D99
:10F29000494E3D312C302C302C302C302C300D0090
:10F2A0002B4347515245513D312C302C302C302CC2
:10F2B000302C300D002B51534D54504346473D22C6
:10F2C00073656E646572222C22002B514346473DC4
:10F2D000226E777363616E6D6F6465220D00233457
:10F2E0003A30323030303030323030303046430D0A
:10F2F0000A00495320414C5245414459204C4F4348
:10F300004B45440D0A002B51494F50454E3D312C81
:10F31000302C22544350222C22002B514955524369
:10F320003A202272656376222C302C002B51534DEB
:10F330005450424F44593D302C312C350D0023346C
:10F340003A303030303030303146460D0A0D0A0048
:10F350002B434744434F4E543D312C224950222CDD
:10F3600022002B434E4D493D332C312C302C302C78
:10F37000300D002B43434C4B3D2230302F30312F8A
:10F3800030312C0053544154453A20434F4E4E45A2
:10F3900043544544005761697420666F7220686564
:10F3A000782E2E0D0A00554E53454E545F42554659
:10F3B0005F46554C4C0D004350494E3A204E4F5439
:10F3C00020494E534552004350494E3A204E4F5427
:10F3D0002052454144590053494D5320554E4C4FFE
:10F3E000434B45440D0A0030362C25732C383430FD
:10F3F0003939303025640030372C25732C383430BF
:10F400003939303025640030362C25732C383431AE
:10F410003939303025640030372C25732C3834319D
:10F420003939303025640030362C25732C38353886
:10F43000393930302564002B51534D5450445354C6
:10F440003D312C312C22002B51534D5450505554EA
:10F450003D3130300D00434D45204552524F523A18
:10F4600020313030004845582053495A45204552F4
:10F47000520D0A005465737454696D653A20256411
:10F480002C200030362C25732C383530393930306B
:10F49000300030372C25732C383530393930303046
:10F4A0000030362C25732C3830313939303030006B
:10F4B00030362C25732C3832313939303030003029
:10F4C000362C25732C383232393930303000303711
:10F4D0002C25732C38323239393030300030362C0C
:10F4E00025732C38323339393030300030362C2502
:10F4F000732C38303439393030300030362C2573A5
:10F500002C38323439393030300030372C25732CD8
:10F5100038303839393030300030362C25732C38BB
:10F52000323939393030300030372C25732C3832AD
:10F530003939393030300030362C25732C3833339C
:10F5400039393032300030372C25732C3833333989
:10F55000393032300030362C25732C38333039397D
:10F560003030310030372C25732C38333039393076
:10F5700030310030362C25732C3830323939303068
:10F58000310030372C25732C383032393930303156
:10F590000030362C25732C38353439393030310071
:10F5A00030362C25732C3835353939303031003030
:10F5B000372C25732C383535393930303100303619
:10F5C0002C25732C38333039393030320030372C19
:10F5D00025732C38333039393030320030362C2511
:10F5E000732C38303239393030320030372C2573B3
:10F5F0002C38303239393030320030362C25732CEB
:10F6000038353439393030320030362C25732C38C7
:10F61000353539393030320030372C25732C3835B8
:10F620003539393030320030362C25732C383330B0
:10F6300039393030330030372C25732C383330399A
:10F64000393030330030362C25732C383534393985
:10F650003030330030362C25732C38333039393084
:10F6600030340030372C25732C3833303939303072
:10F67000340030362C25732C383534393930303459
:10F680000030362C25732C38333039393030350082
:10F6900030372C25732C3833303939303035003041
:10F6A000362C25732C38333039393030360030372A
:10F6B0002C25732C38333039393030360030362C25
:10F6C00025732C38343039393025640030372C25F7
:10F6D000732C38343039393025640030362C25739A
:10F6E0002C38343139393025640030372C25732CCF
:10F6F00038343139393025640030362C25732C38B4
:10F7000035383939302564002B51464C44533D225D
:10F71000554653220D002B51534D54505355423DE5
:10F72000302C22002B51534D54505355423D312C17
:10F73000220051534D54505055543A20302C300033
:10F74000434D45204552524F523A203130004350EC
:10F75000494E3A2053494D2050494E004970525469
:10F76000696D653A25646D2C20002B5149444E5338
:10F770004346473D312C22002B435343533D2249FE
:10F780005241220D0051534D5450424F44593A209A
:10F790002D0051534D5450424F44593A20310043AB
:10F7A0004F4E4E454354204641494C00762E256429
:10F7B0005F6D6F6465300D0A00762E25645F6D6F96
:10F7C0006465310D0A004845582057522045525271
:10F7D0000D0A005349412049503A4F46462C20001B
:10F7E000477072734174743A25642C2000222C22D5
:10F7F000382E382E382E38220D002B514953454EC5
:10F80000443D302C300D002B4950523D31393230BF
:10F81000300D002B434F50533D342C302C220031FF
:10F82000363030203939203030300031333031201B
:10F8300039392030303000333330312039392030FD
:10F84000303000313330322039392030303000331D
:10F8500033303220393920303030003136303220E8
:10F8600039392030303000313339332039392030C4
:10F8700030300031313430203939203030310033EC
:10F8800031343020393920303031003131343020BA
:10F89000393920303032003331343020393920309A
:10F8A00030320031313430203939203030330033B8
:10F8B000313430203939203030330051494E4953EA
:10F8C0005441543A20320051494E49535441543A1C
:10F8D0002037004350494E3A20524541445900498F
:10F8E00053204C4F434B45440D0A005374617941FA
:10F8F000282564292C20005349412049503A4F4E75
:10F900002C20005154696D653A2564732C20004603
:10F910006F7263654F66663A2564002B5149444512
:10F920004143543D310D002B5149444E534346470A
:10F930003D22002B5149435347503D312C33002B7E
:10F940004346554E203D20310D002B51494353472E
:10F95000503D310D002B4356455253494F4E0D003B
:10F960002B51494E49535441540D0051534D54505D
:10F970005055543A200043475245473A20312C30E5
:10F980000043475245473A20312C31004347524506
:10F99000473A20312C320043475245473A20312C18
:10F9A000330043475245473A20312C3400434752F5
:10F9B00045473A20312C3500434F4E4E45435420A5
:10F9C0004F4B0048455820455252310D0A004845DA
:10F9D0005820455252330D0A0049532057524F4E7A
:10F9E000470D0A00434F4445204552520D0A00532B
:10F9F000544154204552520D0A000D0A47432076C7
:10FA000025640D0A00504F5254313A25732C2000C2
:10FA1000504F5254323A25732C20007374616E6437
:10FA20006172742C200064696769706C65782C20A1
:10FA3000002B514953454E443D300D002B51534D41
:10FA40005450434C520D002B514953454E443D30C8
:10FA50002C002B43475245473D310D002B514E574B
:10FA6000494E464F0D002241444D2D43494422004A
:10FA7000514453494D3A20302C00514453494D3A9A
:10FA800020312C00435245473A20312C300043525C
:10FA900045473A20312C3100435245473A20312C1A
:10FAA0003200435245473A20312C330043524547F8
:10FAB0003A20312C3400435245473A20312C35004E
:10FAC000434D45204552524F5200434D532045521D
:10FAD000524F5200434F4445204F4B0D0A005241B4
:10FAE0004D204552520D0A00484558204552520DAE
:10FAF0000A00526573746172740D0A0047454E45E1
:10FB000052414C2C2000554E4B4E4F574E2C20004E
:10FB1000424154204C4F572C20006D6167656C6149
:10FB20006E2C2000756E6B6E6F776E2C2000536507
:10FB30006375726974793A002B51494143543D31E0
:10FB40000D002B43474154543D310D0053454E4465
:10FB5000204641494C002B435344483D300D002B77
:10FB6000434F50533D300D002B434D47443D310D25
:10FB7000002B434D45453D310D002B435245473D3C
:10FB8000310D002B434C49503D310D002B434D4767
:10FB9000443D320D002B434D47443D330D002B4374
:10FBA0004D47443D340D002B43475245473F0D0020
:10FBB0002B434D47463D300D002B434D47463D31CD
:10FBC0000D002B5149535441540D004347415454A7
:10FBD0003A20300043475245473A203100434741DD
:10FBE00054543A2031004445414354204F4B004582
:10FBF00045204552520D0A004353204552520D0AEA
:10FC0000002A2373696D5F6530004C4E723A25649B
:10FC10002C200053413A2025732C2000534D3A20CC
:10FC200025732C2000534E3A2025732C200053506E
:10FC30003A2025732C20004950313A25732C20009E
:10FC40004950323A25732C200041504E3A25732CEE
:10FC50002000444E533A25732C20005757573A251D
:10FC6000732C20006573707269742C200028435235
:10FC70004547256420004347524547256420004EF0
:10FC80006F5F43617264290053696D4C6F636B3A17
:10FC90000050616E537461743A006125732C2573B2
:10FCA0000D0A002B514453494D3F0D002B43474152
:10FCB00054543F0D002B4352433D310D002B435212
:10FCC00045473F0D002B434F50533F0D002B5143F1
:10FCD0004349440D002B4350494E3D22002B4343E2
:10FCE0004C4B3D2200302E302E302E30002B434323
:10FCF0004C4B3F0D002B434D47533D22000A303003
:10FD00003030303000435041533A203000434655A4
:10FD10004E3A203100434F4E4E4543540045525217
:10FD2000256429200044282564292C200070616E58
:10FD3000656C2C20004C3A2025732C20004F6E6CF3
:10FD4000696E653A0047454E4552414C00554E4B51
:10FD50004E4F574E002B4350494E3F0D002B43460C
:10FD6000554E3F0D00514953454E443A0053454EC0
:10FD700044204F4B00286E756C6C29002B43535563
:10FD8000420D002B43494D490D002B4347534E0D67
:10FD9000002B5147534E0D002B43474D520D002B66
:10FDA00051474D520D002B435042523D002B434DC5
:10FDB00047533D00434C49503A2000435042523A89
:10FDC0002000434F50533A200051495552433A00C6
:10FDD00051494F50454E00432F25640D0A004428D9
:10FDE00031292C200053494D312C2000647363319C
:10FDF0002C2000647363322C200042454C4C2C2094
:10FE000000475052532C2000414F66662C20004D75
:10FE10004F66662C20004C3A25732C2000503A2562
:10FE2000732C2000616275732C2000563A25643BC8
:10FE30002000434D4525642000434D532564200098
:10FE400053494D313A280028636F64652900557382
:10FE50006572733A00414354495645004241434B51
:10FE6000555000303030313030002B4353510D00AD
:10FE70002B3030220D002C3134352C002C3132390E
:10FE80002C002B434D474400224E414B220043534C
:10FE9000513A200043434C4B3A00434D47533A00FC
:10FEA00051434349440053494D31200053494D3299
:10FEB000200023343A3130006D6F646530006D6F7F
:10FEC000646531006D6F64653F006E636F6465004B
:10FED00072656465660073696D5F6C007366697254
:10FEE0006D002825642920002F2564292000475310
:10FEF0004D2C2000414F6E2C20004D4F6E2C2000C9
:10FF000028747874290053494D313A004F555431C3
:10FF10003A0053494D323A004F5554323A004D6F32
:10FF200064653A005245434F4E0053494D455200D7
:10FF3000534D534552004D3A202573005147534EBF
:10FF4000006C7461620073746162006C63666700C8
:10FF500073636667006C6C6F67006C746D70006C27
:10FF60007478740073747874006E782C2000257394
:10FF70003B20002F256429004F55543A0025732952
:10FF80003B004E4F4E450047505253004441595399
:10FF90000047525354004D52535400303030380013
:10FFA00045310D004F4E2F00495031002055310092
:10FFB000495032002055320020553300205534007E
:10FFC000494E3A004F4646004255460047534D00C1
:10FFD00045525200444E5300282564002F256400EA
:10FFE000510D0A00480D005530004C3000222C0005
:10FFF00039310041310023005B007C003E000000ED
:020000040001F9
:100000000101926B5F51156F030E6015166F186B2F
:100010000E0E176F7AEC2CF0040E1525956F040E5A
:100020001621966F6051946F9441E8423F0B070B85
:10003000946F95C11FF196C120F122EC1AF001E2F4
:10004000000C12A403D0010194051FE01CA404D0ED
:1000500001019451030A19E0010194519EECCAF088
:10006000EFE332C392F1996B0BD0F9EC8CF0620E96
:100070009925E16EE26A010EE222DFCFE7FF992BBC
:10008000030132510101995DF0E3A1054EE160AF3A
:1000900034D00301B0EC8CF09CEC8CF0310EDF6EB0
:1000A000992B330E77EC8CF05EEC8CF0616F61393C
:1000B0000F0B57EC2EF0DF6E992B5EEC8CF00F0BD4
:1000C00057EC2EF0E3EC8CF09865EED7330E6DEC28
:1000D0008CF0330E992582EC8CF057EC2EF089ECE5
:1000E0008CF057EC2EF0DF6E992B995151ECE4F027
:1000F000D9EC8CF0B5EC0BF015D00301E88115AE0E
:1001000009D0010E01011E6F000EF7ECF0F009ECB2
:100110008DF002D00101996B995135ECD5F002E2D6
:100120000101946B010194511200A151020A4FE1A7
:1001300060AF3AD00301B0EC8CF09CEC8CF0320E46
:10014000DF6E992B330E77EC8CF05EEC8CF0616FE8
:1001500061390F0B57EC2EF0DF6E992B5EEC8CF0B3
:100160000F0B57EC2EF0E3EC8CF09865EED7330EC6
:100170006DEC8CF0030E986F5EEC8CF0616F613962
:100180000F0B57EC2EF0DF6E992B5EEC8CF00F0B03
:1001900057EC2EF0DF6E992B982B040E9865ECD758
:1001A000995151ECE4F0A4D70301E88115AE09D0D0
:1001B000010E01011E6F000EF7ECF0F009EC8DF05E
:1001C00002D00101996B995135ECD5F0A8D7A15116
:1001D000030A4FE160AF3AD00301B0EC8CF09CEC25
:1001E0008CF0330EDF6E992B330E77EC8CF05EECD7
:1001F0008CF0616F61390F0B57EC2EF0DF6E992B8D
:100200005EEC8CF00F0B57EC2EF0E3EC8CF0986565
:10021000EED7330E6DEC8CF0030E986F5EEC8CF025
:10022000616F61390F0B57EC2EF0DF6E992B5EEC8E
:100230008CF00F0B57EC2EF0DF6E992B982B050EE0
:100240009865ECD7995151ECE4F052D70301E8815D
:1002500015AE09D0010E01011E6F000EF7ECF0F093
:1002600009EC8DF002D00101996B995135ECD5F074
:1002700056D7A151060A03E0A151070A5CE160AF1D
:1002800047D00301E86B0101996BA1390F0B57ECC3
:100290002EF00301336F01019CEC8CF0A1510F0B88
:1002A00057EC2EF0DF6E992B330E6DEC8CF0010EB7
:1002B000986F5EEC8CF0616F61390F0B57EC2EF08C
:1002C000DF6E992B5EEC8CF00F0B57EC2EF0E3EC0D
:1002D0008CF09865EED7330E6DEC8CF0030E986FB2
:1002E0005EEC8CF0616F61390F0B57EC2EF0DF6E16
:1002F000992B5EEC8CF00F0B57EC2EF0DF6E992BE8
:10030000982B060E9865ECD7995151ECE4F0F0D695
:100310000301E88115AE09D0010E01011E6F000E28
:10032000F7ECF0F009EC8DF002D00101996B9951D6
:1003300035ECD5F0F4D6A12901E082D6A4C1B7F1FD
:10034000A451190A09E0A451200A06E0A451210A87
:1003500003E0A451220A30E10301E86B010E010120
:10036000986FA451200A02E1020E986FA451210A4D
:1003700002E1030E986FA451220A02E1040E986F65
:1003800098519EECCAF001E25BD6996B07D0F9EC6C
:100390008CF0330E99256EECF2F0992B030132515B
:1003A0000101995DF4E3330E9925D96EDA6A030EE3
:1003B000DA22DF6A36EF8CF0A4518A0A01E0D1D04C
:1003C0000301E86B030E0101A4EC8CF0EBECD8F018
:1003D0002151986F98C199F11BB823D00101976BF7
:1003E00095EC8CF0CD0E9725186F196B000E192324
:1003F000E7EC19F0DF6E95EC8CF0DF5004E0972B02
:100400000F0E9765EDD7330E51EC8CF0FC0E246F78
:10041000370E236F010E266F720E256FEBECD8F0AE
:100420001ED0330E51EC8CF0FC0E246F5B0E236F4C
:10043000060E266F840E256FEBECD8F02151986FD5
:1004400098519927330E51EC8CF0FC0E246F520E0C
:10045000236F050E266FB70E256FEBECD8F058EC26
:100460008CF095EC8CF0C80E9725186F196B000E68
:100470001923E7EC19F0DF6E95EC8CF0DF5004E007
:10048000972B040E9765EDD7330E51EC8CF0FA0ED6
:10049000246F050E236F010E266F720E256FEBEC95
:1004A000D8F058EC8CF095EC8CF08A0E9725186FEC
:1004B000196B010E1923E7EC19F0DF6E95EC8CF047
:1004C000DF5004E0972B0F0E9765EDD7330E51ECFC
:1004D0008CF0FC0E246F400E236F010E266F720EFF
:1004E000256FEBECD8F058EC8CF095EC8CF0850E89
:1004F0009725186F196B010E1923E7EC19F0DF6EC1
:1005000095EC8CF0DF5004E0972B040E9765EDD747
:10051000330E51EC8CF0FA0E246F100E236F010E87
:10052000266F720E256FEBECD8F02151986F985121
:100530009927196B750E186FE7EC19F0986FD89022
:100540009833030E9817330E51EC8CF0F90E246F8C
:100550000F0E236F98C125F1266BEBECD8F036EF28
:100560008CF0A4518B0A01E00DD10301E86B01016D
:10057000996B030EA4EC8CF0EBECD8F02151986F42
:1005800098519927330E51EC8CF0F40E246F740EB1
:10059000236F95C225F1266BEBECD8F02151986FB3
:1005A00098519927330E51EC8CF0F90E246F030EFD
:1005B000236F7DC225F1266BEBECD8F02151986FAB
:1005C00098519927330E51EC8CF0F70E246F5E0E84
:1005D000236FF4C025F1266BEBECD8F02151986F16
:1005E00098519927330E51EC8CF0F70E246F5C0E66
:1005F000236F79C225F1266BEBECD8F02151986F6F
:1006000098519927330E51EC8CF0F70E246FE00EC1
:10061000236F73C225F1266BEBECD8F02151D5EC9A
:100620008CF01CA00AD0330E51EC8CF0F80E246F25
:10063000F70E236FEBECD8F009D0330E51EC8CF0B1
:10064000F70E246FD30E236FEBECD8F02151986F87
:1006500098519927330E51EC8CF0FC0E246F0A0E42
:10066000236FB8C125F1266BEBECD8F02151986FC0
:1006700098519927330E51EC8CF0FF0E246F0C0E1D
:10068000236FEBECD8F02151D5EC8CF00CA20DD0FF
:10069000330E51EC8CF0FA0E246FFC0E236FEBEC52
:1006A000D8F02151D5EC8CF02ED00DA20AD0330E0B
:1006B00051EC8CF0FE0E246FEE0E236FEBECD8F0B5
:1006C000F0D70CA80AD0330E51EC8CF0FE0E246F3C
:1006D000010E236FEBECD8F0E4D708AA0AD0330E52
:1006E00051EC8CF0FD0E246FFA0E236FEBECD8F07A
:1006F000D8D7330E51EC8CF0FB0E246F060E236F0F
:10070000EBECD8F0CED7330E51EC8CF0FF0E246F0B
:10071000180E236FEBECD8F02151D5EC8CF00CA423
:100720000FD0330E51EC8CF0FD0E246F450E236F6D
:10073000EBECD8F02151986F9851992736EF8CF057
:100740000DA40AD0330E51EC8CF0FF0E246FCC0EAA
:10075000236FEBECD8F0EED70CAA0AD0330E51EC95
:100760008CF0FF0E246F870E236FEBECD8F0E2D7EE
:10077000330E51EC8CF0FD0E246F4D0E236FEBEC1D
:10078000D8F0D8D7A4518C0A01E0F1D00301E86B6E
:10079000030E0101A4EC8CF0EBECD8F02151986F22
:1007A00098C199F1330E51EC8CF0FF0E246F6E0E50
:1007B000236F060E266FCF0E256FEBECD8F021517C
:1007C000986F98519927330E51EC8CF0FF0E246FDF
:1007D0006E0E236F060E266F640E256FEBECD8F0BD
:1007E0002151986F98519927330E51EC8CF0FF0EE0
:1007F000246F6E0E236F060E266FBF0E256FEBEC77
:10080000D8F02151986F98519927330E51EC8CF004
:10081000FE0E246F400E236FEBECD8F058EC8CF0FA
:1008200095EC8CF0ED0E9725186F196B000E1923BF
:10083000E7EC19F0DF6E95EC8CF0DF5004E0972BBD
:10084000080E9765EDD7330E51EC8CF0FE0E246F39
:10085000160E236F010E266F720E256FEBECD8F08B
:1008600058EC8CF095EC8CF0F60E9725186F196B00
:10087000000E1923E7EC19F0DF6E95EC8CF0DF50D9
:1008800004E0972B080E9765EDD7330E51EC8CF0F2
:10089000FE0E246F1D0E236F010E266F720E256F44
:1008A000EBECD8F058EC8CF095EC8CF0980E97258A
:1008B000186F196B000E1923E7EC19F0DF6E95EC39
:1008C0008CF0DF5004E0972B1A0E9765EDD7330EAE
:1008D00051EC8CF0FC0E246F490E236F010E266F35
:1008E000720E256FEBECD8F058EC8CF01E0E010167
:1008F0009725D96EDA6A060EDA22720E9725E16E16
:10090000E26A010EE222DFCFE7FF95EC8CF0DF50C8
:1009100004E0972B130E9765E9D7330E51EC8CF05A
:10092000FF0E246F7D0E236F010E266F720E256F52
:10093000EBECD8F02151986F010E1C6F720E1B6FFB
:10094000FA0E1E6FC40E1D6F206B050E1F6FD5ECC7
:1009500011F01C511B1101E0EFD6330E51EC8CF05D
:10096000FC0E246F7F0E236FEBECD8F0E3D6A4517E
:100970008D0A01E09BD30301E86B030E0101A4EC97
:100980008CF0EBECD8F02151986F98C199F1330EAF
:1009900051EC8CF0FF0E246F1E0E236FEBECD8F0A1
:1009A0002151D5EC8CF0B9670AD0330E51EC8CF0A4
:1009B000FA0E246F1B0E236FEBECD8F070D0B951F8
:1009C000080A0AE1330E51EC8CF0FE0E246F240E5F
:1009D000236FEBECD8F063D0B951040A0AE1330E6F
:1009E00051EC8CF0FC0E246F640E236FEBECD8F00E
:1009F00056D0B951060A0AE1330E51EC8CF0FB0EC9
:100A0000246F1A0E236FEBECD8F049D0B9510C0AC1
:100A10000AE1330E51EC8CF0FD0E246FEC0E236FC7
:100A2000EBECD8F03CD0B951020A0AE1330E51EC9C
:100A30008CF0FD0E246F2D0E236FEBECD8F02FD031
:100A4000B9510A0A0AE1330E51EC8CF0FD0E246F05
:100A5000F30E236FEBECD8F022D0B9510E0A0AE165
:100A6000330E51EC8CF0FA0E246F260E236FEBEC54
:100A7000D8F015D0B9050AE1330E51EC8CF0FF0E19
:100A8000246F690E236FEBECD8F009D0330E51ECD4
:100A90008CF0FB0E246F240E236FEBECD8F0215169
:100AA000986F98519927330E51EC8CF0FF0E246FFC
:100AB000060E236FEBECD8F02151D5EC8CF011A48D
:100AC0000DD0330E51EC8CF0FF0E246F820E236F8D
:100AD000EBECD8F02151D5EC8CF016D016AE0AD044
:100AE000330E51EC8CF0FF0E246FD00E236FEBEC25
:100AF000D8F0F0D7330E51EC8CF0FE0E246F550E6B
:100B0000236FEBECD8F0E6D7330E51EC8CF0FD0EF2
:100B1000246FE20E236FEBECD8F02151986F9851BF
:100B20009927330E51EC8CF0FF0E246F120E236FB9
:100B3000EBECD8F02151D5EC8CF011A60DD0330E92
:100B400051EC8CF0FF0E246F820E236FEBECD8F08B
:100B50002151D5EC8CF016D016AE0AD0330E51ECE4
:100B60008CF0FE0E246F550E236FEBECD8F0F0D70F
:100B7000330E51EC8CF0FE0E246F5C0E236FEBEC09
:100B8000D8F0E6D7330E51EC8CF0FD0E246FE20E58
:100B9000236FEBECD8F02151986F98519927330EC1
:100BA00051EC8CF0FF0E246FC00E236FEBECD8F0ED
:100BB0002151D5EC8CF0BCA10CD0330E51EC8CF053
:100BC000FB0E246FDB0E236FEBECD8F02151D5EC3C
:100BD0008CF0BCA30CD0330E51EC8CF0F80E246FCB
:100BE000C50E236FEBECD8F02151D5EC8CF0BCA5F1
:100BF0000CD0330E51EC8CF0FA0E246FAA0E236F3A
:100C0000EBECD8F02151D5EC8CF0BCA70CD0330E16
:100C100051EC8CF0FA0E246FB40E236FEBECD8F08D
:100C20002151D5EC8CF0BCA90CD0330E51EC8CF0DA
:100C3000FA0E246FBE0E236FEBECD8F02151D5ECE9
:100C40008CF0BCAB0CD0330E51EC8CF0F60E246F54
:100C5000AC0E236FEBECD8F02151D5EC8CF0330EB9
:100C600051EC8CF0FD0E246FE20E236FEBECD8F00C
:100C70002151D5EC8CF007A80CD0330E51EC8CF040
:100C8000FB0E246F100E236FEBECD8F02151D5EC46
:100C90008CF0330E51EC8CF0FF0E246F780E236F26
:100CA000EBECD8F02151D5EC8CF08AAE0CD0330EA1
:100CB00051EC8CF0F80E246FC50E236FEBECD8F0DE
:100CC0002151D5EC8CF08AAC0CD0330E51EC8CF069
:100CD000FB0E246FDB0E236FEBECD8F02151D5EC2B
:100CE0008CF0330E51EC8CF0FD0E246FE20E236F6E
:100CF000EBECD8F02151D5EC8CF012AA68D0330E71
:100D000051EC8CF0FC0E246F910E236FEBECD8F0BD
:100D10002151D5EC8CF008AC0CD0330E51EC8CF09A
:100D2000FD0E246FFA0E236FEBECD8F02151D5ECB9
:100D30008CF00101196B540E186FE7EC19F0936FEA
:100D40009351F00B0BE1330E51EC8CF0FD0E246F40
:100D5000250EB8EC8CF0EBECD8F036D09351F00BBC
:100D6000100A0BE1330E51EC8CF0F80E246FEF0EED
:100D7000B8EC8CF0EBECD8F027D09351F00B200AB4
:100D80000BE1330E51EC8CF0FD0E246F250EB8EC08
:100D90008CF0EBECD8F018D09351F00B300A0BE14B
:100DA000330E51EC8CF0F80E246FEB0EB8EC8CF097
:100DB000EBECD8F009D0330E51EC8CF0FD0E246F23
:100DC000DE0E236FEBECD8F02151D5EC8CF0330E16
:100DD00051EC8CF0FE0E246F4E0E236FEBECD8F02E
:100DE0002151986F98519927010E9EECCAF028E383
:100DF000330E51EC8CF0FF0E246FAC0E236FEBEC36
:100E0000D8F02151986F98519927010EB6EC2AF02D
:100E100000090AE1330E51EC8CF0FF0E246F000E36
:100E2000236FEBECD8F009D0330E51EC8CF0FE0EB2
:100E3000246F470E236FEBECD8F02151D5EC8CF0EA
:100E4000020E9EECCAF028E3330E51EC8CF0FF0E3C
:100E5000246FB40E236FEBECD8F02151986F9851AA
:100E60009927020EB6EC2AF000090AE1330E51EC84
:100E70008CF0FF0E246F000E236FEBECD8F009D03E
:100E8000330E51EC8CF0FE0E246F470E236FEBEC0B
:100E9000D8F02151D5EC8CF0030E9EECCAF028E37B
:100EA000330E51EC8CF0FF0E246FB80E236FEBEC79
:100EB000D8F02151986F98519927030EB6EC2AF07B
:100EC00000090AE1330E51EC8CF0FF0E246F000E86
:100ED000236FEBECD8F009D0330E51EC8CF0FE0E02
:100EE000246F470E236FEBECD8F02151D5EC8CF03A
:100EF000040E9EECCAF028E3330E51EC8CF0FF0E8A
:100F0000246FBC0E236FEBECD8F02151986F9851F1
:100F10009927040EB6EC2AF000090AE1330E51ECD1
:100F20008CF0FF0E246F000E236FEBECD8F009D08D
:100F3000330E51EC8CF0FE0E246F470E236FEBEC5A
:100F4000D8F02151D5EC8CF0330E51EC8CF0FD0E25
:100F5000246FE20E236FEBECD8F02151986F98517B
:100F60009927330E51EC8CF0FB0E246F2E0E236F5D
:100F7000EBECD8F02151986F985199274F0E196FCB
:100F8000D30E186FE7EC19F0616F61AD0AD0330E24
:100F900051EC8CF0F80E246FFE0E236FEBECD8F0C2
:100FA00009D0330E51EC8CF0F70E246FDA0E236F5C
:100FB000EBECD8F058EC8CF0330E51EC8CF0FC0ECE
:100FC000246F880E236FEBECD8F02151986F985165
:100FD0009927000E6CECF0F000090FE0330E51EC95
:100FE0008CF0FD0E246FE50E236FEBECD8F0215151
:100FF000986F010E976F98519927010197670FD04D
:10100000330E9925216F226B030E2223F70E246FD6
:10101000DA0E236FEBECD8F02151D5EC8CF0330EC7
:1010200051EC8CF0FD0E246F3D0E236FEBECD8F0ED
:101030002151D5EC8CF012A423D0330E51EC8CF05E
:10104000FF0E246FA40E236FEBECD8F02151D5ECEA
:101050008CF009A00BD0330E51EC8CF0FF0E246FF6
:10106000B00E236FEBECD8F036EF8CF0330E51EC72
:101070008CF0FF0E246FA80E236FEBECD8F0F6D3A4
:1010800014AA0AD0330E51EC8CF0FF0E246F240EFC
:10109000236FEBECD8F0EAD3330E51EC8CF0FF0E5B
:1010A000246FC40E236FEBECD8F0E0D3A4518E0A6A
:1010B00001E0EAD00301E86B1CA40CD0030E01018F
:1010C000226F330E216FFE0E246FFA0E236FEBECAE
:1010D000D8F00BD0030E0101226F330E216FFE0EEC
:1010E000246F0F0E236FEBECD8F02151986F98C14D
:1010F00099F1976B95EC8CF09A0E9725186F196BF8
:10110000010E1923E7EC19F0DF6E95EC8CF0DF503F
:1011100004E0972B1F0E9765EDD7330EC2DBFC0E54
:10112000246F130E236F010E266F720E256FEBECEA
:10113000D8F0BEDBFADBBA0E9725186F196B010EDB
:101140001923E7EC19F0DF6EF0DBDF5004E0972B9A
:10115000050E9765EFD7330EA4DBFC0E246F2E0E21
:10116000236F010E266F720E256FEBECD8F0A0DB1B
:10117000DCDBC00E9725186F196B010E1923E7EC05
:1011800019F0DF6ED2DBDF5004E0972B1F0E97655E
:10119000EFD7330E86DBFD0E246F350E236F010E65
:1011A000266F720E256FEBECD8F02151FEDB1CA2EE
:1011B00009D0330E76DBFE0E246FF40E236FEBECBA
:1011C000D8F008D0330E6DDBFE0E246F080E236FAF
:1011D000EBECD8F06DDBA9DBF10E9725186F196BDE
:1011E000010E1923E7EC19F0DF6E9FDBDF5004E0FE
:1011F000972B0F0E9765EFD7330E53DBFC0E246F42
:10120000250E236F010E266F720E256FEBECD8F0C2
:101210004FDB8BDB9729186F196B020E1923E7EC54
:1012200019F0DF6E82DBDF5004E0972B1F0E97650D
:10123000F0D7330E36DBFC0E246F1C0E236F010E2D
:10124000266F720E256FEBECD8F032DB6EDB210ED1
:101250009725186F196B020E1923E7EC19F0DF6E52
:1012600064DBDF5004E0972B1F0E9765EFD7330E3A
:1012700018DBFF0E246F360E236F010E266F720EE1
:10128000256FEBECD8F0F2D2A4518F0A01E069D2BD
:101290000301E86B0101996B030E226F330E216F7E
:1012A000FF0E246F8C0E236FEBECD8F02151986F5A
:1012B00098519927500E196FBF0E186FE7EC19F06F
:1012C000616F500E196FBE0E186FE7EC19F0966F34
:1012D0006151956F330EE5DA56DBEBECD8F0215116
:1012E000986F98519927500E196FC10E186FE7EC3F
:1012F00019F0616F500E196FC00E186FE7EC19F0FE
:10130000966F6151956F330ECCDA46DBEBECD8F07B
:101310002151986F98519927330EC3DAFF0E246F2D
:10132000A80E236FEBECD8F02151986F98519927B4
:10133000500E196FC50E186FE7EC19F0616F500E63
:10134000196FC40E186FE7EC19F0966F6151956F25
:10135000330EA7DA18DBEBECD8F02151986F9851D7
:101360009927500E196FC30E186FE7EC19F0616FD3
:10137000500E196FC20E186FE7EC19F0966F61519D
:10138000956F330E8EDA23DBEBECD8F02151986F9A
:1013900098519927500E196FCB0E186FE7EC19F082
:1013A000616F500E196FCA0E186FE7EC19F0966F47
:1013B0006151956F330E75DAEFDAEBECD8F021510D
:1013C000986F98519927330E6CDAFF0E246FB00E88
:1013D000236FEBECD8F02151986F98519927500E5C
:1013E000196FC90E186FE7EC19F0616F500E196F85
:1013F000C80E186FE7EC19F0966F6151956F330EB8
:1014000050DAC1DAEBECD8F02151986F9851992756
:10141000500E196FC70E186FE7EC19F0616F500E80
:10142000196FC60E186FE7EC19F0966F6151956F42
:10143000330E37DACCDAEBECD8F02151986F9851B3
:101440009927500E196FCD0E186FE7EC19F0616FE8
:10145000500E196FCC0E186FE7EC19F0966F6151B2
:10146000956F330E1EDA98DAEBECD8F02151986FB5
:1014700098519927330E15DAFF0E246F2A0E236F29
:10148000EBECD8F02151986F98519927500E196FB5
:10149000CF0E186FE7EC19F0616F500E196FCE0E7A
:1014A000186FE7EC19F0966F6151956F330EF9D90B
:1014B0006ADAEBECD8F02151986F98519927500EC9
:1014C000196FD10E186FE7EC19F0616F500E196F9C
:1014D000D00E186FE7EC19F0966F6151956F330ECF
:1014E000E0D95ADAEBECD8F02151986F985199274E
:1014F000330ED7D9FF0E246F300E236FEBECD8F0EC
:101500002151986F98519927500E196FE30E186F5B
:10151000E7EC19F0616F500E196FE20E186FE7ECEF
:1015200019F0966F6151956F330EBBD959DAEBEC18
:10153000D8F02151986F98519927330EB2D9FF0EE8
:10154000246FC80E236FEBECD8F02151986F98519F
:101550009927500E196FE10E186FE7EC19F0616FC3
:10156000500E196FE00E186FE7EC19F0966F61518D
:10157000956F330E96D934DAEBECD8F02151986F91
:1015800098519927330E8DD9FF0E246F910E236F3A
:10159000EBECD8F02151986F98519927500E196FA4
:1015A000DB0E186FE7EC19F0616F500E196FDA0E51
:1015B000186FE7EC19F0966F6151956F330E71D982
:1015C000FC0E246F6D0E236F95C125F196C126F197
:1015D000EBECD8F02151986F98519927500E196F64
:1015E000DD0E186FE7EC19F0616F500E196FDC0E0D
:1015F000186FE7EC19F0966F6151956F330E51D962
:10160000FC0E246F760E236F95C125F196C126F14D
:10161000EBECD8F02151986F98519927500E196F23
:10162000D70E186FE7EC19F0616F500E196FD60ED8
:10163000186FE7EC19F0966F6151956F330E31D941
:10164000FE0E246F320E236F95C125F196C126F14F
:10165000EBECD8F02151986F98519927500E196FE3
:10166000D90E186FE7EC19F0616F500E196FD80E94
:10167000186FE7EC19F0966F6151956F330E11D921
:10168000FE0E246F390E236F95C125F196C126F108
:10169000EBECD8F02151986F98519927500E196FA3
:1016A000DF0E186FE7EC19F0616F500E196FDE0E48
:1016B000186FE7EC19F0966F6151956F330EF1D802
:1016C000FD0E246F1D0E236F95C125F196C126F1E5
:1016D000EBECD8F02151986F98519927330EE1D84F
:1016E000FF0E246F960E236FEBECD8F02151986F0C
:1016F00098519927500E196FD30E186FE7EC19F017
:10170000616F500E196FD20E186FE7EC19F0966FDB
:101710006151956F330EC5D836D9EBECD8F0215115
:10172000986F98519927500E196FD50E186FE7ECE6
:1017300019F0616F500E196FD40E186FE7EC19F0A5
:10174000966F6151956F330EACD8FF0E246F730EF8
:10175000236F95C125F196C126F1EBECD8F09AEFF5
:1017600083F00201965127E00101A451260A09E005
:10177000A451270A06E0A451280A03E0A451290A2B
:1017800075E10201960506E1030E01013AD9EBEC81
:10179000D8F00ED09651020A0BE1030E0101226F20
:1017A000330E216FFA0E246FC40E236FEBECD8F0CA
:1017B0000201966B5BD00101A451300AD8B460BF1E
:1017C00005D0030E1ED9EBECD8F050D060AF37D067
:1017D0000301E86B00011CA02ED00101996B660E7D
:1017E0000301336F0101A8D8660EDF6E992B330E0B
:1017F0007ED864D8616F61390F0B57EC2EF0DF6E25
:10180000992B5CD80F0B57EC2EF0DDD89865F1D7EB
:10181000330E63D8330E992575D857EC2EF079D84E
:1018200057EC2EF0DF6E992B995151ECE4F0C1D8B2
:10183000B5EC0BF01BD0000E01ECA8F017D00301A3
:10184000E88115AE08D0010E01011E6F000EF7EC05
:10185000F0F0DFD802D00101996B995101ECA8F0AA
:10186000995135ECD5F002E20101946B92C132F34B
:101870000101996B10D0620E9925D96EDA6A010EBA
:10188000DA22220E01019925E16EE26A030EE222BC
:10189000DFCFE7FF992B9251995D02E392EF80F041
:1018A000EAD701019925216F226B030E2223120032
:1018B0002151986F98519927976B1200330E0101AF
:1018C0009925D96EDA6A030EDA22A10E9825E16E07
:1018D000E26A010EE222E750120001019925D96E59
:1018E000DA6A030EDA222C0EDF6E992B2C0C992566
:1018F000D96EDA6A030EDA222C0EDF6E992B010EF6
:10190000986F010CD96EDA6A030EDA22A4390F0B34
:101910001200DF6E992B330E01019925D96EDA6A18
:10192000030EDA22A4510F0B1200720E9725D96E06
:10193000DA6A010EDA221200992B330E9925D96E3C
:10194000DA6A030EDA221200226F330E216FFE0EC6
:10195000246F2B0E236F0D0E266F710E256F710CE9
:10196000E86B0101996B300E0301336F0101300CFC
:10197000236F93C161F10F0E61176129256F266BEB
:10198000000E2623000CFF0E246FD80E236F95C186
:1019900025F196C126F11200FE0E246FE80E236F8A
:1019A00095C125F196C126F11200986F985199279B
:1019B0001200410E01019925D96EDA6A0301030E66
:1019C000DA22DF6A000CDF6E992B982B020CFF0ED7
:1019D000246FDC0E236F95C125F196C126F112000C
:1019E000FE0E246FE20E236F95C125F196C126F1FC
:1019F0001200220E01019925D96EDA6A030EDA224D
:101A00001200226F330E216FFD0E246F720E236FB2
:101A10001200090E0101996F090C220E0301FF6FDC
:101A200009964686FE69468246804684060E040173
:101A3000FE6F7FECFBF0BE6B1AD083500F0BB96FBB
:101A4000270EB26F100EB16F01D004000101B10773
:101A5000D8A0B207B129D8B4B229F7E183500F0B4F
:101A6000B91904E0BE5103E0BE0701D0BE2BBE5140
:101A70000A0AE3E10F0EB91BB96705D0158A949CD9
:101A8000829C9484EBD0B951040A10E10A8E949C94
:101A90009484AD947E86090E7F6EC20EB06EAC8EBD
:101AA000AC88AD8A9E9A9F9A9D8AD8D0B951060A71
:101AB00008E1108A949C9484AD847E867F6A670EC8
:101AC000EDD7B9510E0A08E10984949C9484AD9431
:101AD0007E867F6A340EE2D7B90508E1118AF18863
:101AE000F092F08EF088060E766EB8D0B9510A0AE0
:101AF00003E0B9510C0A0AE10F800101B9510A0A49
:101B000001E10F86F19CF292F288A8D0B951080A3F
:101B10000DE10001058CFEEC2AF09896949C9484CB
:101B2000AD947E86010E7F6E370EB8D7B951020A8A
:101B300001E094D04F0E196FD60E186FE7EC19F034
:101B40009D6F9D050BE04F0E196FD60E186FE7ECD9
:101B500019F09D6F9D05D8A40CEC2FF0D00ED76E18
:101B6000F00ED66EF294F184F28AD58E949C949401
:101B700098868B9C030ECA6E128A98968696270EBC
:101B80000101B26F100EB16F01D004000101B10765
:101B9000D8A0B207B129D8B4B229F7E1BD6B040EC1
:101BA00053EC29F0BE6F3E0EBE6102D0BD9301D052
:101BB000BD83080E53EC29F0BE6F3E0EBE6102D00D
:101BC000BD9501D0BD850C0E53EC29F0BE6F3E0EC5
:101BD000BE6102D0BD9701D0BD87BD1F8686270E8E
:101BE000B26F100EB16F01D004000101B107D8A08F
:101BF000B207B129D8B4B229F7E1BF6B040E53EC98
:101C000029F0BE6F3E0EBE6102D0BF9301D0BF83EC
:101C1000080E53EC29F0BE6F3E0EBE6102D0BF9598
:101C200001D0BF850C0E53EC29F0BE6F3E0EBE6195
:101C300002D0BF9701D0BF87BD51BF19BE6FBEB3E1
:101C400003D00CEC2FF008D0BEB503D06FEC28F019
:101C500003D0BEA76EEC2AF086969886080E010186
:101C6000BE6F8D968D948A988A968D9C8D9A8D8C58
:101C70008D8A8D868D848A888A868F808C8EEA0EE6
:101C8000B26F600EB16F01D004000101B107D8A09E
:101C9000B207B129D8B4B229F7E18D9C8D9A8D96FF
:101CA0008D948A988A968F908C9EEA0EB26F600E01
:101CB000B16F01D004000101B107D8A0B207B1296A
:101CC000D8B4B229F7E1BE2FD2D7D08EF28EF28CE3
:101CD000196BFF0E1869E7EC19F00301FF1916E004
:101CE0000101196BFF0E1869E7EC19F00301FF19E8
:101CF0000DE01BECD2F00101186BFF0E1769FFC35A
:101D000019F184EC1FF0010E0101BE6F04ECAFF07D
:101D1000420E0101196F3B0E186FE7EC19F09D6F31
:101D20009D29D8B48F80130E196F890E186FE7ECB8
:101D300019F09D6F9D29D8B48F800501C75113E01C
:101D4000050E01011C6FC70E1B6FFC0E1E6FE50E0A
:101D50001D6F206B070E1F6FD5EC11F01C511B116E
:101D600002E01CA00E800501B75102E01CA00E800D
:101D70003CC2B1F13DC2B2F102013D6B020E3C6FBB
:101D800000014694EAEC2FF0D2EC2FF03D0E010159
:101D9000295D000E2A59F8E3B1C13CF2B2C13DF20F
:101DA0007BEC18F0B66B138600011388D5EC20F09D
:101DB00086CFBDF10101BDA916D0270EB26F100E5E
:101DC000B16FB107D8A0B2070101B129D8B4B229C7
:101DD000F8E186CFBDF1BDA906D000010E86000E48
:101DE000ADEC26F03FD002ECB7F011B83BD018862E
:101DF0001598138C500E0101186FC00E176F000E4E
:101E0000196B84EC1FF0500E0101186FC10E176F93
:101E1000000E196B84EC1FF0CEECD9F017A022D085
:101E20008D8C8D8AEA0E0101B26F600EB16F01D008
:101E300000F00101B107D8A0B207B129D8B4B22986
:101E4000F7E18D9C8D9AEA0EB26F600EB16F01D0F2
:101E500000F00101B107D8A0B207B129D8B4B22966
:101E6000DFE0F6D710BE13A201D00D8A10AE05D068
:101E700000010DAA02D0FF00FFD7000110AE05D06F
:101E80008D8C8D9A010EBEECABF010BE0EA615D057
:101E900086CFBDF10101BDB910D0270EB26F100E73
:101EA000B16FB107D8A0B2070101B129D8B4B229E6
:101EB000F8E186CFBDF1BDA9FF0010BE1BD086CFD3
:101EC000BDF10101BDA916D0270EB26F100EB16F82
:101ED000B107D8A0B2070101B129D8B4B229F8E1FD
:101EE00086CFBDF1BDA906D000010E86010EADEC76
:101EF00026F0B8D704B413AC0BD0139C8D9C14847B
:101F000015AA06D0040EBB6E9E949F949D84948C5B
:101F1000000110BE09D099ECEAF00201996F9951C5
:101F200003E09951DFECD0F012A606D002017F67E2
:101F300003D01FEC2DF01296040E02016D650AD03D
:101F40006D6B500E0101206FDE0E1F6FE6EC21F06D
:101F500002ECB7F003A803D003980201612B040E32
:101F6000020161650AD0616B500E0101206FDE0E27
:101F70001F6FE6EC21F002ECB7F002AE09D0500E74
:101F80000101206FD60E1F6FE6EC21F002ECB7F0D6
:101F900002AC09D0500E0101206FD60E1F6FE6EC87
:101FA00021F002ECB7F003A010D0039002015F2BE8
:101FB000010E5F650AD05F6B500E0101206FD80ED5
:101FC0001F6FE6EC21F002ECB7F003A210D00392F1
:101FD0000201602B010E60650AD0606B500E01019A
:101FE000206FD80E1F6FE6EC21F002ECB7F004A0D2
:101FF00004D00001049070ECCFF009A20FD0099238
:10200000500E0101206FBE0E1F6FE6EC21F0500E46
:102010000101206FC00E1F6FE6EC21F010AE0DA87D
:1020200071D015B86FD00AAE17D0020E0101176F2C
:10203000A70E166F0BEC2AF0020E0101276FA70EF8
:10204000266F2BECC7F05EE2020E0101166FA70EA1
:10205000156F70EC19F054D010AA0FD0020E0101C8
:10206000176FA70E166FBDEC29F0020E0101206F4D
:10207000A70E1F6F64ECC5F0E7D709A40FD0020EBE
:102080000101176FA70E166FBDEC29F0020E0101BA
:102090002A6FA70E296FF1ECC8F0D5D70FA00FD08B
:1020A000020E0101176FA70E166F6CEC23F0020EE3
:1020B0000101276FA70E266F7CECB4F0C4D711AADC
:1020C0000FD0020E0101176FA70E166F89EC29F0D1
:1020D000020E01011F6FA70E1E6F36ECEBF010D041
:1020E00005BC05B80FD0020E0101176FA70E166FC1
:1020F00000EC29F00201A751080A02E1058802D08C
:102100001588158610AE0FA03ED03F50080A25E175
:102110000FB606D002019D51EB0A1FE10B8E1DD0B8
:102120000101B4B51AD0B4A30FD002019D51A50A84
:1021300014E0020E0101B41702019D51EB0A0DE1FA
:10214000040E0101B46F09D002019D51A50A05E1F9
:102150000101B4B1E3D7B481B48318B40BD018A291
:1021600003D018920201936B020193A70CD018843C
:10217000128E09D00B8E18A206D018920201936B12
:1021800018940FAC138010AE05AC92D015B42AD0C1
:10219000020153678DD005A812D0058AAAC216F194
:1021A000A8C217F1010E0101186F0201A9511BEC21
:1021B000F8F01584059EF00E0201536F79D00201EC
:1021C0004D2B450E0101166F4DC217F1186B540EC1
:1021D0001BECF8F002014D510F0AEBE14D6B8F80C3
:1021E0001280E7D7020153670AD01594000105BA9F
:1021F00003D0E9EC06F05CD0059A059859D005AEFD
:1022000057D005AA02D0059A0598059E159402019B
:102210009D51240A06E09D515E0A03E09D51260A65
:1022200030E19D51240A02E1179404D09D515E0AC9
:1022300003E11784069002D01794068002014E51E4
:1022400022EE9EF0DF621DD03E50120A03E03E50A7
:10225000060A17E13E503CEC18F013E302019E51D0
:10226000BAEC2DF00201516F3E50120A1EE108AE89
:102270000BD0150E0101166F4DC217F1186B1BEC38
:10228000F8F0E9EC06F097D7060E0101166F4DC283
:1022900017F1186B1BECF8F0F8ECF8F0020E0101E6
:1022A000176F9D0E166F88EC2BF068EC26F083D725
:1022B00010AE11AA13D011AE08D0119E0201936B7B
:1022C00018A40CD01894138009D0020193A306D04F
:1022D000936B18B403D01884128E0B8E10BE04D0EA
:1022E000000112BAA6ECDAF010AE19B600D117A2AE
:1022F000FED0179216AE16A678D011B676D0000191
:1023000012A408D0D9EC2FF01FEC2DF0148C010E84
:102310000101BE6F310EFAECF4F0BD6FBD5166ECF9
:10232000F9F00DE2000116BA23D0168A1688500E75
:102330000101206FD00E1F6FE6EC21F019D00001D3
:102340000494EAEC2FF009D0000104A406D016AAE8
:102350000CD0169A168C0D9608D0D2EC2FF0410EA8
:102360000101295D9C0E2A59EFE3000104A4DAD78C
:10237000300EFAECF4F0BD6FBF6BBD5166ECF9F0B6
:102380000EE2010E0101BF6F16B221D01682168037
:10239000500E206FCE0E1F6FE6EC21F018D000011A
:1023A0000494EAEC2FF009D0000104A406D016A290
:1023B0000CD0169216840D9608D0D2EC2FF0410E58
:1023C0000101295D9C0E2A59EFE304A4DAD701012B
:1023D000BF5103E002ECB7F002D0F8EC1DF00101B0
:1023E000BE5101E184D0188C82D016BE11B47FD0CA
:1023F000000112A408D0D9EC2FF01FEC2DF0148CA2
:10240000010E0101BE6F300EFAECF4F0BD6FBF6B30
:10241000BD5166ECF9F00EE2010E0101BF6F16B27C
:1024200028D016821680500E206FCE0E1F6FE6EC5D
:1024300021F01FD000010494EAEC2FF009D0000134
:1024400004A406D016A20CD0169216840D9608D0BD
:10245000D2EC2FF0410E0101295D9C0E2A59EFE3C9
:1024600004B407D0010E0101BF6F16B202D016826C
:1024700016800101BF5137E0310EFAECF4F0BD6F68
:10248000BF6BBD5166ECF9F00EE2010E0101BF6FAA
:1024900016BA21D0168A1688500E206FD00E1F6FE4
:1024A000E6EC21F018D000010494EAEC2FF009D0FA
:1024B000000104A406D016AA0CD0169A168C0D960C
:1024C00008D0D2EC2FF0410E0101295D9C0E2A5953
:1024D000EFE304A4DAD70101BF5103E002ECB7F047
:1024E00002D0F8EC1DF00101BE5101E07CD710AE26
:1024F00018A6CED11896FE0E0101176F740E166F36
:10250000010E28EC1DF0130E01012A6F880E296FB1
:10251000BAEC21F00101BE6B16AE02D0010EBE6F07
:102520000101BE516CECF0F0020A07E102018F2BB1
:102530008F51020A04E1FF0002D002018F6BFA0EF4
:102540000101176F5C0E166F010E28EC1DF0880E4E
:102550000101296F130E2A6F000E2B6B2C6B2D6B54
:1025600068EC9EF00101BD6FF90E176F4A0E166FF1
:10257000010E28EC1DF0880E0101296F130E2A6F41
:10258000000E2B6B2C6B2D6B68EC9EF00101BD6F68
:10259000030EBE6F0201662B18D0FE0E176F6A0E77
:1025A000166F010E28EC1DF0880E0101296F130E25
:1025B0002A6F000E2B6B2C6B2D6B68EC9EF00101CB
:1025C000BD6FBD51230A04E0BE070101BE67E5D718
:1025D000BE512BE00201666B0101BF6B850E01014C
:1025E000BF25D96EDA6A050EDA22CF0EBF25E16E5D
:1025F000E26A060EE222DFCFE7FF850EBF25D96E25
:10260000DA6A050EDA22DF5004E0BF2B0F0EBF6539
:10261000E5D7880E0101296F130E2A6F2B6B2C6BE7
:10262000010E2D6F68EC9EF007D0020E0201666568
:1026300003D0666B02ECB7F0030E0101BE6F02011E
:10264000622B69D0FC0E176FC50E166F010E28ECB9
:102650001DF0880E0101296F130E2A6F000E2B6BDF
:102660002C6B2D6B68EC9EF00101BD6FA06BBF6BF6
:10267000850E0101BF25D96EDA6A050EDA22640ED5
:10268000BF25E16EE26A060EE222DFCFE7FFA0512E
:10269000030A0BE1850EBF25D96EDA6A050EDA2230
:1026A000370EDF6202D08C8A0ED00101A051030ADE
:1026B0000AE1850EBF25D96EDA6A050EDA22300EE0
:1026C000DF6201D08C9A850E0101BF25D96EDA6ACE
:1026D000050EDA222C0EDF6201D0A02B850E01013F
:1026E000BF25D96EDA6A050EDA22DF5004E0BF2B6F
:1026F0001F0EBF65BDD7880E0101296F130E2A6F0B
:102700002B6B2C6B010E2D6F68EC9EF00101BD51FF
:10271000130A04E0BE070101BE6794D7BE5103E06F
:102720000201626B07D0020E0201626503D0626B88
:1027300002ECB7F0C9ECF6F017E2500E0101206F81
:10274000DA0E1F6FE6EC21F002ECB7F016B211A61C
:1027500001D00D8616BA11A401D00D8616B216AAA4
:1027600001D00D8614BA188C030E0101BE6F020150
:102770005E2B4FD0FB0E176FA70E166F010E28ECC5
:102780001DF0880E0101296F130E2A6F000E2B6BAE
:102790002C6B2D6B68EC9EF00101BD6FBF6B850E3D
:1027A0000101BF25D96EDA6A050EDA22BF0EBF25F8
:1027B000E16EE26A060EE222DFCFE7FF850EBF255B
:1027C000D96EDA6A050EDA22DF5004E0BF2B0F0E55
:1027D000BF65E5D7880E0101296F130E2A6F2B6B99
:1027E0002C6B010E2D6F68EC9EF00101BD511C0A8F
:1027F00013E0BD511D0A10E0BD511E0A0DE0BD5190
:102800001F0A0AE0BD51200A07E0BD51210A04E079
:10281000BE070101BE67AED7BE510CE0BD51200A14
:1028200009E0BD511E0A06E0BD511F0A03E0020186
:102830005E6B0ED0040E02015E650AD05E6B500E18
:102840000101206FDC0E1F6FE6EC21F002ECB7F007
:10285000D40E01019D6F060E9E6F9DC11BF19EC19E
:102860001CF1B1ECFCF01B51BD6FBD51630A03E1DB
:102870000201746B0DD00B0EBD6102D0010E06D0AB
:10288000100EBD6102D0020E01D0030E0201746F62
:1028900010BE88D218B013A401D0138A13B418A0A4
:1028A000139A17BE07A801D0088607B817AE089676
:1028B00012B404A21DD00492F90E0101176F1B0E71
:1028C000166F010E28EC1DF0D9EC2FF0148C09B016
:1028D00008D0500E0101206FC20E1F6FE6EC21F0F0
:1028E00007D0500E0101206FC60E1F6FE6EC21F0DD
:1028F00018AA0ED0189A12A40BD0000109A008D073
:10290000D9EC2FF01FEC2DF0069A0990188C0B844F
:1029100018ACF3D012A414AAEBD004B408B6E8D0D3
:1029200013BAE6D014BC8AD006BA43D00101BE6BFC
:10293000C70E0101BE25D96EDA6A050EDA22CD0E68
:10294000BE25186F196B000E1923E7EC19F0DF6E26
:10295000C70E0101BE25D96EDA6A050EDA22DF50F4
:1029600004E0BE2B0F0EBE65E3D70101BE6BF90E6E
:102970000101BE25D96EDA6A030EDA22C80EBE2521
:10298000186F196B000E1923E7EC19F0DF6EF90EC2
:102990000101BE25D96EDA6A030EDA22DF5004E0A7
:1029A000BE2B040EBE65E3D70EBA068A000109905D
:1029B00047D000010EAA44D00101BE6BC70E010131
:1029C000BE25D96EDA6A050EDA228A0EBE25186F88
:1029D000196B010E1923E7EC19F0DF6EC70E010128
:1029E000BE25D96EDA6A050EDA22DF5004E0BE2B6E
:1029F0000F0EBE65E3D70101BE6BF90E0101BE25C6
:102A0000D96EDA6A030EDA22850EBE25186F196BAD
:102A1000010E1923E7EC19F0DF6EF90E0101BE2556
:102A2000D96EDA6A030EDA22DF5004E0BE2B040E00
:102A3000BE65E3D7069A0001098002D00001149C0C
:102A4000C9ECF6F014A80AD0020E0101996F000E2D
:102A500053EC1CF00101BE6F149808D0010E010167
:102A6000996F000E53EC1CF00101BE6F0101BE0511
:102A700006E0BE51020A03E0BE51040A20E109B09B
:102A800008D0500E0101206FCA0E1F6FE6EC21F036
:102A900007D0500E0101206FCC0E1F6FE6EC21F025
:102AA0000EAA0BD009B003D00201768102D0020138
:102AB00076837651030A19E1766B0C8E16D0BE67C9
:102AC00014D00201766B0C9E09B008D0500E0101A3
:102AD000206FC40E1F6FE6EC21F007D0500E0101ED
:102AE000206FC80E1F6FE6EC21F00201786B189A78
:102AF0000BA402D00B9401D0189C12B413AE54D086
:102B00000001139EBBEC2CF00101BE6F0201995134
:102B100004E0996B9951DFECD0F00101BE6701D060
:102B2000148C04A217D009B008D0500E0101206FF8
:102B3000C20E1F6FE6EC21F007D0500E0101206F8E
:102B4000C60E1F6FE6EC21F000010492D9EC2FF0C5
:102B5000148C2AD00101BE5103E0BE51050A16E1D2
:102B600009B008D0500E0101206FC20E1F6FE6ECB5
:102B700021F007D0500E0101206FC60E1F6FE6EC4A
:102B800021F0D9EC2FF01FEC2DF00ED0BE51030A2E
:102B900004E1010EDFECD0F007D0BE51040A04E1DD
:102BA000010EDFECD0F0138E0DAE0BD012940D9E03
:102BB0000E90149A0201636B000118961FEC2DF021
:102BC000F1D00EA0EFD00E9012B4ECD0148A010117
:102BD000BE6BC70E0101BE25D96EDA6A050EDA2278
:102BE000CD0EBE25186F196B000E1923E7EC19F0F6
:102BF000DF6EC70E0101BE25D96EDA6A050EDA2234
:102C0000DF5004E0BE2B0F0EBE65E3D70101BE6BA3
:102C1000F90E0101BE25D96EDA6A030EDA22C80E5A
:102C2000BE25186F196B000E1923E7EC19F0DF6E43
:102C3000F90E0101BE25D96EDA6A030EDA22DF50E1
:102C400004E0BE2B040EBE65E3D70990069A00018E
:102C50000EAA02D00001068AC9ECF6F073C299F1FF
:102C6000000E53EC1CF00101BE6F1498BE0505E187
:102C700016BE02D00C8C01D00C860101BE51020A96
:102C800003E0BE51040A55E10E840EAA52D00101A0
:102C9000BE6BC70E0101BE25D96EDA6A050EDA22B7
:102CA0008A0EBE25186F196B010E1923E7EC19F077
:102CB000DF6EC70E0101BE25D96EDA6A050EDA2273
:102CC000DF5004E0BE2B0F0EBE65E3D70101BE6BE3
:102CD000F90E0101BE25D96EDA6A030EDA22850EDD
:102CE000BE25186F196B010E1923E7EC19F0DF6E82
:102CF000F90E0101BE25D96EDA6A030EDA22DF5021
:102D000004E0BE2B040EBE65E3D709800001069ADD
:102D1000C9ECF6F073C299F1000E53EC1CF00101FE
:102D2000BE6F1498BE51020A03E0BE51040A01E1CD
:102D30000E820101BE51050A01E108880101BE05AC
:102D400006E0BE51020A03E0BE51040A13E109B0D5
:102D500008D0500E0101206FCA0E1F6FE6EC21F063
:102D600007D0500E0101206FCC0E1F6FE6EC21F052
:102D70000C8E14D0BE6712D00C9E09B008D0500E35
:102D80000101206FC40E1F6FE6EC21F007D0500E3A
:102D90000101206FC80E1F6FE6EC21F0189C0201A4
:102DA000786B189A10BE23D00EA802D00E981988FE
:102DB00046840101B6511AE08DECF3F00101BE6BBF
:102DC00011D0BE51020D000EF324D96EDA6A050E41
:102DD000DA220101DECF48F1DDCF49F18EECE3F0DC
:102DE00004E3BE2BB651BE5DECE3B66B469410BE59
:102DF000F5D004A4F2D002013951381101E0EDD030
:102E0000010EC0EC22F015C1D9FF16C1DAFFDF5068
:102E1000BD6F020EC0EC22F015C1D9FF16C1DAFF5A
:102E2000DF50BD27030EC0EC22F015C1D9FF16C13B
:102E3000DAFFDF50BD27040EC0EC22F015C1D9FF28
:102E400016C1DAFFDF50BD27050EC0EC22F015C118
:102E5000D9FF16C1DAFFDF50BD27BD6711D00201CF
:102E60009C6B0DAC05D000010D9C1FEC2DF0FF00FC
:102E7000000119A8B2D0010EADEC26F01998ADD022
:102E800002019C2B050E9C6502D0010E9C6F9C518B
:102E9000C0EC22F015C1D9FF16C1DAFFDF50BD6FBB
:102EA000BD6701D09AD09CC218F1000EB4EC2BF093
:102EB00018C1B1F119C1B2F19CC2BAF1B1C19DF111
:102EC000B2C19EF10D0E9F6FD8909E339D339F2F00
:102ED000FBD79D51030B0201556F0101BA050DE1AE
:102EE000000112A40AD0000E0101B1115F6F800E23
:102EF000B211606F00EC80F006D0B1C15FF1B2C1D9
:102F000060F100EC80F0BE6F030E0201396FE80E35
:102F1000386F0101BE6706D0BAC118F1000E1EEC71
:102F200012F05BD0000112A404D0010E0101BA65B9
:102F300002D0C9ECF6F012A404D0010E0101BA656A
:102F40003AD00201756749D000010B8AB9ECBDF097
:102F50001EE2500E0101206FE20E1F6FE6EC21F021
:102F60000101BA51030A0EE11CA40CD002016C2B22
:102F700004806C510A0A06E16C6BBAC118F1000EAC
:102F80001EEC12F00101BA2902016B6F12D002018E
:102F90005F6B606BBAC118F1000E1EEC12F0BA51F3
:102FA000030A04E11CA402D002016C6B060E0201AC
:102FB000756F0B9A12D000010B8A3AECF7F005E21C
:102FC000020E02016B6F6D2BF4D702016D6BBAC15B
:102FD00018F1000E1EEC12F0ECD700F010BE32EF2C
:102FE0008FF0000103A403D0000E3EECFAF00001C4
:102FF00003A632EF8FF0010E3EECFAF032EF8FF0C5
:10300000E8CF50F145C515F150515BEC2BF002E2D1
:10301000D890120003013651740A03E03651540A65
:1030200041E13751720A03E03751520A16E1E75184
:10303000050AEEE10101536BC20E5325176F186BA1
:10304000500E1823000E196B84EC1FF00101532B56
:10305000250E5365F1D7A6EF9DF0050EE76101D06F
:10306000D7D723EEE7F0070EDF6401D0D1D717ECF6
:103070009EF0B1ECFCF01BC151F11CC152F1000EED
:10308000515D010E5259C4E252515111C1E051C17A
:1030900095F2186B550E176F95C219F184EC1FF05D
:1030A000A6EF9DF036516E0A03E036514E0A22E13A
:1030B000050EE76101D0ACD723EEE7F0060EDF6422
:1030C00001D0A6D717EC9EF0B1ECFCF01BC151F17A
:1030D0001CC152F1110E515D000E525999E251C1BD
:1030E000B8F1186B760E176FB8C119F184EC1FF0A8
:1030F000A6EF9DF03651690A04E03651490A01E015
:1031000084D03751690A03E03751490A47E10C0E70
:10311000E76101D07DD723EEE7F0140EDF6401D024
:1031200077D75CEC9EF016D0330E2FEC9EF0C20EDB
:103130005325E16EE26A050EE222DFCFE7FF850E3E
:103140005325176F186B010E0DEC9EF084EC1FF0E9
:103150000101532B0301E7510101535DE5E34EECFF
:103160009EF0850E532548EC9EF084EC1FF00E9ADD
:103170000501C75142E0050E01011C6FC70E1B6F10
:10318000FC0E1E6FE50E1D6F206B070E1F6FD5EC3A
:1031900011F01C511B1131E00E8A2FD00B0EE7618C
:1031A00001D036D723EEE7F0130EDF6401D030D71D
:1031B00060EC9EF016D0330E2FEC9EF0C30E53251C
:1031C000E16EE26A050EE222DFCFE7FFC90E53256A
:1031D000176F186B000E0DEC9EF084EC1FF00101D0
:1031E000532B0301E7510101535DE5E34EEC9EF0E3
:1031F000C90E28EC9EF084EC1FF0069A099000019D
:1032000012B4A4EC2EF0A6EF9DF03651610A04E052
:103210003651410A01E09DD03751610A03E0375130
:10322000410A3BE1060EE76101D0F2D623EEE7F05A
:103230001F0EDF6401D0ECD65CEC9EF019D016AE08
:103240000BD0330E2FEC9EF09F0E5325E16EE26AF9
:10325000060EE222DFCFE7FF1B0E01015325176F99
:10326000186B030E0DEC9EF084EC1FF00101532B44
:103270000301E7510101535DE2E316AE07D09F0E53
:103280005325D96EDA6A060EDA22DF6A1B0E0101B7
:1032900041EC9EF084EC1FF03AD0050EE76101D0BE
:1032A000B7D623EEE7F01E0EDF6401D0B1D660EC96
:1032B0009EF019D016BE0BD0330E2FEC9EF0A00E50
:1032C0005325E16EE26A060EE222DFCFE7FF940E9D
:1032D00001015325176F186B000E0DEC9EF084EC66
:1032E0001FF00101532B0301E7510101535DE2E39C
:1032F00016BE07D0A00E5325D96EDA6A060EDA2262
:10330000DF6A940E010128EC9EF084EC1FF012B4E9
:1033100076D7F30E0101176F500E166F010E28ECD1
:103320001DF0060E0101176FA40E166F000E28EC9B
:103330001DF0220EA7EC2DF00D0EA7EC2DF0130EB4
:1033400001012A6F880E296FBAEC21F01CEC05F000
:1033500056D73651700A03E03651500A63E13751AF
:10336000700A03E03751500A28E1060EE76101D0E8
:103370004FD623EEE7F0090EDF6401D049D65CECAE
:103380009EF00FD0800E5325176F186B010E182377
:10339000330E2FEC9EF0DF50196F84EC1FF001010B
:1033A000532B0301E7510101535DECE3800E5325DC
:1033B00048EC9EF084EC1FF020D7050EE76101D0A9
:1033C00027D623EEE7F0080EDF6401D021D660ECAB
:1033D0009EF016D0330E2FEC9EF0F50E5325E16EC5
:1033E000E26A030EE222DFCFE7FFC40E5325176F18
:1033F000186B000E0DEC9EF084EC1FF00101532BB6
:103400000301E7510101535DE5E3F50E5325D96E44
:10341000DA6A030EDA22DF6AC40E28EC9EF084EC2E
:103420001FF0EBD63651640A03E03651440A44E1FA
:103430003751690A03E03751490A3EE123EEE7F0CC
:10344000140EDF6401D0E4D5E751050A0CE1010E4A
:103450000101186F750E176F000E196B84EC1FF0C9
:103460000501B76BCCD65CEC9EF014D0330EF7DBC5
:10347000B20E5325E16EE26A050EE222DFCFE7FFCE
:10348000700E5325176F186B010EC7DB84EC1FF00D
:103490000101532B0301E7510101535DE7E3B20E34
:1034A0005325D96EDA6A050EDA22DF6A700E5325CB
:1034B000EFDB84EC1FF0A3D63651640A03E03651EB
:1034C000440A38E13751640A03E03751440A32E1D3
:1034D00023EEE7F0250EDF6401D09AD5060EE761F2
:1034E00001D096D5E9DB14D0330EB9DB7F0E53251E
:1034F000E16EE26A060EE222DFCFE7FF500E5325AF
:10350000176F186B010E89DB84EC1FF00101532B40
:103510000301E7510101535DE7E37F0E5325D96EA7
:10352000DA6A060EDA22DF6A500E5325B1DB84EC2C
:103530001FF065D63651770A03E03651570A43E14A
:1035400023EEE7F0130EDF6401D062D5050EE761CC
:1035500001D05ED5B5DB0AD089DB500F01E258D52A
:1035600085DB460F01E354D50101532B0301E751DD
:103570000101535DF1E3040E536F14D0330E6FDB82
:10358000DB0E5325E16EE26A060EE222DFCFE7FF93
:10359000AF0E5325176F186B000E3FDB84EC1FF046
:1035A0000101532B0301E7510101535DE7E3DB0EFA
:1035B0005325D96EDA6A060EDA22DF6AAF0E48DBCF
:1035C00084EC1FF01CD63651720A03E03651520AC1
:1035D00025E1050EE76101D01BD523EEE7F0070ECC
:1035E000DF6401D015D523DBB1ECFCF01BC151F138
:1035F0001CC152F1000E515D010E525901E308D574
:103600005251511101E104D551C179F2186B730E79
:10361000176F79C219F184EC1FF098D236516F0AF6
:1036200003E036514F0A25E1050EE76101D0F0D4E1
:1036300023EEE7F0070EDF6401D0EAD4F8DAB1EC4C
:10364000FCF01BC151F11CC152F1000E515D010E85
:10365000525901E3DDD45251511101E1D9D451C184
:103660007DF2186B700E176F7DC219F184EC1FF09C
:103670006DD236516D0A03E036514D0A25E1050E33
:10368000E76101D0C5D423EEE7F0070EDF6401D077
:10369000BFD4CDDAB1ECFCF01BC151F11CC152F129
:1036A000000E515D010E525901E3B2D45251511135
:1036B00001E1AED451C1F4F0186B720E176FF4C073
:1036C00019F184EC1FF042D23651660A03E03651FC
:1036D000460A38E1E751050A01E09AD40101196B65
:1036E000750E186FE7EC19F0536F03013751300A6C
:1036F00006E1179E1890F90E010153171AD03751A1
:10370000310A06E1178E189001015383539511D0A9
:103710003751320A06E1179E1880010153855393F1
:1037200008D03751330A05E1178E1880060E0101C3
:1037300053130101186B750E176F53C119F184EC07
:103740001FF004D23651650A03E03651450A24E1E0
:10375000E751050A01E05CD40101196B4F0E186FA7
:10376000E7EC19F0536F03013751300A04E11C9460
:103770000101539908D03751310A05E11C84010138
:10378000538970ECCFF00101186B4F0E176F53C1C6
:1037900019F184EC1FF0DAD13651730A03E0365187
:1037A000530A11E1E751050A01E032D43751300ADA
:1037B00003E100010986CAD13751310A01E028D45A
:1037C00000010996C3D13651630A04E03651430A19
:1037D00001E0CFD0E751050A26E13751310A03E174
:1037E0000001098EB3D13751320A03E100010A808A
:1037F000ADD13751330A03E10001098AA7D137510E
:10380000340A03E100010988A1D13751350A03E1E7
:103810000001098C9BD13751360A02E008EF98F07D
:1038200000010A8293D1E7510A0A3FE1F30E010138
:10383000176F730E166F010E28EC1DF00301375140
:10384000A7EC2DF003013851A7EC2DF03A0EA7ECB0
:103850002DF003013951A7EC2DF003013A51A7ECEB
:103860002DF03A0EA7EC2DF003013B51A7EC2DF003
:1038700003013C51A7EC2DF019DA28EC1DF0130ED2
:1038800001012A6F880E296FBAEC21F002E30001D2
:10389000158EEAEC2FF0D2EC2FF0E90E0101295D34
:1038A000030E2A5901E352D1F6D7E751100A01E07D
:1038B0004DD1FC0E0101176FDD0E166F010E28ECC5
:1038C0001DF003013B51A7EC2DF003013C51A7EC87
:1038D0002DF02F0EA7EC2DF003013951A7EC2DF0A0
:1038E00003013A51A7EC2DF02F0EA7EC2DF00301A8
:1038F0003751A7EC2DF003013851A7EC2DF02C0E19
:10390000A7EC2DF003013D51A7EC2DF003013E5132
:10391000A7EC2DF03A0EA7EC2DF003013F51A7ECD8
:103920002DF003014051A7EC2DF03A0EA7EC2DF03D
:1039300003014151A7EC2DF003014251A7EC2DF0FA
:10394000B5D928EC1DF0130E01012A6F880E296FDE
:10395000BAEC21F002E30001158EEAEC2FF0D2EC74
:103960002FF0E90E0101295D030E2A5901E3EED083
:10397000F6D73651790A05E03651590A02E008EFC8
:1039800098F03751790A03E03751590A6EE1060E73
:10399000E76102D008EF98F023EEE7F00E0EDF6447
:1039A00002D008EF98F03851310A2DE18DD917D0A7
:1039B00016AE0AD0330E53D9D10E5325E16EE26A0A
:1039C000050EE222DFCFE7FF350E01015325176F09
:1039D000186B030E22D984EC1FF00101532B030155
:1039E000E7510101535DE4E316AE07D0D10E532534
:1039F000D96EDA6A050EDA22DF6A350E010141D985
:103A000084EC1FF09FD03851320A02E008EF98F0A2
:103A10005BD917D016AE0AD0330E21D9DA0E532552
:103A2000E16EE26A050EE222DFCFE7FF3E0E010102
:103A30005325176F186B030EF0D884EC1FF00101AB
:103A4000532B0301E7510101535DE4E316AE07D0A8
:103A5000DA0E5325D96EDA6A050EDA22DF6A3E0ED7
:103A600001010FD984EC1FF06DD0050EE76102D083
:103A700008EF98F023EEE7F00D0EDF6402D008EFB8
:103A800098F03751310A2DE117D917D016BE0AD058
:103A9000330EE5D8D20E5325E16EE26A050EE2221E
:103AA000DFCFE7FFE80E01015325176F186B000EFB
:103AB000B4D884EC1FF00101532B0301E75101013D
:103AC000535DE4E316BE07D0D20E5325D96EDA6AF1
:103AD000050EDA22DF6AE80E0101BAD884EC1FF085
:103AE00031D03751320A02E008EF98F0E5D817D00C
:103AF00016BE0AD0330EB3D8DB0E5325E16EE26A50
:103B0000050EE222DFCFE7FFF10E01015325176F0B
:103B1000186B000E82D884EC1FF00101532B0301B7
:103B2000E7510101535DE4E316BE07D0DB0E5325D8
:103B3000D96EDA6A050EDA22DF6AF10E010188D841
:103B400084EC1FF0000112A41CEC05F08DECF3F0E6
:103B500001015039F00B536F09AE07D0099E8A0E50
:103B60002F6F535112ECE5F038D00AA008D00A901C
:103B70008B0E01012F6F535112ECE5F02ED009AAE4
:103B800008D0099A8C0E01012F6F535112ECE5F009
:103B900024D009A808D009988D0E01012F6F535128
:103BA00012ECE5F01AD009AC08D0099C8E0E010188
:103BB0002F6F535112ECE5F010D00AA208D00A92F0
:103BC0008F0E01012F6F535112ECE5F006D0830EDA
:103BD00001012F6F535112ECE5F02FC151F130C1AB
:103BE00052F117A604D000011796D88012000501E3
:103BF00045516BEC2FF0F9E35051B6EC2AF0536FBE
:103C000051C139F152C13AF150C13BF153C13CF1BC
:103C1000030E3D6FC5EC1DF0E8D71823330E532576
:103C2000D96EDA6A030EDA22DF50196F1200330EF2
:103C3000E725D96EDA6A030EDA22DF6A370E010150
:103C40004E6F030E4F6F4EC11BF14FC11CF112009E
:103C50005325176F186B000E1823196B000C010108
:103C60005325D96EDA6A030EDA221200330E0101EF
:103C70005325D96EDA6A0301030EDA22DF50800A77
:103C800012005325176F186B030E1823196B000CC5
:103C9000176F186B010E1823196B000CC30E5325F8
:103CA000D96EDA6A050EDA22DF6A1200FE0E010111
:103CB000176F700E166F000C050E0101536F050C87
:103CC000040E0101536F040C060E0101536F060C24
:103CD0002D671BD003010A6B0B6B0C6B0D6B0298ED
:103CE000029A04D0A6ECDAF002B80FD003010D510D
:103CF000800A800F08E1000E0C5D05E1EA0E0B5D05
:103D000002E1610E0A5DEEE30C0C03010A6B0B6B22
:103D10000C6B0D6B02AA029808D0A6ECDAF002A890
:103D200004D002980001F06717D001012C51800ADD
:103D30002E6F03010A510101295D03010B5101019D
:103D40002A5903010C5101012B5903010D51800A1D
:103D500001012E59D9E3E1D7029A01012F6B320EEE
:103D600001012F25D96EDA6A060EDA22850E2F257B
:103D7000E16EE26A050EE222DFCFE7FF850E2F2516
:103D8000D96EDA6A050EDA22DF5004E02F2B310EED
:103D90002F65E5D7050E01011C6F850E1B6FF90E0F
:103DA0001E6FB80E1D6F206B0A0E1F6FD5EC11F041
:103DB0001C511B1106E1000102A8020C0001028A3D
:103DC000020C050E01011C6F850E1B6FF70E1E6F96
:103DD0009F0E1D6F206B0C0E1F6FD5EC11F01C5148
:103DE0001B1106E1000102A82F0C0001028A2F0C12
:103DF000050E01011C6F850E1B6FFD0E1E6F150E4B
:103E00001D6F206B070E1F6FD5EC11F01C511B119D
:103E1000D2E0050E01011C6F850E1B6FF30E1E6FA5
:103E2000840E1D6F206B100E1F6FD5EC11F01C510E
:103E30001B1106E1000102A8060C0001028A060C13
:103E4000050E01011C6F850E1B6FFB0E1E6FE60E2B
:103E50001D6F206B080E1F6FD5EC11F01C511B114C
:103E600006E1000102A8240C0001028A240C050EC0
:103E700001011C6F850E1B6FFD0E1E6F720E1D6FF4
:103E8000206B020E1F6FD5EC11F01C511B1106E1C7
:103E9000000102A8080C0001028A080C050E0101AD
:103EA000236F850E226F060E256FEF0E246F41ECF7
:103EB00011F02351221106E0000102A8030C0001B9
:103EC000028A030C050E01011C6F850E1B6FFD0E8F
:103ED0001E6F0B0E1D6F206B010E1F6FD5EC11F0C6
:103EE0001C511B1106E1000102A80D0C0001028A01
:103EF0000D0C050E01011C6F850E1B6FFB0E1E6F56
:103F0000DB0E1D6F206B010E1F6FD5EC11F01C51E5
:103F10001B1106E1000102A8100C0001028A100C1E
:103F2000050E01011C6F850E1B6FF80E1E6FC50E6E
:103F30001D6F206B010E1F6FD5EC11F01C511B1172
:103F400006E1000102A8110C0001028A110C050E05
:103F500001011C6F850E1B6FF30E1E6F930E1D6FFC
:103F6000206B010E1F6FD5EC11F01C511B1106E1E7
:103F7000000102A80F0C0001028A0F0C050E0101BE
:103F80001C6F850E1B6FFE0E1E6FA00E1D6F206B2B
:103F9000050E1F6FD5EC11F01C511B1106E100013D
:103FA00002A83A0C0001028A3A0C050E01011C6FAE
:103FB000850E1B6FFF0E1E6F3C0E1D6F206B040ED7
:103FC0001F6FD5EC11F01C511B1106E1000102A876
:103FD0003B0C0001028A3B0C050E01011C6F850E93
:103FE0001B6FFD0E1E6FD00E1D6F206B060E1F6F18
:103FF000D5EC11F01C511B1101E1DDD6050E0101BC
:104000001C6F850E1B6FFD0E1E6FC90E1D6F206B82
:10401000060E1F6FD5EC11F01C511B1106E10001BB
:1040200002A8390C0001028A390C050E01011C6F2F
:10403000850E1B6FF40E1E6F560E1D6F206B0E0E3D
:104040001F6FD5EC11F01C511B1106E1000102A8F5
:10405000090C0001028A090C050E01011C6F850E76
:104060001B6FF70E1E6F400E1D6F206B0D0E1F6F26
:10407000D5EC11F01C511B1106E1000102A82C0C1B
:104080000001028A2C0C050E01011C6F850E1B6FAE
:10409000FA0E1E6FC00E1D6F206B090E1F6FD5EC40
:1040A00011F01C511B11D2E0050E01011C6F850E91
:1040B0001B6FFA0E1E6FC40E1D6F206B050E1F6F57
:1040C000D5EC11F01C511B11C1E0050E01011C6F54
:1040D000850E1B6FFA0E1E6FCA0E1D6F206B090E28
:1040E0001F6FD5EC11F01C511B1106E1000102A855
:1040F000320C0001028A320C050E01011C6F850E84
:104100001B6FF90E1E6F760E1D6F206B0A0E1F6F50
:10411000D5EC11F01C511B1106E1000102A81C0C8A
:104120000001028A1C0C050E01011C6F850E1B6F1D
:10413000F90E1E6F810E1D6F206B0A0E1F6FD5ECDE
:1041400011F01C511B1106E1000102A81D0C000119
:10415000028A1D0C050E01011C6F850E1B6FF90EE6
:104160001E6F8C0E1D6F206B0A0E1F6FD5EC11F0A9
:104170001C511B1106E1000102A81E0C0001028A5D
:104180001E0C050E01011C6F850E1B6FF90E1E6FB4
:10419000970E1D6F206B0A0E1F6FD5EC11F01C518E
:1041A0001B1106E1000102A81F0C0001028A1F0C6E
:1041B000050E01011C6F850E1B6FF90E1E6FA20EFE
:1041C0001D6F206B0A0E1F6FD5EC11F01C511B11D7
:1041D00006E1000102A8200C0001028A200C050E55
:1041E00001011C6F850E1B6FF90E1E6FAD0E1D6F4A
:1041F000206B0A0E1F6FD5EC11F01C511B1106E14C
:10420000000102A8210C0001028A210C050E010107
:104210001C6F850E1B6FFF0E1E6FFC0E1D6F206B3B
:10422000010E1F6FD5EC11F01C511B1106E10001AE
:1042300002A8250C0001028A250C050E01011C6F45
:10424000850E1B6FFD0E1E6F6D0E1D6F206B070E12
:104250001F6FD5EC11F01C511B1106E1000102A8E3
:10426000260C0001028A260C050E01011C6F850E2A
:104270001B6FFE0E1E6F9A0E1D6F206B050E1F6FBB
:10428000D5EC11F01C511B1106E1000102A82B0C0A
:104290000001028A2B0C050E01011C6F850E1B6F9D
:1042A000FB0E1E6FD40E1D6F206B080E1F6FD5EC1A
:1042B00011F01C511B1106E1000102A8040C0001C1
:1042C000028A040C050E01011C6F850E1B6FFB0E8C
:1042D0001E6FCB0E1D6F206B080E1F6FD5EC11F0FB
:1042E0001C511B1106E1000102A80B0C0001028AFF
:1042F0000B0C050E01011C6F850E1B6FFB0E1E6F54
:10430000DD0E1D6F206B080E1F6FD5EC11F01C51D8
:104310001B1106E1000102A80A0C0001028A0A0C26
:10432000050E01013CDAD5EC11F01C511B1106E120
:10433000000102A8150C0001028A150C050E0101EE
:104340001C6F850E1B6FFE0E1E6F8E0E1D6F206B79
:10435000050E1F6FD5EC11F01C511B1106E1000179
:1043600002A8230C0001028A230C050E01011C6F18
:10437000850E1B6FFD0E1E6FC20E1D6F206B060E8D
:104380001F6FD5EC11F01C511B1106E1000102A8B2
:10439000130C0001028A130C050E01011C6F850E1F
:1043A0001B6FFD0E1E6F050E1D6F206B070E1F6F1E
:1043B000D5EC11F01C511B1106E1000102A8140CF0
:1043C0000001028A140C050E0101E9D9D5EC11F0A7
:1043D0001C511B11ADE0050E01011C6F850E1B6FFA
:1043E000FA0E1E6F840E1D6F206B090E1F6FD5EC29
:1043F00011F01C511B1106E1000102A8180C00016C
:10440000028A180C050E01011C6F850E1B6FFA0E37
:104410001E6F8E0E1D6F206B090E1F6FD5EC11F0F5
:104420001C511B1106E1000102A8160C0001028AB2
:10443000160C050E01011C6F850E1B6FFA0E1E6F08
:10444000980E1D6F206B090E1F6FD5EC11F01C51DB
:104450001B1106E1000102A8190C0001028A190CC7
:10446000050E01011C6F850E1B6FFA0E1E6FA20E4A
:104470001D6F206B090E1F6FD5EC11F01C511B1125
:1044800006E1000102A81A0C0001028A1A0C050EAE
:1044900001011C6F850E1B6FFA0E1E6FAC0E1D6F97
:1044A000206B090E1F6FD5EC11F01C511B1106E19A
:1044B000000102A81B0C0001028A1B0C050E010161
:1044C0001C6F850E1B6FFA0E1E6FB60E1D6F206BD4
:1044D000090E1F6FD5EC11F01C511B1106E10001F4
:1044E00002A8170C0001028A170C050E01011C6FAF
:1044F000850E1B6FFE0E1E6F940E1D6F206B050E3A
:104500001F6FD5EC11F01C511B1106E1000102A830
:10451000270C0001028A270C050E01011C6F850E75
:104520001B6FF80E1E6FD30E1D6F206B0B0E1F6FCF
:10453000D5EC11F01C511B1106E1000102A8280C5A
:104540000001028A280C050E01011C6F850E1B6FED
:10455000F30E1E6FC70E1D6F206B0F0E1F6FD5EC75
:1045600011F01C511B1106E1000102A8350C0001DD
:10457000028A350C050E01011C6F850E1B6FF70EAC
:104580001E6F4E0E1D6F206B0D0E1F6FD5EC11F0C0
:104590001C511B1106E1000102A8290C0001028A2E
:1045A000290C050E01011C6F850E1B6FF30E1E6F8B
:1045B000B70E1D6F206B0F0E1F6FD5EC11F01C5145
:1045C0001B1106E1000102A8360C0001028A360C1C
:1045D000050E01011C6F850E1B6FF80E1E6FC70EB6
:1045E0001D6F206B0B0E1F6FD5EC11F01C511B11B2
:1045F00006E1000102A82D0C0001028A2D0C050E17
:1046000001011C6F850E1B6FF80E1E6FBB0E1D6F18
:10461000206B0B0E1F6FD5EC11F01C511B1106E126
:10462000000102A82E0C0001028A2E0C050E0101C9
:104630001C6F850E1B6FF70E1E6F850E1D6F206B96
:104640000C0E1F6FD5EC11F01C511B1106E100017F
:1046500002A8300C0001028A300C050E01011C6F0B
:10466000850E1B6FF70E1E6F920E1D6F206B0C0ECA
:104670001F6FD5EC11F01C511B1106E1000102A8BF
:104680003C0C0001028A3C0C050E01011C6F850EDA
:104690001B6FF70E1E6F320E1D6F206B0D0E1F6FFE
:1046A000D5EC11F01C511B1106E1000102A8310CE0
:1046B0000001028A310C050E01011C6F850E1B6F73
:1046C000F90E1E6F6B0E1D6F206B0A0E1F6FD5EC5F
:1046D00011F01C511B1106E1000102A83D0C000164
:1046E000028A3D0C050E01011C6F850E1B6FFA0E30
:1046F0001E6F700E1D6F206B090E1F6FD5EC11F031
:104700001C511B1106E1000102A8330C0001028AB2
:10471000330C050E01011C6F850E1B6FFA0E1E6F08
:104720007A0E1D6F206B090E1F6FD5EC11F01C5116
:104730001B1106E1000102A8340C0001028A340CAE
:10474000050E01011C6F850E1B6FFD0E1E6FB40E52
:104750001D6F206B060E1F6FD5EC11F01C511B1145
:1047600006E1000102A8370C0001028A370C050E91
:1047700001011C6F850E1B6FFD0E1E6F0D0E1D6F50
:10478000206B070E1F6FD5EC11F01C511B1106E1B9
:10479000000102A8380C0001028A380C000C1C6FC2
:1047A000850E1B6FFD0E1E6FBB0E1D6F206B060E60
:1047B0001F6F060C04009E90D10ECF6E200ECE26E9
:1047C00002012C4B2D2B364B372B03010A2B000EED
:1047D0000B230C230D230201304B312B11AC09D0DC
:1047E000119C020E1F6E9D0E1E6E93EC0EF08C8EB1
:1047F000128202013F513E1108E03E07D8A03F0758
:104800003F513E1102E10001F66B020139513811AE
:1048100003E03807D8A03907244B252B0201255186
:10482000800A266E2251245D2351800A265801E316
:104830001B8602011C07D8A01D071D511C1102E197
:1048400010A0109412AA0AD00201812B040E8165D7
:1048500005D0816B0001128CF1EC26F002016B6730
:104860000AD00BAA07B807D014B410BE04D011B0F8
:1048700002D08D8A8D9C02016B5117E0905102E0AD
:1048800090073CD00BB806D08D9A8D9C02019069A0
:104890000B8834D08D9A8D8C020190690B986B0730
:1048A0006B672CD08D8A8D9C29D011A011D002016C
:1048B000912B270E916522D0916B8D8C8D8A722B56
:1048C0007251050A1BE18D9C8D9A726B119016D066
:1048D0000BAA07D00201912B310E916502D0916B8A
:1048E0000CD007A80BD003011E4B1F2BE80E1E5D3A
:1048F000030E1F5903E31E6B1F6B8D7A12A008D0A5
:1049000002017B2B310E7B6503D07B6B12908F9065
:104910000BAC0ED00201852B310E856509D0856B5D
:104920008F70842B3B0E846503D0846B0B9C8F901F
:104930000BAE10D00201892B310E89650BD0896B2B
:104940008C7E872B3B0E876505D0876B8C9E0B9EDC
:1049500018B40B8E12A208D002017C2B310E7C659C
:1049600003D07C6B12928C9E02018E2B1D0E8E65E5
:1049700003D08E6B8D6B8C6B46B4DCD10201862B21
:10498000180E8665D7D1866B0101BB6B3CC221F046
:104990003DC222F05CEC09F00001FF6F12BA0AAAD6
:1049A00004D0FE51E00BFF1903D00001FF51FE19A6
:1049B0000101BB6F9BC21DF0BB51ACEC19F0276E1F
:1049C000275001E18DD013A68AD027A015D012AAB6
:1049D00005D00101BB5132EC13F00ED00101BBA197
:1049E00006D01E6A220E1D6E9FEC07F005D01E6ACF
:1049F000240E1D6E9FEC07F027A215D012AA05D039
:104A00000101BB517BEC0FF00ED00101BBA306D01E
:104A10001E6A260E1D6E9FEC07F005D01E6A280E3A
:104A20001D6E9FEC07F027A415D012AA05D0010136
:104A3000BB51B6EC13F00ED00101BBA506D01E6A27
:104A40002A0E1D6E9FEC07F005D01E6A2C0E1D6EFF
:104A50009FEC07F027A615D012AA05D00101BB5183
:104A60003AEC14F00ED00101BBA706D01E6A2E0E40
:104A70001D6E9FEC07F005D01E6A300E1D6E9FEC78
:104A800007F027A815D012AA05D00101BB51F8ECF8
:104A900013F00ED00101BBA906D01E6A360E1D6EA2
:104AA0009FEC07F005D01E6A380E1D6E9FEC07F0D4
:104AB00027AA15D012AA05D00101BB5100EC2FF096
:104AC0000ED00101BBAB06D01E6A900E1D6E9FEC8E
:104AD00007F005D01E6A920E1D6E9FEC07F013863C
:104AE000BBC19BF2BBC1BCF113A807D00001139856
:104AF0001E6A400E1D6E9FEC07F007AA07D000014A
:104B0000079A1E6A320E1D6E9FEC07F007AC07D0A5
:104B10000001079C1E6A340E1D6E9FEC07F019A25F
:104B200007D0000119921E6A440E1D6E9FEC07F01B
:104B300010AC07D00001109C1E6A3E0E1D6E9FEC4B
:104B400007F015A607D0000115961E6A460E1D6EC9
:104B50009FEC07F00CAC07D000010C9C1E6A880E7D
:104B60001D6E9FEC07F00CA608D000010C96020EFB
:104B70001E6EB40E1D6E9FEC07F00EA407D0000150
:104B80000E941E6A8E0E1D6E9FEC07F00EA208D0CA
:104B900000010E92020E1E6EB60E1D6E9FEC07F007
:104BA00008A807D0000108981E6A960E1D6E9FEC9B
:104BB00007F012AE07D00001129E1E6A3A0E1D6E5B
:104BC0009FEC07F013A007D0000113901E6A3C0E63
:104BD0001D6E9FEC07F016A007D0000116901E6A0C
:104BE0008A0E1D6E9FEC07F016A807D000011698DC
:104BF0001E6A8C0E1D6E9FEC07F016A408D00001F3
:104C00001694020E1E6EB80E1D6E9FEC07F016ACC9
:104C100008D00001169C020E1E6EBA0E1D6E9FEC8F
:104C200007F0020150510AE0DE0E50251D6E1E6A8B
:104C3000020E1E229FEC07F00201506B0AA407D05F
:104C400000010A941E6A200E1D6E9FEC07F00BA255
:104C500007D000010B921E6A860E1D6E9FEC07F0B6
:104C60000AAC07D000010A9C1E6A940E1D6E9FECD0
:104C700007F0020149671CD013B60CB219D006A286
:104C800003D006B645D046D006AE03D007B240D01A
:104C900041D00DA203D00DB63BD03CD00CA803D020
:104CA0000CBE36D037D008A003D008B431D032D0F3
:104CB00000F002014A673BD0000113A638D0000182
:104CC0000CB435D006A404D0000106B629D02AD0F1
:104CD00007A004D0000107B223D024D00DA404D033
:104CE00000010DB61DD01ED00CBA12AA04D00001CE
:104CF00006BC16D017D00CAA04D000010CBE10D0F0
:104D000011D0000108A213D0000108B409D00AD0C4
:104D10008A8C02D08A9CCCD7030E0201496FC8D777
:104D20008A8E02D08A9E03D0030E02014A6F00F0E1
:104D3000DAEC25F011B402D011A603D00201716B98
:104D400003D0010E0201716F0301124B132B10519E
:104D5000125D1151135934E3126B136B0201716729
:104D600008D016BE03D08A988A962AD08D968D9444
:104D700027D0710525E11BAA16D01B9A16BE08D0B4
:104D800016BA03D08A988A860AD08A888A9607D06B
:104D900016B203D08D968D8402D08D868D9403013A
:104DA000116B640E0CD01B8A16BE03D08A988A96AB
:104DB00002D08D968D941F0E0301116F400E106F5F
:104DC0000301164B172B1451165D1551175960E34B
:104DD000166B176B04B402D00201746B0201746786
:104DE00023D01BAC0CD01B9C16BE03D08D868D949B
:104DF00002D08A888A960301156B640E13D01B8C2F
:104E000016BE03D08D968D9402D08A988A9604B4EB
:104E100005D0010E0301156F900E04D0090E030199
:104E2000156FC40E146F34D0740512E11BAC2AD078
:104E30001B9C16BE03D08D868D9402D08A888A96DC
:104E400012B4ECD7D8D78A988A9612B4D4D7E6D7BA
:104E50007451020A0AE11BAC15D01B9C16BE02D08D
:104E60008D860CD08A888A86EBD77451030A10E1AC
:104E70001BAC08D01B9C16BE03D08D968D84E0D74A
:104E80008A98F1D71B8C16BEDED78D968D94DDD710
:104E900010AE04D08D968D948A988A9603011C4B8F
:104EA0001D2BE80E1C5D030E1D595EE31C6B1D6B74
:104EB0000201344B352B000110AEABEC12F00201B5
:104EC0007F0712AA05D0525103E0522F01D0188E4D
:104ED0000401FE51D8A4FE0702019A51D8A49A07F2
:104EE0007D517E2B7E5D02E37E6B138E0201632B70
:104EF0001D0E636502D0636B188618A808D0580E83
:104F00000201205D020E215902E2204B212B06A84E
:104F10000AD002011F511E1103E18A9C069803D09A
:104F20001E07D8A01F0719A609D00301215120117F
:104F300002E1199603D02007D8A0210712A80AD0B1
:104F400002013B513A1103E18A9E129803D03A07BD
:104F5000D8A03B0702014951D8A449074A51D8A417
:104F60004A077551D8A4750703011A4B1B2B600E15
:104F70001A5DEA0E1B59D8A012001A6B1B6B0201B6
:104F8000932B12AA07D04C5105E04C2F03D0089C5C
:104F900008BA8A9C0001F4510201832B835D02E36D
:104FA000836B188C02017951782B785D02E3786B62
:104FB000188A0201542B020E546501D0546B030170
:104FC000184B192B0A0E185D000E195911E3186BB6
:104FD000196B0201672B8F0E676502D0676B098220
:104FE00002019551942B945D03E3946B198217820F
:104FF0000201822B020E8265020C826B0001138279
:105000001200E8CF38F10101406B010E3F6F96DBD3
:10501000366F36390F0B57EC2EF0DF6E402B8EDBE0
:105020000F0B57EC2EF0DF6E402B3F2B020E3F652F
:10503000EED7390E4025D96EDA6A010EDA22DF6A20
:1050400038C140F1A451310A0CE170DBF50E246F38
:10505000550E236F010E266F390E256FEBECD8F03D
:1050600049D3A451910A0CE161DBF50E246F640E63
:10507000236F010E266F390E256FEBECD8F03AD373
:10508000A451320A0CE152DBF50E246FBE0E236FE1
:10509000010E266F390E256FEBECD8F02BD3A451FF
:1050A000920A0CE143DBF50E246FCD0E236F010E47
:1050B000266F390E256FEBECD8F01CD3A451330AC0
:1050C0000CE134DBF60E246F270E236F010E266FE2
:1050D000390E256FEBECD8F00DD3A451930A0CE1F7
:1050E00025DBF60E246F360E236F010E266F390E68
:1050F000256FEBECD8F0FED2A451340A0CE116DB9C
:10510000F60E246F540E236F010E266F390E256F95
:10511000EBECD8F0EFD2A451940A0CE107DBF60EC9
:10512000246F630E236F010E266F390E256FEBEC93
:10513000D8F0E0D2A451390A0CE1F8DAF60E246F67
:10514000810E236F010E266F390E256FEBECD8F020
:10515000D1D2A451990A0CE1E9DAF60E246F900E2F
:10516000236F010E266F390E256FEBECD8F0C2D2FB
:10517000A451890A0CE1DADAF60E246F9F0E236F30
:10518000010E266F390E256FEBECD8F0B3D2A45187
:10519000900A0CE1CBDAF60E246FAE0E236F010EEF
:1051A000266F390E256FEBECD8F0A4D2A451980AE3
:1051B0000CE1BCDAF50E246F0A0E236F010E266F88
:1051C000390E256FEBECD8F095D2A451350A0CE1DD
:1051D000ADDAF40E246FBF0E236F010E266F390E69
:1051E000256FEBECD8F086D2A451950A0CE19EDA3B
:1051F000F40E246FCE0E236F010E266F390E256F2D
:10520000EBECD8F077D2A451960A0CE18FDAF40EC9
:10521000246FDD0E236F010E266F390E256FEBEC28
:10522000D8F068D2A451380A0CE180DAF40E246F69
:10523000FB0E236F010E266F390E256FEBECD8F0B5
:1052400059D2A451710A0CE171DAF40E246FEC0EFC
:10525000236F010E266F390E256FEBECD8F04AD282
:10526000A451850A0CE162DAF50E246F910E236FCA
:10527000010E266F390E256FEBECD8F03BD2A4510E
:10528000880A0CE153DAF50E246FFA0E236F010E33
:10529000266F390E256FEBECD8F02CD2A451460ABC
:1052A0000CE144DAF60E246F450E236F010E266FD3
:1052B000390E256FEBECD8F01DD2A451450A0CE154
:1052C00035DAF60E246F720E236F010E266F390E3B
:1052D000256FEBECD8F00ED2A451030A05E126DAD3
:1052E0003BDAEBECD8F006D2A451050A05E11EDA50
:1052F00033DAEBECD8F0FED1A451040A0CE116DA53
:10530000F50E246F820E236F010E266F390E256F66
:10531000EBECD8F0EFD1A451060A05E107DA25DA63
:10532000EBECD8F0E7D1A451080A05E1FFD91DDA6A
:10533000EBECD8F0DFD1A451070A0CE1F7D9F50E58
:10534000246FEB0E236F010E266F390E256FEBECE9
:10535000D8F0D0D1A451360A0CE1E8D9F50E246F6B
:10536000370E236F010E266F390E256FEBECD8F048
:10537000C1D1A451370A0CE1D9D9F50E246F460EDC
:10538000236F010E266F390E256FEBECD8F0B2D1EA
:10539000A451390A0CE1CAD9F40E246F830E236F8D
:1053A000010E266F390E256FEBECD8F0A3D1A45176
:1053B000990A0CE1BBD9F40E246F920E236F010EF3
:1053C000266F390E256FEBECD8F094D1A46712D07C
:1053D000330E01014025216F226B030E2223F50EAF
:1053E000246F190E236F010E266F390E256FEBEC1B
:1053F000D8F080D1A451780A0CE198D9F50E246F29
:10540000280E236F010E266F390E256FEBECD8F0B6
:1054100071D1A451700A0CE189D9F40E246FB00E39
:10542000236F010E266F390E256FEBECD8F062D199
:10543000A451400A0CE17AD9F50E246FA00E236F17
:10544000010E266F390E256FEBECD8F053D1A45125
:10545000410A0CE16BD9F60E246F090E236F010E81
:10546000266F390E256FEBECD8F044D1A451420AD7
:105470000CE15CD9F50E246FAF0E236F010E266F81
:10548000390E256FEBECD8F035D1A451430A0CE16D
:105490004DD9F60E246F180E236F010E266F390EAC
:1054A000256FEBECD8F026D121EEA4F09F0EDF643F
:1054B0002DD0B00EA4612AD0A451610F3E6F0A0E08
:1054C0003E6115D0330E01014025216F226B030E82
:1054D0002223F30E246FF70E236F010E266F390E71
:1054E000256F3EC127F1286BEBECD8F003D11ED914
:1054F000F60E246FCC0E236F010E266F390E256F2A
:105500003EC127F1286BEBECD8F0F4D021EEA4F0EB
:10551000AF0EDF642DD0C00EA4612AD0A451510F6C
:105520003E6F0A0E3E6115D0330E01014025216FFA
:10553000226B030E2223F30E246FE70E236F010E5E
:10554000266F390E256F3EC127F1286BEBECD8F0A2
:10555000D1D0ECD8F60E246FBD0E236F010E266F4E
:10556000390E256F3EC127F1286BEBECD8F0C2D085
:1055700021EEA4F0CF0EDF642DD0E00EA4612AD07E
:10558000A451310F3E6F0A0E3E6115D0330E01015A
:105590004025216F226B030E2223F40E246F170E79
:1055A000236F010E266F390E256F3EC127F1286B40
:1055B000EBECD8F09FD0BAD8F60E246FEA0E236F2A
:1055C000010E266F390E256F3EC127F1286BEBECDB
:1055D000D8F090D021EEA4F0DF0EDF642DD0F00ED5
:1055E000A4612AD0A451210F3E6F0A0E3E6115D04E
:1055F000330E01014025216F226B030E2223F40E8E
:10560000246F070E236F010E266F390E256F3EC1E2
:1056100027F1286BEBECD8F06DD088D8F60E246F0C
:10562000DB0E236F010E266F390E256F3EC127F169
:10563000286BEBECD8F05ED021EEA4F0BF0EDF6457
:105640002DD0D00EA4612AD0A451410F3E6F0A0E76
:105650003E6115D0330E01014025216F226B030EF0
:105660002223F40E246F270E236F010E266F390EAE
:10567000256F3EC127F1286BEBECD8F03BD056D814
:10568000F60E246FF90E236F010E266F390E256F6B
:105690003EC127F1286BEBECD8F02CD0A451230AA3
:1056A0001EE0A451240A1BE0A451250A18E0A451CD
:1056B000260A15E0A451270A12E0A451280A0FE097
:1056C000A451300A0CE0A451150A09E0A451790A4A
:1056D00006E0A451840A03E0A451830A0DE126D810
:1056E000F40E246FA10E236F010E266F390E256F65
:1056F000EBECD8F021513F6F3F51382551ECE4F0ED
:10570000330E0101366F030E376F38513627000E06
:1057100037233F513627000E37230E0E3625D96E1C
:10572000000E3721DA6EDF6AB5EF0BF0330E0101A0
:105730004025216F226B030E22231200390E4025D3
:10574000D96EDA6A010EDA22A10E3F25E16EE26A15
:10575000010EE222E7501200F50E246F730E236F44
:10576000010E266F390E256F1200F50E246FDC0E28
:10577000236F010E266F390E256F1200E8CFFFF25E
:105780000201FF050FE1020E0101166FB80E156F41
:10579000F1EC29F00201FE6FFE6701D01200826B6E
:1057A000139228D0FE6B14D00201FE51800A400FE4
:1057B00021E2330EFE25D96EDA6A030EDA22B80E24
:1057C000FE25E16EE26A020EE222DFCFE7FFFE2B4A
:1057D000E7C392F10101936BFEC294F1956B94BF04
:1057E00095079551800A966F9251945D9351800A66
:1057F0009659DAE30201826B1392FF0561E1020E12
:1058000001011C6FB80E1B6FFE0E1E6FD60E1D6FB2
:10581000206B050E1F6FD5EC11F01C511B1112E10E
:10582000130E376F6A0E366F396B1E0E386FC9DA7A
:1058300093ECC3F001013751361104E10201FF512D
:1058400038EC2CF0020E01011C6FB80E1B6FFC0E21
:105850001E6F010E1D6F206B080E1F6FD5EC11F02F
:105860001C511B112DE1130E186F6A0E176F000EDD
:10587000196B84EC1FF0130E0101186F790E176F6E
:10588000000E196B84EC1FF00101196B750E186F77
:10589000E7EC19F00201F86FF851F70BF96F01010D
:1058A000186B750E176FF9C219F184EC1FF0F30E27
:1058B0000101166FD70E156F0F0E176F96EC2EF0B5
:1058C0000201FF0529E1020E01011C6FB80E1B6FDA
:1058D000FE0E1E6FD00E1D6F206B050E1F6FD5ECD8
:1058E00011F01C511B1118E1186BFF0E1769196993
:1058F00084EC1FF04F0E0101186FD60E176F000ECB
:10590000196B84EC1FF0F20E0101166F320E156F49
:10591000160E176F96EC2EF0020E01011C6FB80EDA
:105920001B6FFE0E1E6FC40E1D6F206B050E1F6FCA
:10593000D5EC11F01C511B1149E112AA02D006BC92
:10594000FED14F0E0101196FD30E186FE7EC19F05D
:10595000926F92AD2BD0020E0101226FB80E216F13
:10596000F70E246FB90E236F0D0E266F710E256F83
:10597000EBECD8F021510201FE6FFF5109E0020E5D
:105980000101166FB80E156FFEC217F196EF2EF0DB
:10599000020E01012C6FB80E2B6F0201FE510101A6
:1059A0002D6F2E6B2DBF2E07D1EFEBF0020E0101F4
:1059B000226FB80E216FF70E246FAC0E236F0D0E01
:1059C000266F710E256FEBECD8F0D4D7020E0101D3
:1059D0001C6FB80E1B6F60EC04F01BC1FCF21CC105
:1059E000FDF24F0E196FD50E186FE7EC19F0926F9C
:1059F0004F0E196FD40E186FE7EC19F00201FB6F10
:105A0000010192510201FA6FE4D9FE0E1E6FB80E29
:105A10001D6F206B050E1F6FD5EC11F01C511B1173
:105A20001BE10201FB51FD1902E1FA51FC1901E0F1
:105A300099D04F0E0101196FD30E186FE7EC19F0D2
:105A40000201FE6F3F0EFE17D7D984EC1FF0020152
:105A5000FF51E0EC2BF075D0ABD9FE0E1E6FBE0EE1
:105A60001D6F206B050E1F6FD5EC11F01C511B1123
:105A70001AE10201FB51FD1902E1FA51FC1901E0A2
:105A800071D04F0E0101196FD30E186FE7EC19F0AA
:105A90000201FE6FFE8DB0D984EC1FF00201FF51B0
:105AA000E0EC2BF04ED084D9FE0E1E6FCA0E1D6F97
:105AB000206B050E1F6FD5EC11F01C511B1141E13D
:105AC0000201FE51800A720F06E3FB51FD1902E14B
:105AD000FA51FC1901E046D00A0EFE6F84D9500F2E
:105AE00003E381D9460F01E33DD0FE2BFE51800A2E
:105AF000720FF4E3C66BC20E0101926F020E936F38
:105B000092C11BF193C11CF160EC04F01BC1FCF2CB
:105B10001CC1FDF24F0E186FD40E176F0201FD511C
:105B20000101196F84EC1FF04F0E0101186FD50EA3
:105B3000176FFCC219F184EC1FF00201FF51E0EF76
:105B40002BF04F0E0101196FD30E186FE7EC19F00F
:105B5000926F92AD0AD00201FB51FD1902E1FA5198
:105B6000FC1903E0FF5122EF2CF033D9FF0E1E6F1A
:105B70004B0E1D6F206B040E1F6FD5EC11F01C51E6
:105B80001B1141E146B604D0000111A86CECECF009
:105B90000101376B366B040E396F386B020E3B6FA9
:105BA000B80E3A6FFFC23CF193ECC3F001013751DC
:105BB000361104E10201FF5138EC2CF0000146B629
:105BC0001200010E0101186F000E176B196B84ECA7
:105BD0001FF0010E0101186F110E176F000E196BE7
:105BE00084EC1FF0010E0101186F220E176F000EDA
:105BF000196B84EC1FF0010E0101186F330E176F43
:105C0000196B84EF1FF0D4D8FF0E1E6F550E1D6F59
:105C1000206B040E1F6FD5EC11F01C511B110BE112
:105C2000040E376F366B0D0E396FE80E386FC9D81A
:105C300093ECC3F048D0BCD8FF0E1E6F5F0E1D6FF3
:105C4000206B040E1F6FD5EC11F01C511B110CE1E1
:105C5000130E376F880E366F2E0E396FB30E386FF6
:105C6000B0D893ECC3F02FD0A3D8FF0E1E6F410E17
:105C70001D6F206B040E1F6FD5EC11F01C511B1112
:105C80000CE1420E376F3B0E366F0B0E396FB80EBC
:105C9000386F97D893ECC3F016D08AD8FF0E1E6FDA
:105CA0005A0E1D6F206B040E1F6FD5EC11F01C51A6
:105CB0001B1112E1510E376F366B2F0E396F386B97
:105CC00080D893ECC3F0010137513611D8A41200EB
:105CD0000201FF5138EF2CF06BD8FE0E1E6FDC0E68
:105CE0001D6F206B050E1F6FD5EC11F01C511B11A1
:105CF0000DE112AA02D006BC22D0020E0101386FBB
:105D0000B80E376FFFC239F1DDEFB1F051D8FF0E99
:105D10001E6F500E1D6F206B040E1F6FD5EC11F01F
:105D20001C511B1110E112AA02D006BC08D00101BF
:105D30007D6B7C6B040E7F6F7E6B020E19D00201AF
:105D4000FF510CEF2CF034D8FF0E1E6F640E1D6F48
:105D5000206B040E1F6FD5EC11F01C511B110FE1CD
:105D6000130E7D6F880E7C6F2E0E7F6FB30E1CD0CE
:105D7000816FB80E806FFFC282F1AFEFC1F018D80B
:105D8000FF0E1E6F460E1D6F206B040E1F6FD5ECAD
:105D900011F01C511B11D8A41200420E7D6F3B0E56
:105DA0007C6F0B0E7F6FB80E7E6F020E0101E0D785
:105DB000BD0E926F020E936F92C11BF193C11CF145
:105DC0001200020E01013B6FB80E3A6FFFC23CF1A8
:105DD0001200BD0E0101926F020E936F92C11BF172
:105DE00093C11CF11200B80EFE25D96EDA6A020EBC
:105DF000DA22DF50800A12004F0E0101186FD30E15
:105E0000176FFEC219F1D30C0101266B280E010198
:105E10002625D96EDA6A050EDA222651186F196B1B
:105E200018BF1907E7EC19F0DF6E262B2651800A00
:105E3000610FECE3266B000E01012625D96EDA6AAC
:105E4000030EDA22800E6ADAE7EC19F0DF6E262BF9
:105E50002651800A7A0FEFE3196B550E186FE7ECA5
:105E600019F00201956F0101196B4B0E186FE7ECE9
:105E700019F0236F226B196B4A0E186FE7EC19F0BB
:105E8000221102013C6F0101235102013D6F01010A
:105E9000196B520E186FE7EC19F00001FE6F01014B
:105EA000196B560E186FE7EC19F00201596F0101DA
:105EB000196B570E186FE7EC19F002015B6F0101C7
:105EC000196B760E186FE7EC19F0B86F196B590E55
:105ED000186FE7EC19F0236F226B196B5A0E186FCD
:105EE000E7EC19F02211AF6F2351B06F196B4F0E11
:105EF000186FE7EC19F0266F1C90010126B51C8085
:105F00001C9226B71C821C9426B91C84196B750E32
:105F1000186FE7EC19F0266F1696010126B1168668
:105F2000179E26B3178E109626B71086189026B5A2
:105F300018800C920692069E0D920C9808900C9474
:105F4000069407900D940C9A0892196B4C0E186FDA
:105F5000E7EC19F0266F266702D00C8214D026B128
:105F6000FCD726A302D006820ED026A502D0068E2C
:105F70000AD026A702D00D8206D026A902D00C880E
:105F800002D026BB08800101196B4D0E186FE7EC9B
:105F900019F0266F266702D00C8414D026B1FCD7E6
:105FA00026A302D006840ED026A502D007800AD0F0
:105FB00026A702D00D8406D026A902D00C8A02D0D2
:105FC00026BB08820101196B6C0E186FE7EC19F003
:105FD0000001FA6F199EFAB7198E070EFA17010120
:105FE000196B680E186FE7EC19F00001FB6F1A9837
:105FF000FBB71A88070EFB170101196B690E186FA2
:10600000E7EC19F00001FC6F1A9EFCB71A8E070E20
:10601000FC170101196B6A0E186FE7EC19F000010B
:10602000FD6F1B94FDB71B84070EFD170101196B53
:10603000540E186FE7EC19F0266F2651F00B09E1AA
:10604000069C179826C122F10F0E01012217222962
:1060500025D02651F00B100A0FE1068C179826C1A7
:1060600022F10F0E0101221722290001EE6F020119
:106070002B6B010E2A6F14D02651F00B200A03E17E
:10608000069C1788DFD72651F00B300A03E1068CF7
:106090001788E5D7069C07941798010E02014F6FE9
:1060A00019AE1AB804D01ABE02D01BA402D0178AA7
:1060B00001D0179A0101196B640E186FE7EC19F003
:1060C0000201686F0101196B650E186FE7EC19F09A
:1060D0000201696F0101196B660E186FE7EC19F088
:1060E00002016F6F0101196B670E186FE7EC19F071
:1060F00002015C6F0101196B6B0E186FE7EC19F070
:10610000266F1090010126B110800A9A26B50A8ADE
:10611000089A12AA07D0088A0C920692069E0D923F
:106120000C9808900101196B700E186FE7EC19F0CC
:1061300002017D6F0101196B720E186FE7EC19F007
:106140000001F46F0101196B710E186FE7EC19F083
:106150000201736F0101196B730E186FE7EC19F0F0
:106160000201796F0101266BE2D88A0ECBD8E7ECE9
:1061700019F0DF6EDCD8DF5005E0262B2651800AAF
:10618000700FF2E30E9A0501C75112E0050E0101EE
:106190001C6FC70E1B6FFC0E1E6FE50E1D6F206B74
:1061A000070E1F6FD5EC11F01C511B1101E00E8A78
:1061B0000101266BBCD8CD0EB1D8E7EC19F0DF6E2B
:1061C000B6D8DF5005E0262B2651800A700FF2E387
:1061D0000101266BDF0EBDD8B30EA0D8E7EC19F095
:1061E000DF6EDF0EB6D8DF5005E0262B2651800A81
:1061F000700FF0E30101266BB3D8DD0E8FD8E7EC0A
:1062000019F0DF6EADD8DF5005E0262B2651800A4D
:10621000700FF2E30101256B980E246F16AE04D0C7
:10622000030E256F200E246F0101266BA8D887D896
:10623000E7EC19F0DF6EA3D8DA22DF5005E0262B59
:106240002651800A650FF2E30101256BED0E246FE4
:1062500016AE04D0030E256F3B0E246F0101266B92
:1062600095D86DD8E7EC19F0DF6E90D8DA22DF50C0
:1062700005E0262B2651800A770FF2E30101256BFA
:10628000F60E246F16AE04D0030E256F440E246F55
:106290000101266B6DD853D8E7EC19F0DF6E68D892
:1062A000DA22DF5005E0262B2651800A770FF2E331
:1062B0000101266B72D8550E25D8E7EC19F0DF6E78
:1062C0006CD8DF5005E0262B2651800A600FF2E3E0
:1062D0000101266B6AD8750E15D8E7EC19F0DF6E50
:1062E00064D8DF5005E0262B2651800A700FF2E3B8
:1062F000420E0101196F3A0E186FE7EC19F0020116
:10630000976F1200226F010E236F22512625186FFE
:10631000000E26BFFF0E2321196F12002625186FCD
:10632000E86AD8B0E82A26BFE806196F1200C70E3F
:1063300001012625D96EDA6A050EDA221200DA2268
:1063400024512625186F000E26BFFF0E2521196F38
:10635000120001012625D96EDA6A060EDA22120031
:10636000EF0E01012625D96EDA6A060EDA22120036
:10637000E00E01012625D96EDA6A050E1200A40E80
:1063800001012625D96EDA6A060E1200D70E010128
:106390002625D96EDA6A050E1200840E0101262523
:1063A000D96EDA6A060EDA221200B70E010126252E
:1063B000D96EDA6A050EDA221200049C049E0001EE
:1063C000F26B0201646B986B01017F6B806BD1EC07
:1063D000E5F010E30101390506E1FA0E166FDE0E55
:1063E000156F090E3FD0FA0E2C6FDE0E2B6F2E6B41
:1063F000090E3CD014A010D00101390506E1F20EBF
:10640000166F1B0E156F160E2DD0F20E2C6F1B0E75
:106410002B6F2E6B160E2AD00101836B846B856B5C
:10642000866B28D00201826B139283C116F184C15E
:1064300017F185C118F186C119F1FF0E01011A6922
:10644000E3EC2CF083C116F184C117F185C118F17A
:1064500086C119F14EEC2CF03A6F3A290AE0390561
:1064600004E1BBD7176F96EF2EF0BDD72D6FD1EF9C
:10647000EBF03CDA8651800A800F08E1020E855D60
:1064800005E1000E845D02E1000E835DCBE339057A
:1064900009E1F30E166F950E156F100E176F96EC3F
:1064A0002EF009D0F30E2C6F950E2B6F2E6B100E65
:1064B0002D6FD1ECEBF00D900BD00101390504E10B
:1064C000FA0E166FF20E8CD7FA0E2C6FF20E8ED7D4
:1064D00037C11DF138C11EF13C0E01011F6F39C1DA
:1064E00020F1E6EC1FF00101876F19B4E6D7875160
:1064F0003A0AEEE17F4B802B37C127F138C128F1F2
:106500000A0E296F39C12AF1B8EC27F0876F19B448
:10651000D4D787C181F181C156F237C127F138C183
:1065200028F10A0E0101296F39C12AF1B8EC27F0D0
:10653000876F19B4C2D7010187513B6F3A6B3C6B2F
:106540003B513D6F3CC183F13DC184F1856B866B4E
:1065500037C127F138C128F10A0E296F39C12AF154
:10656000B8EC27F0876F19B4A8D7010187518313BE
:1065700037C127F138C128F10A0E296F39C12AF134
:10658000B8EC27F07E6F19B498D704AE93D101010F
:10659000D890852B000E86238DD137C127F138C1C5
:1065A00028F10A0E296F39C12AF1B8EC27F0826F61
:1065B00019B483D701018651800A800F08E1010ECA
:1065C000855D05E1FC0E845D02E1000E835D27E23E
:1065D00083C116F184C117F185C118F186C119F183
:1065E00082C11AF1E3EC2CF083C116F184C117F1DA
:1065F00085C118F186C119F14EEC2CF082191EE00C
:10660000390506E1F70E166FC60E156F0C0E2AD768
:10661000F70E2C6FC60E2B6F2E6B0C0E27D739057D
:1066200006E1F40E166F650E156F0E0E1BD7F40EF5
:106630002C6F650E2B6F2E6B0E0E18D757D9810756
:1066400001018129AAE137C12DF138C12EF10A0ECD
:106650002F6F39C130F146EC20F001E3048C19B4FE
:106660002CD736D737C12DF138C12EF10A0E2F6F36
:1066700039C130F146EC20F001E3048C19B41DD788
:1066800004AC10D00101390506E1FB0E166FF80EBF
:10669000156F080EE7D6FB0E2C6FF80E2B6F2E6BC6
:1066A000080EE4D6000E0101166B176B186B196B00
:1066B0004EEC2CF0660A1EE1010E166F000E176BF1
:1066C000186B196B4EEC2CF0EF0A14E1020E166FEA
:1066D000000E176B186B196B4EEC2CF0FE0A0AE1DA
:1066E000030E166F000E176B186B196B4EEC2CF027
:1066F000F00A0AE0390504E1F90E166FC30E15D051
:10670000F90E2C6FC30E17D0600EEAD84EEC2CF0A9
:10671000220A06E1610EE4D84EEC2CF0280A0FE0C4
:10672000390506E1F90E166FCE0E156F0A0E9AD6D0
:10673000F90E2C6FCE0E2B6F2E6B0A0E97D6010E14
:10674000226F3E0E216FFD0E246FD70E236F7FC187
:1067500025F180C126F1EBECD8F02151876F390586
:106760001EE1010E166F3E0E156F87C117F196ECF4
:106770002EF0F10E0101166F690E156F1C0E176FCA
:1067800096EC2EF0270E0101806F100E7F6F7F07B1
:10679000D8A08007010180517F111CE0F8D7010EBD
:1067A0002C6F3E0E2B6F87C12DF12E6BD1ECEBF0D1
:1067B000F10E01012C6F690E2B6F2E6B1C0E2D6FCD
:1067C000D1ECEBF0F90E0101176F1B0E166F010EE5
:1067D00028EC1DF0FB0E0101166F1769010E186FF2
:1067E000196B460E1A6FE3EC2CF0FC0E166F17694E
:1067F000010E186F196B4C0E1A6FE3EC2CF0FD0EA6
:10680000166F1769010E186F196B410E1A6FE3ECC2
:106810002CF0FE0E166F1769010E186F196B530ED0
:106820001A6FE3EC2CF016691769010E186F196BDB
:10683000480E1A6FE3EC2CF0FF001200826B0DD0B3
:1068400037C127F138C128F10A0E296F39C12AF161
:10685000B8EC27F0821319B430D6010181078129E1
:10686000EFE18251F00B100A02E1048E01D0049E88
:106870002DD846EC20F0F1D637C127F138C128F1E8
:106880000A0E296F39C12AF1B8EC27F0826F19B4CA
:1068900014D6010181078129EFE182C13AF10F0E7F
:1068A0003A173A0502E1048E01D0049E0FD846EC57
:1068B00020F0D3D601017E5101E1C1D6010A01E1E8
:1068C000D1D6030ABBE0060AE4E002D637C12DF1B7
:1068D00038C12EF10A0E01012F6F39C130F10A0CB7
:1068E000166F040E176F186B196B000C832B000EBC
:1068F000842385238623000C20EE01F02651D9261F
:106900002751DA22DF50286F26C1D9FF27C1DAFFCD
:10691000DF502D6F28512C6F090E2C5D000E2D5964
:1069200019E3290E2C5D000E2D5914E220EE04F01F
:106930001ADA130EDF6E26C1D9FF27C1DAFFDF6A2C
:1069400004DAF80FDF6E26C11EF127C11FF153ECE8
:1069500008F0F9D1290E2C5D000E2D590AE3490EDD
:106960002C5D000E2D5905E217DA2BDAEED9D80F7F
:10697000E9D7560E2C5D000E2D5913E3760E2C5DD3
:10698000000E2D590EE220EE04F0EDD9380EDF6E28
:1069900026C1D9FF27C1DAFF300EDF6ED6D9AB0F83
:1069A000D1D7760E2C5D000E2D590CE3960E2C5D82
:1069B000000E2D5907E2F0D90FDA300EDF6EC5D97F
:1069C0008B0FC0D7990E2C5D000E2D590AE3BB0E1C
:1069D0002C5D000E2D5905E2DFD9D2D9B6D9680F4A
:1069E000B1D7C00E2C5D000E2D590CE3E20E2C5DCC
:1069F000000E2D5907E220EE04F0B5D9D9D9A5D95A
:106A0000410FA0D74C0E2C5D010E2D5913E36C0ED7
:106A10002C5D010E2D590EE220EE04F0A4D9380EA3
:106A2000DF6E26C1D9FF27C1DAFF400EDF6E8DD998
:106A3000B50F88D76C0E2C5D010E2D590BE38C0E13
:106A40002C5D010E2D5906E2A7D9C6D9DF6A7DD982
:106A5000950F78D78C0E2C5D010E2D5912E3AC0EDC
:106A60002C5D010E2D590DE220EE04F07CD9380E7C
:106A7000DF6E26C1D9FF27C1DAFFDF6A66D9750F3D
:106A800061D7910E2C5D030E2D591BE3A10E2C5DD9
:106A9000030E2D5916E220EE04F02651D926275177
:106AA000DA22070EDF6E20EE03F0265195D9400E54
:106AB000DF6E20EE01F02651D9262751DA22000E92
:106AC00041D7A10E2C5D030E2D590DE3B10E2C5DA7
:106AD000030E2D5908E220EE04F02651D926275145
:106AE000DA22060EDFD7000E2C5D040E2D5912E3BC
:106AF000200E2C5D040E2D590DE220EE04F033D94A
:106B0000130EDF6E26C1D9FF27C1DAFFDF6A1DD958
:106B1000210F18D7200E2C5D040E2D590BE3400ECB
:106B20002C5D040E2D5906E237D94BD90ED9286FAA
:106B3000282908D7400E2C5D040E2D5913E3600E52
:106B40002C5D040E2D590EE220EE04F00CD9380E07
:106B5000DF6E26C1D9FF27C1DAFF300EDF6EF5D810
:106B6000E10FF0D6600E2C5D040E2D590CE3800E63
:106B70002C5D040E2D5907E20FD92ED9300EDF6E91
:106B8000E4D8C10FDFD6000E2C5D050E2D590AE3A7
:106B9000050E2C5D050E2D5905E2FED8F1D8D5D88D
:106BA000230FD0D6050E2C5D050E2D590AE33A0EA3
:106BB0002C5D050E2D5905E2EFD8E2D8C6D8260F78
:106BC000C1D63A0E2C5D050E2D590CE33F0E2C5DFF
:106BD000050E2D5907E220EE04F0C5D8E9D8B5D846
:106BE000E90FB0D63F0E2C5D050E2D590CE3740E47
:106BF0002C5D050E2D5907E220EE04F0B4D8D8D84C
:106C0000A4D8EC0F9FD6400E2C5D140E2D5909E32D
:106C1000600E2C5D140E2D5904E2BED8DDD8000E96
:106C20009DD7600E2C5D140E2D5910E3800E2C5D47
:106C3000140E2D590BE220EE04F095D8380EDF6EBD
:106C400026C1D9FF27C1DAFF000E99D7420E2B6F5C
:106C50003B0E2A6F296B20EE01F02651D9262751D1
:106C6000DA22DF50286F2AC118F12BC119F1E7ECA5
:106C700019F0281902E0060E11D02A4B2B2B26C141
:106C8000D9FF27C1DAFFDF50286F2AC118F12BC1C5
:106C900019F1E7EC19F0281908E0050E2A27000E73
:106CA0002B23292B9F0E2965D6D72951A00A02E153
:106CB000D88012002A4B2B2B2AC118F12BC119F1B5
:106CC000E7EC19F0286F20EE04F026518FD8E7EC9E
:106CD00019F0286F20EE03F0265188D8E7EC19F060
:106CE000286F20EE01F0265181D8E7EC19F026C17B
:106CF000D9FF27C1DAFFDF6E20EE02F02651D92638
:106D00002751DA22DF50CFEC26F0296F20EE02F077
:106D10002651D9262751DA2229C128F1283B0F0E06
:106D2000281710EE01F02651E1262751E222E75004
:106D3000F00B2811DF6E09D8286F0F0E281729399C
:106D4000F00B2811DF6ED890120020EE01F02651D2
:106D5000D9262751DA2210EE01F02651E1262751DB
:106D6000E222E75012002651D9262751DA22060ED8
:106D7000DF6E20EE03F02651D9262751DA221200C9
:106D8000D9262751DA22400EDF6E26C1D9FF27C14E
:106D9000DAFF100EDF6E100C20EE04F02651D9261B
:106DA0002751DA22070EDF6E20EE03F02651120083
:106DB000400EDF6E26C1D9FF27C1DAFF100EDF6E4D
:106DC000100CD9262751DA22130EDF6E26C1D9FF07
:106DD00027C1DAFFDF6A130CD9262751DA22380ED1
:106DE000DF6E26C1D9FF27C1DAFF380CD92627511B
:106DF000DA2228C1DFFF2A4B2B2B2AC118F12BC125
:106E000019F11200CF0EF66EF00EF76E000EF86E4E
:106E100021EE4EF0090E0900F5CFDEFFE82EFBD77C
:106E2000000146B024D0148816BE11D0500E0101C6
:106E3000206FCE0E1F6FE6EC21F0000116B217D0C6
:106E40001682000111B613D00001168010D0500E2A
:106E50000101206FD00E1F6FE6EC21F0000116BA81
:106E600006D0168A000111B402D0000116889C9E3B
:106E7000A8847C867D6A670EAB6E9C8E9C88A88AEF
:106E8000A49AA59AA38AFBECDDF0FDE3000146A0DD
:106E900007D04690000111A603D0000111B418D00C
:106EA000F8EC1DF086CF58F1010158A916D0270E35
:106EB0005A6F100E596F5907D8A05A070101592966
:106EC000D8B45A29F8E186CF58F158A906D00E86D1
:106ED00000011188010EADEF26F0FB0E176FB90E01
:106EE000166F010E28EC1DF0130E01012A6F880E9B
:106EF000296FBAEC21F0BBE3F20E0101176F490EC6
:106F0000166F010E28EC1DF0130E01012A6F880E7A
:106F1000296FBAEC21F0F0E3F10E0101176F860E34
:106F2000166F010E28EC1DF0130E01012A6F880E5A
:106F3000296FBAEC21F0E0E3FB0E0101176F560E4A
:106F4000166F010E28EC1DF0130E01012A6F880E3A
:106F5000296FBAEC21F08BE3F30E0101176F620E7B
:106F6000166F010E28EC1DF0130E01012A6F880E1A
:106F7000296FBAEC21F001E27AD7FD0E0101176FFB
:106F80009F0E166F010E28EC1DF0130E01012A6FE3
:106F9000880E296FBAEC21F0FD0E0101176F980ED3
:106FA000166F010E28EC1DF0130E01012A6F880EDA
:106FB000296FBAEC21F0F90E0101176F550E166F0B
:106FC000010E28EC1DF0130E01012A6F880E296FA7
:106FD000BAEC21F0FD0E0101176F7C0E166F010E49
:106FE00028EC1DF0130E01012A6F880E296FBAECF0
:106FF00021F0F70E0101176F080E166F010E28EC35
:107000001DF0130E01012A6F880E296FBAEC21F0D2
:10701000F10E0101176FBB0E166F010E28EC1DF06B
:10702000130E01012A6F880E296FBAEC21F0F20EBF
:107030000101176FCA0E166F010E28EC1DF0130E1A
:1070400001012A6F880E296FBAEC21F0FB0E0101B5
:10705000176F7A0E166F010E28EC1DF0130E01014A
:107060002A6F880E296FBAEC21F001E200D7FA0EE0
:107070000101176F520E166F010E28EC1DF0130E52
:1070800001012A6F880E296FBAEC21F001E2EFD6D8
:1070900074EC13F0FB0E0101176F830E166F010ED7
:1070A00028EC1DF0130E01012A6F880E296FBAEC2F
:1070B00021F0FC0E0101176FB50E166F010E28ECC2
:1070C0001DF0130E01012A6F880E296FBAEC21F012
:1070D000F70E0101176F780E166F010E28EC1DF0E8
:1070E000130E01012A6F880E296FBAEC21F0010EF0
:1070F0000101196F440E186FE7EC19F0586F5851E1
:1071000027E0582925E0F80E176F130E166F010EB1
:1071100028EC1DF001015B6B440E5B25186F196BA9
:10712000010E1923E7EC19F0576F576701D008D00B
:107130005751A7EC2DF001015B2B100E5B65ECD7CE
:10714000FE0E176F730E166F000E28EC1DF007D0A1
:10715000FB0E176F5F0E166F010E28EC1DF0A3ECEF
:10716000BFF068EC9EF00C0A04E1A3ECBFF068EC01
:107170009EF0468603940396FB0E0101176F680E7E
:10718000166F010E28EC1DF008ECD7F068EC9EF0AD
:10719000FB0E0101176F8C0E166F010E28EC1DF00F
:1071A00008ECD7F068EC9EF0FB0E0101176F950E0E
:1071B000166F010E28EC1DF008ECD7F068EC9EF07D
:1071C000FB0E0101176F9E0E166F010E28EC1DF0CD
:1071D00008ECD7F068EC9EF001015A6B980E596FDD
:1071E00016AE04D0030E5A6F200E596F01015B6B6F
:1071F0007BD872D8E7EC19F0DF6E76D8DA22DF5050
:1072000004E05B2B1A0E5B65F3D701015A6BED0EA0
:10721000596F16AE04D0030E5A6F3B0E596F010121
:107220005B6B69D859D8E7EC19F0DF6E64D8DA22C5
:10723000DF5004E05B2B080E5B65F3D701015A6B4E
:10724000F60E596F16AE04D0030E5A6F440E596FE6
:1072500001015B6BE00E01015B25D96EDA6A050E58
:107260003BD8E7EC19F0DF6EE00E01015B25D96E2B
:10727000DA6A0501050EDA22DF5005E001015B2B19
:10728000080E5B65E7D716EC23F08EEC06F00001E4
:107290001CB470ECCFF0029C029E01015B6B4E0EA1
:1072A0005B25D96EDA6A010EDA22CF0E01015B2569
:1072B000E16EE26A060EE222DFCFE7FF5B2B070EEC
:1072C0005B65EDD7CF0E5B25D96EDA6A0601060E37
:1072D000DA22000EDF6E000CDA225B515925186F9E
:1072E000000E5A21196F1200A40E01015B25D96E00
:1072F000DA6A060E1200D70E01015B25D96EDA6A32
:10730000050E12003F6B3A6B3B6B3C6B38C121F1B1
:1073100039C122F1FC0E246FFD0E236FEBECD8F087
:1073200021513F6F3FC140F105DAFA0E246F660E1E
:10733000236FEBECD8F021513F6F3F51402736C10E
:1073400015F137C116F1C8EC0FF015C13DF116C1AA
:107350003EF1E9D910EE01F03D51E1263E51E22225
:10736000E75057EC2EF0DF6E402BDDD910EE02F027
:107370003D51E1263E51E222E75057EC2EF0DF6E00
:10738000402BD1D910EE03F03D51E1263E51E222CF
:10739000E75057EC2EF0DF6E402BC5D910EE04F00D
:1073A0003D51E1263E51E222E75057EC2EF0DF6ED0
:1073B000402BC0D9FF0E246FEA0E236FEBECD8F000
:1073C00021513F6F3F51402703013351660A01E0CD
:1073D000B8D03451660A01E0B4D035512C0A01E02E
:1073E000B0D00101A7D9FF0E246FF60E236FEBEC8E
:1073F000D8F06DD9A6D9EBECD8F069D9D96E000ECA
:107400003921DA6E7C0EDF6E402BB751310A08E16C
:1074100091D9F80E246F730E236FEBECD8F083D064
:10742000B751910A08E186D9F80E246F7F0E236FB9
:10743000EBECD8F078D0B751320A08E17BD9F80EDE
:10744000246F8B0E236FEBECD8F06DD0B751920AFE
:1074500008E170D9F80E246F970E236FEBECD8F08B
:1074600062D0B751330A08E165D9F80E246FA30E34
:10747000236FEBECD8F057D0B751930A08E15AD9F3
:10748000F80E246FAF0E236FEBECD8F04CD0B75151
:10749000980A08E14FD9F80E246F1F0E236FEBEC0A
:1074A000D8F041D0B751350A08E144D9F80E246F1D
:1074B000430E236FEBECD8F036D0B751950A08E1B4
:1074C00039D9F80E246F4F0E236FEBECD8F02BD088
:1074D000B751390A08E12ED9F80E246F2B0E236F0D
:1074E000EBECD8F020D0B751990A08E123D9F80E77
:1074F000246F370E236FEBECD8F015D0B751960AF6
:1075000008E118D9F80E246F5B0E236FEBECD8F06E
:107510000AD0B751710A0AE10DD9F80E246F670E2F
:10752000236FEBECD8F021513F6F04D00101366B93
:10753000376B12003F514027F6D85D0EDF6E402BAF
:1075400068D03351300A06E13451360A03E135512F
:107550002C0A09E03351300AE9E13451370AE6E1F7
:1075600035512C0AE3E10101E5D8FF0E246FF60E38
:10757000236FEBECD8F0ABD8E4D8EBECD8F0A7D87D
:10758000216F000E3921226FFF0E246FFA0E236F38
:10759000EBECD8F021513F6F3F51402703013351AD
:1075A000300A09E13451360A06E10101BCD8310E36
:1075B000DF6E402B04D00101B6D8330EF9D7B3D813
:1075C0003BC3DFFF0101402BAED83CC3DFFF402BA4
:1075D000AAD83DC3DFFF402BA6D8200EDF6E402B7C
:1075E000A2D83EC3DFFF402B9ED83FC3DFFF402B16
:1075F0009AD8200EDF6E402B96D840C3DFFF402B79
:1076000092D841C3DFFF402B8ED842C3DFFF402B0F
:1076100093D74051F90F3C6F86D80D0EDF6E070EE1
:107620003F6F13D03AC115F13BC116F13F513825D8
:10763000D96E000E3921DA6EDF50176FA3EC29F0F6
:1076400015C13AF116C13BF13F2B40513F5DEAE3D2
:1076500020EE01F03851D9263951DA223B51DF6E44
:1076600020EE02F03851D9263951DA223AC1DFFF33
:107670003C390F0B406F090E406504D00A0E405F85
:10768000410E01D0300E402720EE05F03851D926AA
:107690003951DA2240C1DFFF3C510F0B406F090E18
:1076A000406504D00A0E405F410E01D0300E4027E5
:1076B00020EE06F03851D9263951DA2240C1DFFFD9
:1076C000080E3C25366F376B000E3723000C215116
:1076D0003F6F3F51402740513825D96E000E392168
:1076E000DA6E36C3DFFF0101402B40513825D96ED9
:1076F000000E3921DA6E37C3DFFF402B40513825A9
:10770000D96E000E3921DA6E38C3DFFF402B4051AD
:107710003825D96E000E3921DA6E39C3DFFF402BD0
:1077200040513825120040513825D96E000E3921BC
:10773000DA6E120040513825216F000E3921226F78
:107740001200216F000E3921226FFF0E246FF80EF8
:10775000236F1200E8CFE7F0E00EF66EF00EF76E42
:10776000000EF86E20EECBF0070E0900F5CFDEFF1D
:10777000E82EFBD7D80EF66EF00EF76E000EF86E00
:1077800020EEC3F0080E0900F5CFDEFFE82EFBD790
:10779000820EF66EF00EF76E000EF86E20EE8EF092
:1077A0000E0E0900F5CFDEFFE82EFBD7900EF66E29
:1077B000F00EF76E000EF86E20EE9CF00E0E090033
:1077C000F5CFDEFFE82EFBD7640EF66EF00EF76EF7
:1077D000000EF86E20EE70F00F0E0900F5CFDEFF00
:1077E000E82EFBD7730EF66EF00EF76E000EF86EF5
:1077F00020EE7FF00F0E0900F5CFDEFFE82EFBD75D
:10780000E70EF66EF00EF76E000EF86E20EED2F078
:10781000070E0900F5CFDEFFE82EFBD7EE0EF66E61
:10782000F00EF76E000EF86E20EED9F0070E09008C
:10783000F5CFDEFFE82EFBD7AC0EF66EF00EF76E3E
:10784000000EF86E20EEAAF00D0E0900F5CFDEFF57
:10785000E82EFBD7F50EF66EF00EF76E000EF86E02
:1078600020EEE0F0070E0900F5CFDEFFE82EFBD793
:10787000B90EF66EF00EF76E000EF86E20EEB7F051
:107880000C0E0900F5CFDEFFE82EFBD7540EF66E86
:10789000F00EF76E000EF86E20EE60F0100E09008C
:1078A000F5CFDEFFE82EFBD7E7512B0A03E10001FD
:1078B000EC6B1200E7510A0A29E1EBC0F0F03ED967
:1078C000DF6AEB6B0288E86BD90EEB25D96EDA6ABA
:1078D000000EDA22DF501D6E320E0001E825D96E4F
:1078E000DA6A060EDA22DF501D1802E0EB6B02D0D6
:1078F0000001EB2BEB51060A02E1048204D0E82BD5
:10790000090EE865E1D70001EB6B1200E7510D0AA3
:1079100016E014D9E7C0DFFFEB2B310EEB6501D089
:10792000EB6B470E0001EC25D96EDA6A050EDA2200
:10793000E7C0DFFFEC2B1D0EEC651D0CB8D7EC6724
:1079400001D01200060EE86F08D0E807CB0EE8253C
:10795000D96EDA6A000EE1D82AE10001E867F5D7AE
:1079600003B403D00384010E04D003B6A0D703866A
:10797000030E0001E86F0C0EEC650CD0060EE82536
:10798000D96EDA6A030EDA2252C5DFFFDFD853C59B
:10799000DFFF8DD7060E0001E825D96EDA6A030EE7
:1079A000DA22300EDF6ED2D852C5DFFF80D7D5D8AD
:1079B00008D0E807700EE825D96EDA6A000EADD857
:1079C00005E10001E867F5D7038071D7C6D808D074
:1079D000E8077F0EE825D96EDA6A000E9ED805E129
:1079E0000001E867F5D7038262D70C0E0001E86F4B
:1079F00008D0E807AA0EE825D96EDA6A000E8DD8FD
:107A000005E10001E867F5D7038851D7AAD808D067
:107A1000E8078E0EE825D96EDA6A000E7ED805E1F9
:107A20000001E867F5D7028E42D79BD808D0E80757
:107A30009C0EE825D96EDA6A000E6FD805E10001C8
:107A4000E867F5D7028C33D7070E0001E86F08D03E
:107A5000E807C30EE825D96EDA6A000E5ED805E1A4
:107A60000001E867F5D7038E22D77FD808D0E80752
:107A7000E00EE825D96EDA6A000E4FD804E1000165
:107A8000E867F5D714D70B0E0001E86F08D0E807B8
:107A9000B70EE825D96EDA6A000E3FD805E100017D
:107AA000E867F5D7048003D760D808D0E807D20E7E
:107AB000E825D96EDA6A000E30D81DE10001E867CA
:107AC000F5D7070EEC6501D016D005014D51310AEE
:107AD00003E04D51350A02E104840DD04D51300AC6
:107AE00009E04D51320A06E04D51330A03E04D5191
:107AF000340A01E104940F0E0001E86F09D0E80791
:107B0000600EE825D96EDA6A000E07D801E0CFD6FC
:107B10000001E867F4D70482CAD6DA22DF501D6E6E
:107B20001E6A1DBE1E06470E0001E825D96EDA6AE0
:107B3000050EDA22DF501D181E101200320E000151
:107B4000EB25D96EDA6A060EDA221200050EE82558
:107B5000D96EDA6A030EDA2212000E0E0001E86F07
:107B60000E0C0D0E0001E86F0D0C060E0001E86F03
:107B7000060C000109A602D0D89012001CA409D05E
:107B80000101BA51030A05E12EECD6F0F5E3D880E5
:107B900012001CA071D00101BA056EE1020155511D
:107BA000030A6AE1324B332B100E325D270E335934
:107BB00003E3336B010E326F030E0B01A06FA56B55
:107BC00003D0CAD9DF6AA52BA551A00AFAE132C2B7
:107BD00036F133C237F10B0E0101396F000E386FE9
:107BE00082ECB9F036C1A3FB37C1A4FB0B01A45151
:107BF000A31142E03CD003A803D003980201612BFB
:107C0000FB0E0101176FC20E166F010E28EC1DF05E
:107C1000080E0101296F4C0E2A6F010E2B6F000E0A
:107C20002C6B2D6B68EC9EF00B01A56FA551080A1B
:107C30001EE1080E0101F0ECE7F068EC9EF00B018C
:107C4000A56FA551060A09E18ED931EC21F00FE3A9
:107C50001286140E02017F6F9AD7B5EC1FF000094F
:107C600004E181D931EC21F0F2D71FEC2DF00B01AA
:107C7000A007A02981E0BFD70301E8A186D0FB0EB1
:107C80000101176FB00E166F010E28EC1DF0130ED8
:107C900001012A6F880E296FBAEC21F00B01A56B48
:107CA00010D0330E0B01A525D96EDA6A030EDA2245
:107CB000000EA525E16EE26A0B0EE222DFCFE7FFA0
:107CC000A52BA551A00AEDE1E5ECF5F0D890E7353C
:107CD0000101466F476B4737330E486F030E496FFC
:107CE00048C115F149C116F103EC21F046511525A3
:107CF0004A6F475116214B6F020E4A250B01A36FA5
:107D0000000E01014B210B01A46F020EA35F000EB8
:107D1000A45BD890A433A333A3CB15F1A4CB16F165
:107D2000C8EC0FF015C1A1FB16C1A2FBFD0E176F29
:107D3000AD0E166F010E28EC1DF00B0120EE02F0C7
:107D4000A151D926A251DA22DF5057EC2EF0A7EC30
:107D50002DF00B0120EE03F0A151D926A251DA2219
:107D6000DF5057EC2EF0A7EC2DF00B0120EE04F0C5
:107D7000A151D926A251DA22DF5057EC2EF0A7EC00
:107D80002DF00D0EA7EC2DF030D0FB0E0101176F7A
:107D9000B90E166F010E28EC1DF0130E01012A6FAB
:107DA000880E296FBAEC21F0FC0E0101176FF50E59
:107DB000166F010E28EC1DF00B01A56B0DD0220EE5
:107DC0000B01A525D96EDA6A0301030EDA22DF5012
:107DD000A7EC2DF00B01A52B030132510B01A55D82
:107DE000EEE3D3ECD0F028EC1DF0EAEC2FF00AD053
:107DF000BDEC2FF007E3EEEC2FF00B01A56FA551C2
:107E00003E0A0EE0D2EC2FF0890E0101295D130E1F
:107E10002A59EEE31B0EA7EC2DF087EC2EF0ACD622
:107E2000330E0101466F030E476F46C116F147C17D
:107E300017F1000E28EC1DF00301E8A12BD0E73963
:107E40000F0B57EC2EF0A7EC2DF00301E7510F0BB1
:107E500057EC2EF0A7EC2DF00B01A56B16D07CD8BB
:107E6000DF500101466F46390F0B46BFF00957EC52
:107E70002EF0A7EC2DF00B016FD8DF500F0B57EC55
:107E80002EF0A7EC2DF00B01A52B0301E7510B0100
:107E9000A55DE5E31A0EA7EC2DF055D868EC9EF031
:107EA0000B01A56FA5512B0A2AE0A551320A27E044
:107EB000A5510C0A24E0EAEC2FF0600E0101296FB5
:107EC000EA0E2A6F2B6B2C6B010E2D6F68EC9EF067
:107ED0000B01A56FA5512B0A12E0A551320A0FE044
:107EE000A5510C0A0CE0D2EC2FF0610E0101295DC6
:107EF000EA0E2A59E2E31B0EA7EC2DF08ED7A5510E
:107F0000320A03E0A5510C0A04E11B0EA7EC2DF088
:107F100084D7EAEC2FF0D00E0101FBECF3F068EC13
:107F20009EF00B01A56FA551080A03E187EC2EF026
:107F30002ED6D2EC2FF0D10E0101295D070E2A5961
:107F400001E36BD7E8D7600E0101296FEA0E2A6FB3
:107F50002B6B2C6B2D6B000C000EA525D96EDA6AED
:107F60000B0EDA2212000B0E0101386F000E376F74
:107F7000A3CB39F1A4CB3AF11200E8CF3DF1020EC8
:107F8000F66EF10EF76E000EF86E21EE32F0060E70
:107F90000900F5CFDEFFE82EFBD746A607D1010189
:107FA0003D052EE12B0508E1010E186F000E176B41
:107FB000196B84EC1FF022D03E6B2C050FE10301FE
:107FC00022512B0A0BE0010E0101186F176B2B0ECB
:107FD000196F84EC1FF0010E01013E6F01013F6B30
:107FE00006D097D9A0D984EC1FF001013F2B7FD98F
:107FF000F8E38FD92D25A6D984EC1FF0D880120084
:108000003D51020A31E12B0509E1010E186F110EF5
:10801000176F000E196B84EC1FF0F0D73E6B2C0528
:1080200010E1030122512B0A0CE0010E0101186F2F
:10803000110E176F2B0E196F84EC1FF0010E01014A
:108040003E6F01013F6B07D064D9110E6CD984ECEF
:108050001FF001013F2B4BD9F7E35BD9110E2D2502
:1080600071D984EC1FF0CAD73D51030A31E12B05C9
:1080700009E1010E186F220E176F000E196B84ECC8
:108080001FF0BCD73E6B2C0510E1030122512B0AD7
:108090000CE0010E0101186F220E176F2B0E196FE5
:1080A00084EC1FF0010E01013E6F01013F6B07D010
:1080B00030D9220E38D984EC1FF001013F2B17D99B
:1080C000F7E327D9220E2D253DD984EC1FF096D752
:1080D0003D51040A31E12B0509E1010E186F330E01
:1080E000176F000E196B84EC1FF088D73E6B2C05C0
:1080F00010E1030122512B0A0CE0010E0101186F5F
:10810000330E176F2B0E196F84EC1FF0010E010157
:108110003E6F01013F6B07D0FCD8330E04D984ECCD
:108120001FF001013F2BE3D8F7E3F3D8330E2D25E1
:1081300009D984EC1FF062D73D51050A35E12B05C2
:1081400009E1020E186F410E176F000E196B84ECD7
:108150001FF054D73E6B2C0510E1030122512B0A6E
:108160000CE0020E0101186F410E176F2B0E196FF4
:1081700084EC1FF0010E01013E6F01013F6B0BD03B
:10818000C8D8E6D8220E01013F25FFECECF084ECC4
:108190001FF001013F2BABD8F3E3BBD8D9D8000EB9
:1081A000196B84EC1FF02AD7D89012000101010E40
:1081B000176F320E166F010E28EC1DF03D0EA7EC66
:1081C0002DF001013DC115F1166BC8EC0FF015C182
:1081D0003BF116C13CF120EE03F03B51D9263C5156
:1081E000DA22DF5057EC2EF03A6F20EE04F03B51CC
:1081F000D9263C51DA22DF5057EC2EF0396F3A5134
:10820000A7EC2DF001013951A7EC2DF001012B67EE
:1082100043D02C0EA7EC2DF0220EA7EC2DF001017F
:108220003F6B0DD0220E01013F25D96EDA6A0301A2
:10823000030EDA22DF50A7EC2DF001013F2B57D8B7
:10824000F1E3220EA7EC2DF001012C6708D0FE0E01
:10825000176F7C0E166F000E28EC1DF007D0FE0E77
:10826000176F760E166F000E28EC1DF0220EA7EC8D
:108270002DF0550EA7EC2DF001013DC115F1166B47
:10828000C8EC0FF03A51A7EC2DF001013951A7ECE1
:108290002DF0220EA7EC2DF00D0EA7EC2DF0EAEC40
:1082A0002FF00101386B19D0BDEC2FF016E3EEEC86
:1082B0002FF001013E6F0DD03E519EEC2BF00DE3EF
:1082C0000101382B0AD03E5172EC2BF001E396D617
:1082D00004D03851F1E0010AF6E0D2EC2FF0D10ED3
:1082E0000101295D070E2A5901E35ED7DDD732C3AC
:1082F0002DF101012E6B3FC12FF1306B2FBF3007E5
:108300003051800A316F2D512F5D2E51800A315925
:1083100012003E513FC12DF12E6B2DBF2E072D2790
:10832000000E2E23000C2D25176F010E2E21186F25
:10833000220E01013F25D96EDA6A030EDA22DF50E0
:10834000196F1200176F010E2E21186F196B000C98
:10835000410E2D25176F020E2E21186F1200049A60
:108360000001F26B0201646B986B0B01456B466B6D
:10837000510E01012E6F000E2D6B7EC12FF17FC1BA
:1083800030F1B7EC0AF0820509E1F30E166F950E95
:10839000156F100E176F96EC2EF009D0F30E2C6FA0
:1083A000950E2B6F2E6B100E2D6FD1ECEBF00D9008
:1083B0000201426B436B0BD00101820504E1FA0E0E
:1083C000166FF20E0CD1FA0E2C6FF20E10D180C186
:1083D0001DF181C11EF13C0E01011F6F82C120F110
:1083E000E6EC1FF00B014D6F19B4E6D74D513A0A78
:1083F000EEE1454B462B80C127F181C128F10A0EE1
:108400000101296F82C12AF1B8EC27F00B014D6FF1
:1084100019B4D2D74DCB48FB48CB56F264D9B8EC4F
:1084200027F00B014D6F19B4C7D74D510101846F6F
:10843000836B856B8451866F0B0185C149FB86C1B7
:108440004AFB4B6B4C6B4FD9B8EC27F00B014D6FCF
:1084500019B4B2D74D5149130101836B510E846F8A
:108460007C51835F7D51845B83510B01492701015E
:1084700084510B014A23000E4B234C2334D9B8EC12
:1084800027F00B01446F19B497D723D12CD9B8EC3E
:1084900027F00B01476F19B48FD7000E0001F225AA
:1084A000D96EDA6A0B0EDA2247CBDFFFF22B0B0113
:1084B0004C51800A800F08E1000E4B5D05E1510E22
:1084C0004A5D02E1000E495D0DE34C51800A800FC8
:1084D00008E1000E4B5D05E1800E4A5D02E1010EF0
:1084E000495D10E30101820506E1F70E166FC60E25
:1084F000156F0C0E76D0F70E2C6FC60E2B6F2E6BF1
:108500000C0E78D0492B000E4A234B234C2300013C
:10851000F251400A15E1C00E0B0149250101176F08
:10852000FF0E0B014A210101186F0B0E1A6F000E8E
:10853000196F400E1B6F5DEC0CF0E9D804EC09F0EC
:108540000B0148074829A2E10001F25116E0F2515F
:108550000B01495D0101176F0B014A51D8A04A0573
:108560000101186F0B0E1A6F000E196FF2C01BF18C
:108570005DEC0CF0CCD804EC09F0BFD846EC20F050
:1085800001E3048A19B418D722D7B7D846EC20F0F3
:1085900001E3048A19B410D704AA10D0010182059E
:1085A00006E1FB0E166FF80E156F080E1AD0FB0EC3
:1085B0002C6FF80E2B6F2E6B080E1CD001017D5115
:1085C0007C111BE1510E196FFF0E1869E7EC19F0D1
:1085D000220A13E0820508E1FA0E166FE80E156F05
:1085E000090E176F96EF2EF0FA0E2C6FE80E2B6F18
:1085F0002E6B090E2D6FD1EFEBF07CC12DF17DC1FB
:108600002EF17EC12FF17FC130F182C131F1E0EC5A
:10861000EFF00B0E0101226F000E216FFD0E246F93
:10862000D70E236F45CB25F146CB26F1EBECD8F0E6
:1086300021510B014D6F0101820510E10B0E166FE8
:10864000000E156F4DCB17F196EC2EF0000111B80E
:108650001200000146A607ECD8F012000B0E010133
:108660002C6F000E2B6F4DCB2DF12E6BD1ECEBF060
:10867000D9EC2FF0F90E0101176F1B0E166F010ECA
:1086800028EC1DF0EAEC2FF0D2EC2FF0E90E0101FE
:10869000295D030E2A59F8E3FF00FF0004ECAFF058
:1086A000000146A607ECD8F01CEC05F070ECCFF00A
:1086B000148C0001188C120016D8B8EC27F019B4ED
:1086C0007BD60B0148074829F7E117D846EC20F084
:1086D00057D70B01445101E133D7010A01E155D7C6
:1086E000050AEFE074D680C127F181C128F10A0E96
:1086F0000101296F82C12AF10A0C80C12DF181C1CB
:108700002EF10A0E01012F6F82C130F10A0C0B010C
:10871000406F0B0E0101166F000E156F0B0E186FD8
:10872000400E176F12008B6B8C6B3951381103E1BF
:10873000366B376B1200000E196B186BE7EC19F0F3
:10874000B351F6E136C13DF137C13EF138513D2715
:1087500039513E233DC187F13EC188F1896B8A6B57
:108760008A51800A800F08E1000E895D05E1800EC4
:10877000885D02E1010E875DDBE236C185F137C11C
:1087800086F1526B02012E6B2F6B01013C0509E152
:10879000F20E166FDE0E156F130E176F96EC2EF09D
:1087A00016D0F20E306FDE0E2F6F326B130E316F5C
:1087B000A5EC0DF00CE3D9EC2FF01FEC2DF0188C8C
:1087C000148C000E0101376F010E366F010C010190
:1087D0008B4B8C2BFFD0916B906B68D985C118F1B6
:1087E00086C119F1E7EC19F0DF6E854B862B420E3E
:1087F0009025D96EDA6A010EDA22DF1C02E0010E42
:10880000916F902B0F0E9065E8D7916705D0100EF1
:108810003627000E3723DED0010E166F520E156F6D
:10882000FE0E186FB20E176FFAEC24F0100E8E6F5A
:1088300037518F6F42D903EC21F02FD98F390F0BAD
:1088400057EC2EF0DF6E91C13DF13D2B1FD98F51BA
:108850000F0B57EC2EF0DF6E91C13DF1020E3D275C
:1088600015D9DF6A36C18FF128D903EC21F015D96B
:108870008F390F0B57EC2EF0DF6E91C13DF13D2B80
:1088800005D98F510F0B57EC2EF0DF6E91C13DF1E2
:10889000020E3D27FBD8DF6A166F520E156FF80ED9
:1088A000186F280E176FFAEC24F0906BFFD8DF508A
:1088B0008D6F364B372B8D518E27010E166F520E52
:1088C000156F03EC21F0E9D88D390F0B57EC2EF022
:1088D000DF6E91C13DF13D2BD9D88D510F0B57EC77
:1088E0002EF0DF6E91C13DF1020E3D27CFD8DF6A39
:1088F000902B0F0E9065DAD78E5100088E6F010E07
:10890000166F520E156F03EC21F0C7D88E390F0B7E
:1089100057EC2EF0DF6E91C13DF13D2BB7D88E5153
:108920000F0B57EC2EF0DF6E91C13DF1020E3D278B
:10893000ADD80D0EDF6E91C13DF1030E3D27A6D8D7
:108940000A0EDF6E91C13DF1040E3D279FD8DF6A0C
:10895000166F520E156F03EC21F01551916F906B4D
:10896000520E9025D96EDA6A010EDA2290513A251C
:10897000E16E000E3B21E26EDFCFE7FF902B300E61
:108980009065EED73C0509E13AC115F13BC116F1FE
:1089900091C117F196EC2EF00BD03AC12FF13BC1EB
:1089A00030F191C131F1326BA5EC0DF001E303D749
:1089B00001018B4B8C2B526B070E846FD00E836F93
:1089C00001D000F001018307D8A084078329D8B41F
:1089D0008429F7E136513D6F37513E6F3F6B406B55
:1089E0004051800A416F87513D5D88513E59895100
:1089F0003F598A51800A415901E2EDD63C0509E10F
:108A0000F30E166F3E0E156F110E176F96EC2EF0CB
:108A10000BD0F30E306F3E0E2F6F326B110E316F95
:108A2000A5EC0DF001E3C7D601018B4B8C2B010E99
:108A3000226F520E216FFD0E246FD70E236F8BC154
:108A400025F18CC126F1EBECD8F02151906F3C055B
:108A500009E1010E166F520E156F90C117F196ECD9
:108A60002EF00FD0010E306F520E2F6F90C131F1EA
:108A7000326BA5EC0DF001E39ED6B9EC18F001E3E2
:108A80009AD68BC136F18CC137F11200520E3D25BA
:108A9000D96EDA6A010EDA2212001551916F520E68
:108AA0009125D96EDA6A010EDA221200420E902563
:108AB000D96EDA6A010EDA2212008F518E27010E6A
:108AC000166F520E156F1200360E96D9DF620FD058
:108AD00020EE04F08CD983D9130EDF6E8DD9000EF1
:108AE000DF6E1FC115F120C116F141EF1BF0380EEA
:108AF00083D9DF6205D020EE04F01F518CD9EBD76B
:108B0000570E7AD9DF6206D020EE04F070D967D90B
:108B1000100EE3D7580E70D9DF6206D020EE04F0B5
:108B200066D95DD9570ED9D7370E66D9DF6204D022
:108B300020EE04F05CD908D0390E5ED9DF6207D090
:108B400020EE04F01F5167D94AD9110EC6D7420E44
:108B500053D9DF6209D020EE04F049D940D9130E71
:108B6000DF6E4AD9700EBCD7430E46D9DF6205D0FE
:108B700020EE04F01F514FD9F1D7530E3DD9DF62DB
:108B800009D020EE04F033D92AD9140EDF6E34D97F
:108B9000300EA6D7540E30D9DF6205D020EE04F097
:108BA0001F5139D9F1D7550E27D9DF6209D020EEF0
:108BB00004F01DD914D9140EDF6E1ED9500E90D7B3
:108BC000560E1AD9DF6205D020EE04F01F5123D9CA
:108BD000F1D7510E11D9DF6204D020EE04F007D98D
:108BE00008D0520E09D9DF6207D020EE04F01F51E1
:108BF00012D9F5D8380E71D7490EFED8DF6209D0E8
:108C000020EE04F0F4D8EBD8380EDF6EF5D8400E25
:108C100067D7500EF1D8DF6205D020EE04F01F5167
:108C2000FAD8F1D7290EE8D8DF620AD020EE04F096
:108C30001F51F1D8D4D8400EDF6EDED8100E50D7B9
:108C4000310EDAD8DF6204D020EE04F0D0D8F2D7AB
:108C5000320ED2D8DF6206D020EE04F0C8D8BFD8DA
:108C6000400E3BD7330EC8D8DF6209D020EE04F0A7
:108C7000BED8B5D8400EDF6EBFD8600E31D7280EF3
:108C8000BBD8DF6209D020EE04F0B1D8A8D8450ED9
:108C9000DF6EB2D8800E24D7AFD8DF50350A01E19D
:108CA0003DD7410EA9D8DF6201D038D7480E246FD6
:108CB000530E236F256B20EE01F01F51D926205152
:108CC000DA22DF50216F23C118F124C119F1E7EC3A
:108CD00019F0211902E0060E11D0234B242B1FC1DD
:108CE000D9FF20C1DAFFDF50216F23C118F124C161
:108CF00019F1E7EC19F0211908E0050E2327000E01
:108D00002423252B770E2565D6D72551780A30E107
:108D100020EE02F01F51D9262051DA22DF50256FB4
:108D200020EE04F064D85BD81FC1E1FF20C1E2FF50
:108D3000E750216F21390F0BDF6E79D81FC1E1FF9A
:108D400020C1E2FFE750226F2239F00B211167D8D2
:108D50001FC1E1FF20C1E2FFDFCFE7FF20EE01F0FE
:108D60001F51D9262051DA222539F00BDF6E12006F
:108D700020EE04F01F5145D8E7EC19F030D8234B12
:108D8000242B23C118F124C119F1E7EC19F0DF6E8F
:108D900020EE01F01F5135D8E7EC19F0DF6E234BC0
:108DA000242B23C118F124C119F1E7EC19F024D8C0
:108DB000DF6E20EE02F01F51D9262051DA22DF505B
:108DC000256F35D840D8F00B211129D83CD8216F18
:108DD0000F0E21172539F00B2111DF6E1200DF6E07
:108DE00020EE03F01F51D9262051DA2212001F5124
:108DF000D9262051DA22060C1FC1D9FF20C1DAFF83
:108E00001200D9262051DA22234B242B23C118F13A
:108E100024C119F11200D9262051DA22070CDF6E85
:108E200020EE01F01F51D9262051DA22120020EE47
:108E300002F01F51D9262051DA2225C121F1213B10
:108E40000F0E21170F0C10EE01F01F51E1262051DB
:108E5000E222E7501200590E9DD9DF6212D020EEB7
:108E600004F093D98AD9130EDF6E94D9000E97D9E6
:108E7000000EDF6E26C11EF127C11FF1B3EC09F011
:108E800036D1490E87D9DF620BD020EE04F07DD9B0
:108E900074D9130EDF6E7ED9000E81D9010EE9D789
:108EA000790E78D9DF620BD020EE04F06ED965D947
:108EB000130EDF6E6FD9000E72D9020EDAD75E0E76
:108EC00069D9DF6208D020EE04F02651D926275157
:108ED000DA22070EC7D74E0E5DD9DF6208D020EE2A
:108EE00004F02651D9262751DA22070ED1D77E0E5B
:108EF00051D9DF6208D020EE04F02651D92627513F
:108F0000DA22070ED4D75D0E45D9DF620BD020EEF2
:108F100004F02651D926275126D9130EDF6E3AD9EF
:108F2000700EA5D74D0E36D9DF620BD020EE04F0BF
:108F30002651D926275117D9130EDF6E2BD9700E63
:108F4000ACD77D0E27D9DF620BD020EE04F026517E
:108F5000D926275108D9130EDF6E1CD9700EACD755
:108F6000580E18D9DF620DD020EE04F02651D92614
:108F70002751DA22070E01D9400EDF6E0BD9100EF1
:108F800076D7480E07D9DF620DD020EE04F02651C7
:108F9000D9262751DA22070EF0D8400EDF6EFAD814
:108FA000100E7BD7780EF6D8DF620DD020EE04F0DD
:108FB0002651D9262751DA22070EDFD8400EDF6E60
:108FC000E9D8100E79D75B0EE5D8DF6204D020EE29
:108FD00004F0DBD8D0D74B0EDDD8DF6204D020EE12
:108FE00004F0D3D8D9D77B0ED5D8DF6204D020EED9
:108FF00004F0CBD8E2D75F0ECDD8DF6208D020EEE8
:1090000004F02651D9262751AED8570E2DD74F0E32
:10901000C1D8DF6208D020EE04F02651D9262751AE
:10902000A2D8570E37D77F0EB5D8DF6208D020EE12
:1090300004F02651D926275196D8570E3AD7450E17
:109040002A6FFB0E296F2B6B20EE01F02651D926DB
:109050002751DA22DF50286F29C118F12AC119F1EE
:10906000E7EC19F0281902E0060E11D0294B2A2B43
:1090700026C1D9FF27C1DAFFDF50286F29C118F1B7
:109080002AC119F1E7EC19F0281908E0050E292783
:10909000000E2A232B2B630E2B65D6D72B51640A87
:1090A00028E120EE04F02651D92627515CD826C1AC
:1090B000E1FF27C1E2FFE750286F28390F0B6FD877
:1090C00026C1E1FF27C1E2FFE750286F2839F00BE6
:1090D00078D826C1E1FF27C1E2FFDFCFE7FF20EE0E
:1090E00001F02651D9262751DA22000EDF6ED890E2
:1090F000120020EE04F026515AD8E7EC19F03DD8C2
:10910000294B2A2B29C118F12AC119F1E7EC19F0D2
:10911000DF6E20EE01F026514AD8E7EC19F0DF6E41
:10912000294B2A2B29C118F12AC119F1E7EC19F0B2
:1091300031D835D8DF502B6F20EE02F02651D926DA
:109140002751DA222BC128F1283B0F0E281741D8CE
:10915000F00B281136D83DD8286F0F0E28172B3961
:10916000F00B2811C3D7DA22060EDF6E20EE03F0D3
:109170002651D9262751DA221200DF6E20EE03F0A5
:109180002651D9262751DA2212002651D9262751F5
:10919000DA22060C26C1D9FF27C1DAFF1200DF6EE2
:1091A00020EE02F02651D9262751DA221200D926C4
:1091B0002751DA22294B2A2B29C118F12AC119F18A
:1091C0001200DF6E20EE01F02651D9262751DA2257
:1091D000120010EE01F02651E1262751E222E7505D
:1091E0001200190E93D9DF6210D020EE04F093D94B
:1091F00085D9110EDF6E8AD9000EDF6E29C11EF1EE
:109200002AC11FF1D2ECF9F077D11B0E7FD9DF62B2
:1092100005D020EE04F0295183D9EAD71F0E76D964
:10922000DF6209D020EE04F076D968D9120EDF6E25
:109230006DD9100EE2D7180E69D9DF6204D020EE86
:1092400004F069D915D0210E61D9DF6209D020EE72
:1092500004F061D953D9140EDF6E58D9400ECDD722
:109260001A0E54D9DF6207D020EE04F0295158D9E4
:1092700045D9130EBFD7220E49D9DF6205D020EEA3
:1092800004F029514DD9E6D72A0E40D9DF6204D027
:1092900020EE04F040D910D0290E38D9DF6204D076
:1092A00020EE04F038D913D02C0E30D9DF6207D06D
:1092B00020EE04F0295134D921D9380EB8D72B0E1D
:1092C00025D9DF6207D020EE04F0295129D916D91B
:1092D000380EC2D71BD9DF500A0A04E0090E16D98E
:1092E000DF6205D020EE04F029511AD92BD00B0EE5
:1092F0000DD9DF620AD020EE04F0295111D9FED831
:10930000400EDF6E03D9900E78D700D9DF50100AD7
:1093100008E0FCD8DF50110A04E0120EF7D8DF6233
:1093200006D020EE04F0F7D8E9D8400E63D7EED887
:10933000DF500E0A04E00D0EE9D8DF6206D020EE01
:1093400004F0E9D8DBD8400E72D70F0EDFD8DF6209
:1093500004D020EE04F0DFD8D2D7D8D8DF50130ADB
:1093600008E0D4D8DF50140A04E0150ECFD8DF622D
:1093700009D020EE04F0CFD8C1D8400EDF6EC6D899
:10938000600E3BD71C0EC2D8DF6204D020EE04F082
:10939000C2D815D01D0EBAD8DF6209D020EE04F075
:1093A000BAD8ACD8450EDF6EB1D8200E26D72E0E17
:1093B000ADD8DF6207D020EE04F02951B1D89ED895
:1093C000450E35D72F0EA2D8DF6205D020EE04F06F
:1093D0002951A6D8E6D73A0E99D8DF6206D020EEFA
:1093E00004F099D88BD8530E22D73B0E8FD8DF626A
:1093F00006D020EE04F08FD881D8530ED4D786D86B
:10940000DF50170A04E0380E81D8DF6204D020EE66
:1094100004F081D808D0390E79D8DF6207D020EE69
:1094200004F029517DD86AD8570EE4D64B0E2E6F22
:10943000230E2D6F2C6B20EE02F02951D9262A51D4
:10944000DA22DF502B6F2DC118F12EC119F1E7EC94
:1094500019F02B1902E0060E11D02D4B2E2B29C12D
:10946000D9FF2AC1DAFFDF502B6F2DC118F12EC1B1
:1094700019F1E7EC19F02B1908E0050E2D27000E65
:109480002E232C2B770E2C65D6D72C51780A02E18F
:10949000D880120020EE04F0295146D8E7EC19F0EC
:1094A0002DD82D4B2E2B2DC118F12EC119F1E7EC23
:1094B00019F0DF6E20EE02F0295136D8E7EC19F0F2
:1094C000DF6E2D4B2E2B2DC118F12EC119F1E7ECBB
:1094D00019F01CD8DF6E20EE01F02951D9262A514F
:1094E000DA2210EE01F02951E1262A51E222E7505A
:1094F0002B6F2B39F00BDF6ED8901200DF6E20EE51
:1095000003F02951D9262A51DA22120029C1D9FFA4
:109510002AC1DAFF12002951D9262A51DA22060C73
:10952000D9262A51DA22070CD9262A51DA222D4BC4
:109530002E2B2DC118F12EC119F11200E8CF38F1F0
:10954000FC0EF66EF00EF76E000EF86E21EE30F0A7
:10955000060E0900F5CFDEFFE82EFBD746A691D018
:10956000010138051EE1010E196F000E186BE7ECC2
:1095700019F0000902E1D89012003C6B000E3C2566
:10958000186F196B010E1923E7EC19F03B6F3B675D
:1095900001D003D06CD93C65F1D73CC132F3D880FF
:1095A00012003851020A19E1010E196F110E186FDD
:1095B000E7EC19F00009DFE03C6B110E3C25186F59
:1095C000196B010E1923E7EC19F03B6F3B6701D0D3
:1095D000E4D74DD93C65F1D7E0D73851030A19E1FA
:1095E000010E196F220E186FE7EC19F00009C3E0A5
:1095F0003C6B220E3C25186F196B010E1923E7EC0A
:1096000019F03B6F3B6701D0C8D731D93C65F1D722
:10961000C4D73851040A19E1010E196F330E186FBF
:10962000E7EC19F00009A7E03C6B330E3C25186FFE
:10963000196B010E1923E7EC19F03B6F3B6701D062
:10964000ACD715D93C65F1D7A8D73851050A93E1B5
:10965000020E196F410E186FE7EC19F000098BE04C
:109660003C6B410E3C25186F196B020E1923E7EC79
:1096700019F03B6F3B6701D090D7F9D83C65F1D723
:109680008CD70101010E176F300E166F010E28ECFA
:109690001DF03D0EA7EC2DF0010138C115F1166B40
:1096A000C8EC0FF015C136F116C137F120EE03F00A
:1096B0003651D9263751DA22DF5057EC2EF0A7EC7D
:1096C0002DF0010120EE04F03651D9263751DA226F
:1096D000DF5057EC2EF0A7EC2DF00D0EA7EC2DF07F
:1096E000D00E0101296F070E2A6F000E2B6B2C6B19
:1096F0002D6B68EC9EF001013C6F3C51150A23E094
:109700003C51080A20E03C510C0A1DE0EAEC2FF025
:10971000D00E0101FBECF3F068EC9EF001013C6F10
:109720003C51150A10E03C51080A0DE03C510C0A6E
:109730000AE0D2EC2FF0D10E0101295D070E2A5963
:1097400001E319D7E5D73C51080A01E114D73C5190
:109750000C0A01E110D73C51150A71E13C6B92D81B
:109760002C0E176F44EC2BF015C139F116C13AF1EC
:109770003A51391101E1FFD6394B3A2B39C115F174
:109780003AC116F1186B2C0E176F44EC2BF015C173
:1097900039F116C13AF13A51391101E1ECD6394BA0
:1097A0003A2B39C11BF13AC11CF1B1ECFCF01B5151
:1097B0003B6F3B51910A06E12B0E0301226F010E14
:1097C00001013C6F5FD8220E176F44EC2BF015C1DE
:1097D00039F116C13AF13A51391101E1CCD6394B80
:1097E0003A2B220E39C1D9FF3AC1DAFFDF6201D02C
:1097F00013D00F0E3C6501D00FD039C1D9FF3AC14B
:10980000DAFF220E01013C25E16EE26A030EE2223C
:10981000DFCFE7FF3C2BE3D73CC132F33B6B050EB8
:109820000101256F850E246FFF0E276FE70E266F4F
:1098300043EC16F02551241102E0010E3B6FEAECD7
:109840002FF0D00E0101FBECF3F068EC9EF001016B
:109850003C6F3C51080A08E0D2EC2FF0D10E010118
:10986000295D070E2A59EDE33B6799D684D6220E6F
:1098700001013C25D96EDA6A030EDA223BC1DFFF13
:109880003C2B0F0C050E0101166F850E156F186B22
:109890001200E8CF48F14F6B526B1CD0340E4F25AD
:1098A000D96EDA6A010EDA22DF6A330E010152251F
:1098B000D96EDA6A030EDA224FC130F1302B340E42
:1098C0003025E16EE26A010EE222DFCFE7FF522B84
:1098D000020E4F272F515263E1D74F6B2F512F2587
:1098E000526F506B516B0DD0340E5025D96EDA6A21
:1098F000010EDA22330E010150256EECF2F0504BCE
:10990000512B52C130F145D9EFE3415025E042508F
:1099100023E0330E010124D9280EDF6E522B41289B
:1099200005E152518AECF8F0526F0BD0330E010171
:1099300017D941C0DFFF522B330E12D942C0DFFFCF
:10994000522B330E01010CD9290EDF6E522B330E30
:1099500007D9200EDF6E522B48074851330D8D0E6C
:10996000F324496F130EF4204A6F49C118F14AC11C
:1099700019F1E7EC19F04D6F4E6B4E51800A800FD4
:10998000020ED8B44D5D07E34E51800A800F180EC9
:10999000D8B44D5D03E352C1E7F31200D8904D35C2
:1099A000306F4E35316F52513025506F000E3121DE
:1099B000516F5151800A800FA10ED8B4505DEBE277
:1099C00050C1E7F35007D8A05107D8904D35306FFC
:1099D0004E35316F4851330D3051F324326F3151D0
:1099E000F420336F8D0E3225496F130E33214A6FE9
:1099F00059D049C118F14AC119F1E7EC19F0306F9B
:109A0000FF0E4925186FFF0E4A21196FE7EC19F078
:109A10004C6F30514B6F4B513F0A4C1132E14F2B81
:109A2000030E01014F6501D04F6BCCD8DF6A4F05A3
:109A300008E1330E5025D96EA1D80F0B57EC2EF04C
:109A40001ED04F51020A0DE1330E01015025D96E8F
:109A500095D8306F30390F0B30BFF00957EC2EF02E
:109A60000ED04F51030A13E19ED810EE02F02D5193
:109A7000E1262E51E222E7500F0B57EC2EF0DF6E5D
:109A800006D0A0D84C51DF6E96D84BC1DFFF4D07F2
:109A9000D8A04E07FE0E5027FF0E5123020E495F3D
:109AA000000E4A5B4E51800A800F010ED8B44D5D06
:109AB000A0E2506B516B1CD076D8DF50316F306B09
:109AC000340E5025D96EDA6A030EDA22DF50326F77
:109AD000336B32BF3307325130114B6F31514C6F02
:109AE0004B51240A4C1109E0020E5027000E51235D
:109AF000E7C330F101014DD8DFE30301E751010174
:109B000050195111D8B41200020E5027000E5123E3
:109B1000526B10D0504B512B330E01015025D96E92
:109B2000030E5121DA6E330E52256EECF2F0504BDB
:109B3000512B522BE7C330F101012BD8EBE33BD87B
:109B4000DF6A330E306F030E316F30C115F131C152
:109B500016F103EC21F015510301E76FE86B1200D9
:109B60005225D96EDA6A030EDA22DF6A522B330EDF
:109B70005225D96EDA6A030EDA221200DA6A030E6F
:109B8000DA2210EE03F02D51E1262E51E222E750A9
:109B90001200316B5151800A326F3051505D31519A
:109BA000800A32591200330E01015025D96EDA6A4B
:109BB000030EDA221200330E5025D96EDA6A030E34
:109BC000DA221200320E01015025D96EDA6A030E34
:109BD000DA221200A496BC0E776E786A15A02CD0FB
:109BE00002018A51436206D0F092F088A3960001E8
:109BF000159012000001F56705D08A92432A0A0EDB
:109C0000F56F0A0CF50506E1436602D08A9211D081
:109C10008A820FD0F5510A0AFBE054D9DF500101C6
:109C2000096F09A102D08A9201D08A824BD9D890BB
:109C3000DF320001F50712000001F75143E0158003
:109C40000A0EF56F436AF70515E143D9A20EEA6FD4
:109C50004E0EEB6FF3C0ECF3030E0101016FE90E42
:109C6000006F8AC202F158ECF6F0E9C0EDF340C291
:109C7000EEF326D0F751020A03E12BD9A10EE7D764
:109C8000F751030A0DE1040E02018A6F080E030169
:109C9000E96F400EEA6F480EEB6F500EEC6F10D07C
:109CA000F751040A0DE1050E02018A6F080E030147
:109CB000E96F440EEA6FEB6B4C0EEC6FA00EED6F8C
:109CC0000001F76B15A2E9D00001F567DBD0159212
:109CD000F092F088A39681B4ACD7E90E4324D96EF4
:109CE000DA6A030EDA220201881DDF6E432A0F0EA4
:109CF000436401D0436A030E0101016FE90E006F56
:109D000043C002F1E9EC23F004E3040E0001F76F15
:109D1000118E0001F6672CD0030E0101016FE90ED0
:109D2000006F43C002F1CEEC2AF001E2A2D0C2D80B
:109D300058ECF6F001E29DD00301EC51FE1901E16F
:109D400098D046A204D0ECC3FEF3469292D0FEC354
:109D5000F3F00001F351B80A02E1F36B01D0F32BE9
:109D6000010EF66F130E02013F6F880E3E6F81D019
:109D7000F60514E1030E0101016FE90E006F43C007
:109D800002F138EC29F075E395D858ECF6F071E360
:109D9000010E0001F76F020EF66F6BD0F651020A4A
:109DA00038E1030E0101016FE90E006F43C002F1BB
:109DB0002DEC2BF05EE37ED858ECF6F05AE3020E61
:109DC0000001F76F030EF66F0301EB510A0A03E17E
:109DD00002019D6B02D0EBC39DF20301EC510A0A14
:109DE00003E102019E6B02D0ECC39EF20301ED5130
:109DF0000A0A03E102019F6B02D0EDC39FF2030147
:109E0000EE510A0A03E10201A06B33D0EEC3A0F2C7
:109E100030D0F651030A2DE1030E0101016FE90E66
:109E2000006F43C002F116EC2BF023E343D858EC4B
:109E3000F6F01FE3030E0001F76FF66BF3C0FEF3BD
:109E40000301EE290201A16FF1C309F1060E010120
:109E50000A6FD89009330A2FFCD7030E09170301A4
:109E6000F0390F0B0C0B010109110201A26FA22B9B
:109E7000118C0001F75101E1DCD67768786AF0981F
:109E8000A386D7D6F50503E181A4436AD2D6D8903C
:109E900081B4D88002018833CCD6000114BE81A4DD
:109EA00012000201886B149E1582090E0001F56FE5
:109EB000F098090C030E0101016FE90E006F43C019
:109EC00002F11200E90E4324D96EDA6A030EDA2297
:109ED0001200060E02018A6F080E0301E96F080CDA
:109EE000010E0101196F9A0E186FE7EC19F04D6F12
:109EF0004D51D8B412004D29D8B41200020E196F7A
:109F0000210E186FE7EC19F04D6F4D51D8B41200C7
:109F10004D29D8B41200FA0E176F3C0E166F010EC1
:109F200028EC1DF0130E01012A6F880E296FBAEC80
:109F300021F0F20E0101176F030E166F010E28ECCF
:109F40001DF011ECD7F028EC1DF0130E01012A6F63
:109F5000880E296FBAEC21F0F20E0101176F750E11
:109F6000166F010E28EC1DF011ECD7F028EC1DF057
:109F7000130E01012A6F880E296FBAEC21F0F10E41
:109F80000101176FA20E166F010E28EC1DF00101E2
:109F90004D6B02D99A0E4D25186F196B010E1923BE
:109FA000E7EC19F0DF6EF8D8DF5004E04D2B1F0E00
:109FB0004D65EFD7010E176F2D0E166F000E28ECB2
:109FC0001DF0FF0E0101176FED0E166F000E28EC4D
:109FD0001DF001014D6BE0D8BA0E4D25186F196BBD
:109FE000010E1923E7EC19F0DF6ED6D8DF5004E03C
:109FF0004D2B050E4D65EFD7010E176F2D0E166F09
:10A00000000E28EC1DF00D0EA7EC2DF0130E010133
:10A010002A6F880E296FBAEC21F01CA249D0F20EEB
:10A020000101176F5F0E166F010E28EC1DF0010184
:10A030004D6BB2D8C00E4D25186F196B010E192348
:10A04000E7EC19F0DF6EA8D8DF5004E04D2B1F0EAF
:10A050004D65EFD7010E176F2D0E166F000E28EC11
:10A060001DF0A7D828EC1DF001014D6B95D8E00E2E
:10A070004D25186F196B010E1923E7EC19F0DF6EEF
:10A080008BD8DF5004E04D2B0F0E4D65EFD7010E3E
:10A09000176F2D0E166F000E28EC1DF084D828ECDB
:10A0A0001DF0130E01012A6F880E296FBAEC21F002
:10A0B000F20E0101176FB50E166F010E28EC1DF0A0
:10A0C00001014D6B69D8F10E4D25186F196B010E0A
:10A0D0001923E7EC19F0DF6E5FD8DF5004E04D2B59
:10A0E0000F0E4D65EFD7010E176F2D0E166F000E78
:10A0F00028EC1DF05ED828EC1DF001014D6B4CD80A
:10A100004D29186F196B020E1923E7EC19F0DF6E59
:10A1100043D8DF5004E04D2B1F0E4D65F0D7010EE4
:10A12000176F2D0E166F000E28EC1DF03CD828EC92
:10A130001DF0130E01012A6F880E296FBAEC21F071
:10A14000F40E0101176F370E166F010E28EC1DF08B
:10A1500001014D6B21D8210E4D25186F196B020E90
:10A160001923E7EC19F0DF6E17D8DF5004E04D2B10
:10A170001F0E4D65EFD7010E176F2D0E166F000ED7
:10A1800028EC1DF010D828EC1DF0130E01012A6FE9
:10A19000880E296FBAEF21F02D0E4D25D96EDA6A9F
:10A1A000010EDA221200FE0E0101176F730E166FF8
:10A1B000000CF30E0101176F160E166F000CE8CF9E
:10A1C00097F10301E70528E037D00101975116EC1C
:10A1D00020F002E2D8901200D880120001019751BD
:10A1E00020EC25F0F6D7010197515CEC1AF0F1D77D
:10A1F0000101975179EC1BF0ECD701019751F3EC79
:10A200001CF0E7D7010197515CEC1EF0E2D7010189
:10A21000975115EC10F0DDD733512A0AD6E01A0A0F
:10A22000DDE0010AE0E0030AE3E0010AE6E0070AF4
:10A23000E9E00D0AECE0CED734512E0A0BE010D045
:10A24000010197510DECF3F0C4D70101975181EC56
:10A25000F1F0BFD73351310AF3E0020AF6E0BAD782
:10A26000E751020A4BE13351380A1FE02CD00101BB
:10A2700097516BEC25F0ADD70101975122EC1FF0FF
:10A28000A8D701019751F1EC1EF0A3D70101975116
:10A29000C0EC1EF09ED70101975153EC1FF099D7E7
:10A2A00001019751B2EC2EF094D73451300ADFE01F
:10A2B000010AE2E0030AE5E0010AE8E0070AEBE050
:10A2C000010AEEE087D73351390A10E017D00101B7
:10A2D0009751CFEC1AF07DD70101975108EC1BF094
:10A2E00078D70101975196EC1AF073D73451320A9E
:10A2F000EEE0010AF1E0070AF4E06CD735512E0ACE
:10A300007AE13351300A06E009D00101975109EC96
:10A310000CF05FD73451300AF8E05CD73351310A82
:10A3200015E01ED0010197518CECF2F052D70101DB
:10A3300097518CECF2F04DD701019751D6EC05F016
:10A3400048D70101975151ECE9F043D73451300A15
:10A35000E9E0010AECE0030AEFE0070AF2E03AD78D
:10A360003351380A0BE010D00101975161EC0BF02A
:10A3700030D7010197510AEC0AF02BD73451360A35
:10A38000F3E0010AF6E026D73351390A24E033D04E
:10A39000010197519FECDFF01CD7010197517CEC34
:10A3A000DBF017D70101975151ECDCF012D7010116
:10A3B000975126ECDDF00DD70101975114ECFBF01D
:10A3C00008D701019751A9ECFAF003D70101975181
:10A3D00000EC98F0FED63451310ADAE0030ADDE0F1
:10A3E000010AE0E0070AE3E0010AE6E0030AE9E027
:10A3F0000F0AECE0EFD636512E0A0EE13351300A47
:10A400000BE13451380A08E13551310A05E1010107
:10A4100097515DEC1DF0DDD633512E0A05E10101A7
:10A42000975154EC0DF0D5D6000112A4D3D6000EEE
:10A43000BEECABF0CFD60101746B756B786B300E50
:10A440007825D96EDA6A010EDA22DF68782B785126
:10A45000800A400FF4E3766B776BF9D8400E2A6FD1
:10A460008BEC26F0400E7427000E7523764B772B6D
:10A470007751800A800F100ED8B4765DEEE3030E9C
:10A48000776F4E0E766F746B756B000E2D6F040E2A
:10A490002E6F2DC115F12EC116F1176B186BCBEC79
:10A4A0002FF03FD0C00E76252D6FFF0E77212E6F37
:10A4B0002E51800A800F010ED8B42D5D15E3786B04
:10A4C0000900CED87851800A400FFAE3C0D8400E78
:10A4D0002A6F8BEC26F0400E7427000E7523C00EF9
:10A4E0007627FF0E77231DD0786B02D00900B8D8ED
:10A4F00078C12DF12E6B2DBF2E072E51800A2F6FA4
:10A5000076512D5D7751800A2F59F0E3A0D876C19E
:10A510002AF18BEC26F07651742777517523766BF0
:10A52000776B77517611BEE14F0E186FD30E176F10
:10A53000020EF66E040EF76E000EF86E0800F5CFF0
:10A5400019F184EC1FF04F0E0101186FD40E176F34
:10A55000620EF66E040EF76E000EF86E0800F5CF70
:10A5600019F184EC1FF04F0E0101186FD50E176F13
:10A57000630EF66E040EF76E000EF86E0800F5CF4F
:10A5800019F184EC1FF0130E0101196F6A0E186F98
:10A59000E7EC19F02D6F300E2D5D1AE3130E196FD5
:10A5A0006A0E186FE7EC19F02D6F3A0E2D5D10E270
:10A5B000196B750E186FE7EC19F0706F7051080980
:10A5C000716F186B750E176F71C119F184EC1FF064
:10A5D000130E0101196F790E186FE7EC19F02D6F4A
:10A5E000300E2D5D1AE3130E196F790E186FE7EC1C
:10A5F00019F02D6F3A0E2D5D10E2196B750E186F64
:10A60000E7EC19F0726F72510809736F186B750ED1
:10A61000176F73C119F184EC1FF00101786BBE0E46
:10A620002D6F500E2E6F2D517825176F000E78BFAD
:10A63000FF0E2E21186F000E196B84EC1FF0010124
:10A64000782B7851800A560FEAE378EF27F074C12F
:10A6500026F175C127F1010E296F300E286F120007
:10A660000101300E7825D96EDA6A010EDA22F5CFB3
:10A67000DFFF782B120032C344F10101436B030169
:10A6800022512B0A04E1010E0101436F440701012D
:10A69000B8510BE0B851445D456F4551800A7F0FBA
:10A6A00004E345514327B8C144F1000146A647D011
:10A6B000EAEC2FF0D2EC2FF0D00E0101295D070E4D
:10A6C0002A59F8E3010E236F000E226B43C124F1D7
:10A6D00044C125F1FAEC07F001E3010C010E236FF0
:10A6E000110E226F43C124F144C125F1FAEC07F0A9
:10A6F00001E3020C010E236F220E226F43C124F1ED
:10A7000044C125F1FAEC07F001E3030C010E236FBD
:10A71000330E226F43C124F144C125F1FAEC07F056
:10A7200001E3040C020E236F410E226F43C124F19A
:10A7300044C125F1FAEC07F001E3050C000C010E11
:10A740000101426FFD0E176FA60E166F010E28EC69
:10A750001DF001014251300FA7EC2DF00D0EA7ECBA
:10A760002DF0D00E0101296F070E2A6F000E2B6B02
:10A770002C6B2D6B68EC9EF00101466F46512A0A46
:10A780006FE046510C0A6CE0466701D069D0465133
:10A79000150A66E14251050A01E01980880E01019F
:10A7A000296F130E2A6F2B6B2C6B010E2D6F68EC2B
:10A7B0009EF00101466B850E0101462556D8DF62E9
:10A7C00001D005D00101462B310E4665F4D70101B9
:10A7D000462B310E466501D043D0B8511DE046C12D
:10A7E00045F14551800A4E0F0AE2850E01014525CB
:10A7F0003CD8DF6201D003D00101452BF2D7010123
:10A800004551800A4E0F2CE2B851455F465145BF75
:10A8100003D0FF0A4525D8A046C145F1850E3E6FFD
:10A82000050E3F6F45513E27000E3F233EC11BF1F1
:10A830003FC11CF1220E406F030E416F4351402770
:10A84000000E412340C11DF141C11EF144C11FF161
:10A85000206BD5EC11F01C511B1102E1425112008A
:10A86000422B050E42656ED7000CD96EDA6A050ED2
:10A87000DA22220C01014A6B476B16D0330E4725B2
:10A88000D96EDA6A010EDA22DF6ADED847C130F10A
:10A89000302B330E3025E16EE26A010EE222DFCF6B
:10A8A000E7FF4A2B020E47272F514A63E7D72F5164
:10A8B0002F254A6F486B496B0DD0330E4825D96E52
:10A8C000DA6A010EDA22330E010148256EECF2F04D
:10A8D000484B492B4AC130F1316B4951800A326FE4
:10A8E0003051485D3151800A3259E7E3415025E04B
:10A8F000425023E0330E010199D8280EDF6E4A2B17
:10A90000412805E14A518AECF8F04A6F0BD0330E2A
:10A9100001018CD841C0DFFF4A2B330E87D842C0DB
:10A92000DFFF4A2B330E010181D8290EDF6E4A2B3F
:10A93000330E7CD8200EDF6E4A2B330E010176D801
:10A940002DC1E1FF2EC1E2FFE750306F30390F0B10
:10A9500030BFF00957EC2EF0DF6E4A2B75D8DF6A56
:10A960004A2B330E4A25D96EDA6A0301030EDA2226
:10A970002DC1E1FF2EC1E2FFE7500F0B57EC2EF087
:10A98000DF6E4A2B330E010151D810EE01F064D86E
:10A9900030BFF00957EC2EF0DF6E4A2B330E010169
:10A9A00045D810EE01F02D51E1262E51E222E7505C
:10A9B0000F0B57EC2EF0DF6E4A2B330E010136D809
:10A9C00010EE02F049D830BFF00957EC2EF0DF6EE0
:10A9D0004A2B330E01012AD810EE02F02D51E12648
:10A9E0002E51E222E7500F0B57EC2EF0DF6E4A2B70
:10A9F000330E01011BD810EE03F02ED830BFF00942
:10AA000057EC2EF0DF6E4A2B330E01010FD810EEFB
:10AA100003F02D51E1262E51E222E7500F0B57ECA7
:10AA20002EF0DF6E4A2B4AC1E7F312004A25D96E99
:10AA3000DA6A030EDA22DF6A4A2B330E4A25D96E10
:10AA4000DA6A030EDA221200330E01014A25D96EAA
:10AA5000DA6A030EDA2212002D51E1262E51E2228B
:10AA6000E750306F30390F0B1200E8CF57F112EC7E
:10AA700024F041501EE042501CE03F0E196FF70ECB
:10AA8000186FE7EC19F05E6F110E5E6501D05E6F16
:10AA90005E510DE10ED0A6ECDAF001015E51B0EC92
:10AAA0001BF004E341685EC142F003D05E075E67BD
:10AAB000F2D75751F8ECE9F016C15CF117C15DF11E
:10AAC000130E196F880E186FE7EC19F0566FDF0E32
:10AAD000566501D0566F56670FD0020197A10AD074
:10AAE0005CC12DF15DC12EF157C12FF13AECD4F0CC
:10AAF000D8801200D890120056C15EF13FD0A6EC6B
:10AB0000DAF001015E5139EC24F01FC15AF120C185
:10AB10005BF15E5100EC04F01FC158F120C159F106
:10AB20005829D8B4592902E05E0728D08DD8DF62B1
:10AB3000FBD720EE01F076D8DF62F6D720EE02F0E8
:10AB40005C51D9265D51DA2210EE02F077D8DF622F
:10AB5000EBD720EE03F05C51D9265D51DA2210EEDE
:10AB600003F06CD8DF62E0D75CC12DF15DC12EF13E
:10AB700057C12FF15E5149ECCCF0BAD75E67BFD711
:10AB800056C15EF14CD0A6ECDAF001015E5139EC11
:10AB900024F01FC15AF120C15BF15E5100EC04F0BA
:10ABA0001FC158F120C159F14FD8DF6237D020EED4
:10ABB00001F038D8DF6232D020EE02F05A51D926A7
:10ABC0005B51DA22DF50536F5915546F20EE02F0BB
:10ABD0005C51D9265D51DA22DF50556F5915541951
:10ABE0001DE120EE03F05A51D9265B51DA22DF50E5
:10ABF0005815536F20EE03F05C51D9265D51DA22CF
:10AC0000DF50581553190AE15CC12DF15DC12EF1D9
:10AC100057C12FF15E5149ECCCF06AD75E075E67F1
:10AC2000B2D75BD75C51D9265D51DA2210EE01F024
:10AC30005A51E1265B51E222E75012005A51E126B7
:10AC40005B51E222E75012005AC1D9FF5BC1DAFF23
:10AC5000DF505CC1D9FF5DC1DAFF12000301E8A13A
:10AC600068D0F70E0101176F240E166F010E28EC45
:10AC70001DF0E7C336F123EEE7F0640EDF6402D087
:10AC80000101366F0101386B51D0330E0101CFD86D
:10AC9000356F382B330ECBD8376F382B3551346F97
:10ACA0003751336F800E335D000E34590EE2373961
:10ACB0000F0B57EC2EF0A7EC2DF0010137510F0BC5
:10ACC00057EC2EF0A7EC2DF02ED033C130F134C16B
:10ACD00031F1060E326FD89031333033322FFBD73B
:10ACE00030511F0BC009356F33513F0B8009376F4F
:10ACF00035390F0B57EC2EF0A7EC2DF00101355133
:10AD00000F0B57EC2EF0A7EC2DF0010137390F0B8C
:10AD100057EC2EF0A7EC2DF0010137510F0B57EC3B
:10AD20002EF0A7EC2DF0020E0101365F3667ADD78D
:10AD30001DD0F70E0101176F160E166F010E28ECCD
:10AD40001DF00101386B330E010171D80FE0330E95
:10AD50003825D96EDA6A0301030EDA22DF50A7EC38
:10AD60002DF00101382B630E3865EDD7FE0E010181
:10AD7000176F730E166F000E28EC1DF049D868ECA3
:10AD80009EF0F30E0101176F2C0E166F010E28ECCA
:10AD90001DF0880E0101296F130E2A6F2B6B2C6B8F
:10ADA000010E2D6F68EC9EF03CD828EC1DF0600E73
:10ADB0000101296FEA0E2A6F2B6B2C6B010E2D6F90
:10ADC00068EC9EF025D868EC9EF0F40E0101176F38
:10ADD000470E166F010E28EC1DF01AD868EC9EF095
:10ADE0000101366F3651080A02E0D8901200B80E01
:10ADF000296F050E2A6F010E2B6F2C6B2D6F68ECDF
:10AE00009EF00101366F3651310AEFE1D880120011
:10AE1000880E0101296F130E2A6F2B6B2C6B2D6B83
:10AE2000000CFE0E0101176F740E166F000C382512
:10AE3000D96EDA6A030EDA22DF501200E8CF4BF146
:10AE4000496B4B39F00B4E6FBCA10CD0492B8DECEC
:10AE5000F3F0310E01012F6F4E5112ECE5F0C7D81F
:10AE6000C5EC1DF0BCA30CD0492B8DECF3F0320ED9
:10AE700001012F6F4E5112ECE5F0B9D8C5EC1DF071
:10AE8000BCA50CD0492B8DECF3F0330E01012F6FD4
:10AE90004E5112ECE5F0ABD8C5EC1DF0BCA70CD0C0
